:100000000C94AC1A0C94DD1A0C94DD1A0C94DD1AC5
:100010000C94DD1A0C94DD1A0C94DD1A0C94DD1A84
:100020000C94DD1A0C94DD1A0C94DD1A0C94DD1A74
:100030000C94DD1A0C94DD1A0C94DD1A0C94DD1A64
:100040000C94DD1A0C94EDEF0C94DD1A0C94DD1A6F
:100050000C94DD1A0C94DD1A0C9452DB0D94C22B17
:100060000C94DD1A0C94604A0C94564A0C94DD1AD8
:100070000C94DD1A0C94DD1A0C94DD1A0C94DD1A24
:100080000C94D32C0C94DD1A0C94DD1A0C94DD1A0C
:100090000C94DD1A0C94DD1A0C94DD1A0C94DD1A04
:1000A0000C94DD1A0C94DD1A0C94A52C0C94DD1A1A
:1000B0000C94DD1A0C94DD1A0C94DD1A0C94DD1AE4
:1000C0000C94DD1A0C94DD1A0C94DD1A0C94882D16
:1000D0000C94522D0C94DD1A0C94DD1A0C94DD1A3C
:1000E0000C94DD1A084AD73B3BCE016E84BCBFFDA1
:1000F000C12F3D6C74319ABD56833DDA3D00C77FF8
:1001000011BED9E4BB4C3E916BAAAABE0000008090
:100110003F05A84CCDB2D44EB93836A9020C50B91F
:10012000918688083CA6AAAA2ABE000000803F004B
:100130000C941A2E0D94AA0F0D9433220C94064B96
:100140000C9488C10C94392E0D94020F0D94C21E8C
:100150000D949F1E0C9427BF0C943DC30D948C22CC
:100160000D94CD0F0D9468230D947F220C94B9ABA0
:100170000D94D70F0D947C130D94371F0D943C24D0
:100180000D94F41D0C94DC4A0D94F51E0D940F1C77
:100190000D94680F0C944C2E0C945EAC0C949E4AFB
:1001A0000C94222E0D94F3150D948C0F0D94E10FE9
:1001B0000D94FC0E0D94E40E0D947C0F0C9465C20E
:1001C0000D9432320C9400C20D94140F0C9426BF7F
:1001D0000D94C30E0C94042E0D94D61E0D94C416CB
:1001E0000C9480C20C942E2E0C94CD4A0D94921C2B
:1001F0000D942D220C94442E0C94132E0C942A2E24
:100200000C940A4B0D941C270D94BE1D0D94EE0EFC
:100210000D9461140D94621E0C941C4B0D944A1F96
:100220000C94244B0D94B90F0D94E10E0C94EB4AF1
:100230000D948B1E0D9436220D940A0F0C94F24AE5
:100240000C94F64A0C9421C20C94322E0D94590F42
:100250000D9450320D94BE0E0C94FE4A0D94510F25
:100260000C94E5AB0C9407C40D94F80E0D94C91AC8
:100270000D945B120D94D50E0C949EA90C9410C392
:100280000D94EB0F0D94D90E0C946BC10C94A4BE7D
:100290000D94060F0C94C62D0D94720F0D94840FBF
:1002A0000D94100F0D945E0F0C94FEC20D94960FDA
:1002B0000D942E1D0D94DD0E0D94A00F0D94522261
:1002C0000C94262E0D9461220C94EDA90C94F52D1E
:1002D0000D948B140D94F40E0D9442180D94FB1F85
:1002E0000C9426AC0D9479230C94F1A90D94EA0E8C
:1002F0000C94FA4A0D945E1C0C94024B0D94421C13
:100300000C94114B0C941E2E0D9406220D94C30FC9
:100310000D946B224E414E494E495459494E46CD9B
:10032000CCCC3D0AD7233C17B7D13877CC2B3295AC
:1003300095E6241FB14F0A000020410000C842008A
:10034000401C4620BCBE4CCA1B0E5AAEC59D740054
:10035000407A10F35A00A0724E18090010A5D4E894
:100360000000E87648170000E40B54020000CA9A27
:100370003B000000E1F50500008096980000004079
:10038000420F000000A086010000001027000000BE
:1003900000E803000000006400000000000A000004
:1003A0000000000100000000002C76D888DC674FB8
:1003B0000823DFC1DFAE59E1B1B796E5E3E453C6E8
:1003C0003AE651997696E8E6C28426EB898C9B62E0
:1003D000ED407C6FFCEFBC9C9F40F2BAA56FA5F48A
:1003E00090055A2AF75C936B6CF9676DC11BFCE0B2
:1003F000E40D47FEF520E6B500D0ED902E03009405
:100400003577050080841E080000204E0A00000099
:10041000C80C333333330F986E12831141EF8D21A3
:1004200014893BE65516CFFEE6DB18D1844B381B0A
:10043000F77C1D901DA4BBE424203284725E2281CF
:1004400000C9F124ECA1E53D27434F4D4D554E49E0
:10045000434154494F4E0044525952554E00455263
:10046000524F525300494E464F004543484F0045B6
:1004700072726F722077726974696E6720746F2070
:10048000454550524F4D210A0053544F505045445A
:100490002E20005072696E7465722073746F7070D4
:1004A00065642064756520746F206572726F727365
:1004B0002E2046697820746865206572726F7220FC
:1004C000616E6420757365204D39393920746F2051
:1004D000726573746172742E202854656D70657234
:1004E00061747572652069732072657365742E205E
:1004F0005365742069742061667465722072657337
:1005000074617274696E67290A004E6F20436865D2
:10051000636B73756D2077697468206C696E6520F4
:100520006E756D6265722C204C617374204C696E1F
:10053000653A20004E6F20436865636B73756D20CC
:1005400077697468206C696E65206E756D6265727E
:100550002C204C617374204C696E653A20006368EE
:1005600065636B73756D206D69736D617463682C61
:10057000204C617374204C696E653A20004C696EA2
:1005800065204E756D626572206973206E6F7420F0
:100590004C617374204C696E65204E756D62657296
:1005A0002B312C204C617374204C696E653A20000D
:1005B0004D3131300053657269616C207374617420
:1005C0007573206D69736D617463680A0077616982
:1005D000740A0053442072656164206572726F7200
:1005E0000A002121204B494C4C20636175736564DE
:1005F00020627920746F6F206D75636820696E6169
:1006000063746976652074696D65202D2063757249
:1006100072656E7420636F6D6D616E643A20004880
:100620006F74656E642049646C652054696D656FF4
:10063000757400486F74656E642049646C6520545D
:10064000696D656F75740A002A2A2A496E69746992
:100650006E672063617264206973204F4B2A2A2AD7
:10066000004D6564696120496E736572746564004C
:100670004D656469612052656D6F766564004D312A
:100680003030305300627573793A2070617573654C
:100690006420666F7220696E7075740A00627573EB
:1006A000793A2070617573656420666F7220757386
:1006B00065720A00627573793A2070726F636573B0
:1006C00073696E670A002A2A2A6B696C6C2A2A2AC7
:1006D00000706F7765726F6666004B494C4C4544FD
:1006E0002E20005072696E7465722068616C7465AA
:1006F000642E206B696C6C28292063616C6C6564C6
:10070000210A0053544F505045442E200050726926
:100710006E7465722073746F7070656420647565A3
:1007200020746F206572726F72732E204669782074
:10073000746865206572726F7220616E64207573D3
:1007400065204D39393920746F2072657374617278
:10075000742E202854656D70657261747572652001
:1007600069732072657365742E20536574206974F3
:100770002061667465722072657374617274696E4B
:1007800067290A006563686F3A004572726F723AB2
:100790000042696C696E656172204C6576656C69B2
:1007A0006E6720477269643A0A0021212053544F32
:1007B000502063616C6C656420626563617573656C
:1007C000206F6620424C546F756368206572726FAB
:1007D00072202D2072657374617274207769746859
:1007E000204D3939390A0021212053544F502063BC
:1007F000616C6C65642062656361757365206F660A
:1008000020424C546F756368206572726F72202DA0
:1008100020726573746172742077697468204D3931
:1008200039390A002F2F616374696F6E3A00656E63
:10083000640053656E64204D31303820746F20722F
:100840006573756D650A00496E736572742066691B
:100850006C616D656E7420616E642073656E6420DA
:100860004D3130380A005265686561742066696EE2
:1008700069736865642E0052656865617420446F11
:100880006E6500526568656174696E672E2E2E0074
:1008900052656865617400486561746572205469C9
:1008A0006D656F75740053656E64204D313038206E
:1008B000746F2068656174206E6F7A7A6C650A00C7
:1008C0004E6F7A7A6C65205061726B656400486F78
:1008D00074656E6420746F6F20636F6C640A0070BF
:1008E000617573656400506175736500507572675A
:1008F000654D6F7265005061757365640070726F4D
:100900006D70745F0073686F7700627574746F6EDA
:1009100000626567696E004C6F61642046696C61B6
:100920006D656E74004C6F61642046696C616D6525
:100930006E74205400496E736572742066696C6130
:100940006D656E7420616E642073656E64204D3138
:1009500030380A00726573756D6564005265737591
:100960006D696E670057616974696E6720666F72A2
:10097000206865617475702E0A004C656176696E39
:100980006720473236003F53706563696669656466
:1009900020582C5920636F6F7264696E61746520F2
:1009A0006F7574206F6620626F756E64732E0A0017
:1009B0003F28522965706561742076616C756520E9
:1009C0006E6F7420706C61757369626C653B206D2D
:1009D000757374206265206174206C656173742086
:1009E000312E0A003F2852296570656174206D75AB
:1009F000737420626520737065636966696564203D
:100A00007768656E206E6F74207573696E672061FC
:100A10006E204C43442E0A003F537065636966693B
:100A20006564206E6F7A7A6C652074656D7065728E
:100A30006174757265206E6F7420706C6175736976
:100A4000626C652E0A003F53706563696669656470
:100A50002066696C616D656E742073697A65206EBD
:100A60006F7420706C61757369626C652E0A003F4B
:100A7000537065636966696564207072696D65208D
:100A80006C656E677468206E6F7420706C6175732E
:100A900069626C652E0A003F5072696D65206C6555
:100AA0006E677468206D757374206265207370655D
:100AB000636966696564207768656E206E6F74206F
:100AC0007573696E6720616E204C43442E0A003FA7
:100AD000537065636966696564206E6F7A7A6C65C8
:100AE0002073697A65206E6F7420706C617573690C
:100AF000626C652E0A003F52657472616374696F9F
:100B00006E204D756C7469706C696572206D7573BB
:100B100074206265207370656369666965642E0A76
:100B2000003F53706563696669656420526574723D
:100B3000616374696F6E204D756C7469706C696562
:100B400072206E6F7420706C61757369626C652EB3
:100B50000A003F537065636966696564206C61795A
:100B6000657220686569676874206E6F7420706CA8
:100B700061757369626C652E0A0043292E0A003F75
:100B80005370656369666965642062656420746595
:100B90006D7065726174757265206E6F7420706C13
:100BA00061757369626C65202834302D00473236D8
:100BB000207374617274696E672E2E2E0A004F4680
:100BC000460A0046616465204865696768742000CC
:100BD000426564204C6576656C696E6720004661ED
:100BE000696C656420746F20656E61626C6520427B
:100BF0006564204C6576656C696E670A00496E769F
:100C0000616C6964206D6573682E0A0050726F62B2
:100C1000696E6720506F696E740025532025692F17
:100C20002569002E0A002F0050726F62696E6720DE
:100C30006D65736820706F696E74200020284452BF
:100C40005952554E2900473239204175746F204260
:100C50006564204C6576656C696E67003F20284CA2
:100C60002C522C462C4229206F7574206F6620620E
:100C70006F756E64732E0A003F2856296572626F85
:100C80007365206C6576656C20696D706C61757339
:100C900069626C652028302D34292E0A0042616477
:100CA000205A2076616C75650A004E6F2062696C6F
:100CB000696E65617220677269640A0044657669CD
:100CC0006174696F6E0025533A2025730046696E82
:100CD0006973686564210A003A207A3A2000206F1F
:100CE000662000476F696E6720746F3A2058004392
:100CF000570A00206469723A0020616E676C653A99
:100D0000005374617274207261646975733A004DA6
:100D1000343820506F696E740025533A2025642FB3
:100D2000256400506F736974696F6E696E67207413
:100D300068652070726F62652E2E2E0A003F4C652A
:100D40006773206F66206D6F76656D656E742069C0
:100D50006D706C61757369626C652028302D31355A
:100D6000292E0A003F2028582C5929206F757420FD
:100D70006F6620626F756E64732E0A0050726F6228
:100D800065206F7574206F6620626F756E647300E6
:100D90003F53616D706C652073697A65206E6F7466
:100DA00020706C61757369626C652028342D353054
:100DB000292E0A004D3438205A2D50726F6265205A
:100DC0005265706561746162696C697479205465FB
:100DD00073740A003F2856296572626F7365206C30
:100DE0006576656C20696D706C61757369626C65A0
:100DF0002028302D34292E0A005374616E646172EC
:100E00006420446576696174696F6E3A20002052EF
:100E1000616E67653A2000204D61783A2000204DD0
:100E2000696E3A2000205369676D613A20004D6574
:100E3000616E3A20005741524E494E4721204C6F77
:100E400077205A204A65726B206D6179206C65614C
:100E50006420746F20756E77616E746564207061B4
:100E6000757365732E0A00546F6F6C6368616E67EB
:100E7000653A0020204D32313700205700204C00C9
:100E8000204100204700204600205500205200202D
:100E9000530020204D61783A2000200020204D6929
:100EA0006E3A2000536F667420656E6473746F70C1
:100EB000733A20002E0A002028302D3130290020DE
:100EC00076616C7565206F7574206F662072616E37
:100ED000676500416476616E6365204B003D3D4F60
:100EE0006E506F7765724C6F7373526573756D6575
:100EF0003D3D004D32342053256C642054256C64F4
:100F0000004739322E3920452573004731204625C8
:100F100064004739322E39205A2573004731205A50
:100F20003020463230300047312058257320592573
:100F30007320463330303000473132004D34323088
:100F400020532569205A2573004D31303620502515
:100F50006920532569005425692053004D323030F3
:100F600020542569204430004D323030205425690A
:100F700020442573004732385230585900473932DF
:100F80002E39204530205A300A47315A2573004DFA
:100F900031303920532569004D31393020532569CE
:100FA000004D343230205330205A300020496E76C4
:100FB000616C69642065787472756465722000479D
:100FC000322F47332062616420706172616D6574F5
:100FD0006572730A00536C6565702E2E2E005A20C0
:100FE00050726F62652050617374204265640A001C
:100FF0005A2050726F62652050617374204265649C
:10100000004732384C30004D3131372050726F621A
:1010100065206661696C65642E0A4732380A007083
:10102000726F62655F72657769706500473239205B
:101030005265747279696E670050726F62696E678B
:10104000204661696C6564004D313137204265642A
:10105000206C6576656C696E67206661696C656495
:101060002E0A4730205A31300A4D3330302050326A
:101070003520533838300A4D333030205035302049
:1010800053300A4D33303020503235205338383009
:101090000A4D333030205035302053300A4D333034
:1010A000302050323520533838300A4D333030201C
:1010B0005035302053300A47342053310070726F5E
:1010C00062655F6661696C6564004D31313720424D
:1010D0006564206C6576656C696E6720646F6E650B
:1010E0002E00205A3A200020593A20004265642000
:1010F000583A20004D65736820706F696E74206FD8
:101100007574206F662072616E67650A004D30202D
:1011100053746F70004D312053746F7000436F6EC5
:1011200074696E756500436C69636B20746F20523F
:101130006573756D652E2E2E004E6F204D6F766592
:101140002E00456E642066696C65206C6973740AB4
:1011500000426567696E2066696C65206C6973740E
:101160000A004E6F206D656469610A0052657375EF
:101170006D696E6720534400286E6F2066696C6548
:10118000290043757272656E742066696C653A2039
:10119000005072696E742074696D653A20000A53BC
:1011A000746174733A2046696C616D656E74207564
:1011B0007365643A20002C204C6F6E676573742051
:1011C0006A6F623A2000546F74616C2074696D65B7
:1011D0003A200053746174733A20002C20466169F0
:1011E0006C65643A20002C2046696E6973686564FA
:1011F0003A20005072696E74733A2000537461741F
:10120000733A20006F6B006F6666006A0465045EC7
:10121000045704490444454255473A004D3131339F
:1012200020530042656420436F6F6C696E672E2EF9
:101230002E004265642048656174696E672E2E2E0B
:1012400000544D33442043522D58204F46462E0023
:101250002F2F00205200416363656C6572617469D1
:101260006F6E3A2050004D32303620580046523AC8
:101270000020466C6F773A20003A200020536572B8
:10128000766F2000206F7574206F662072616E6724
:10129000650A00536572766F200020643A00206969
:1012A0003A0020703A00496E76616C696420657876
:1012B0007472756465720A0020643A0020693A000D
:1012C00020703A0064697300656E0043290A00616A
:1012D000626C656420286D696E2074656D702000F5
:1012E000436F6C64206578747275646573206172F5
:1012F000652000504944204175746F74756E650017
:10130000504944204175746F74756E65206661693B
:101310006C65642120426164206865617465722097
:1013200069640A004D34323120696E636F727265F0
:10133000637420706172616D65746572207573618C
:1013400067650A004D65736820706F696E74206F61
:101350007574206F662072616E67650A004F66665D
:1013600073657473204170706C69656400457272B6
:101370003A20546F6F206661722100546F6F2066AF
:1013800061722066726F6D207265666572656E634C
:101390006520706F696E740A00454550524F4D20AC
:1013A0004F4B0A004F4646004F4E00506F77657214
:1013B0002D6C6F7373207265636F76657279200090
:1013C0004D383400446F6E65207072696E74696EBA
:1013D000672066696C650A004D3737004D33310070
:1013E0004361703A004D4541545041434B00434FD7
:1013F0004F4C45525F54454D50455241545552450E
:10140000004348414D4245525F54454D504552417D
:101410005455524500424142595354455050494E4B
:10142000470041524353004D4F54494F4E5F4D4F7B
:1014300044455300544845524D414C5F50524F541F
:10144000454354494F4E004C4F4E475F46494C452B
:101450004E414D45004155544F5245504F52545FF7
:1014600053445F5354415455530053445F575249BA
:101470005445005245504541540053444341524461
:101480000050524F4D50545F535550504F525400DE
:10149000454D455247454E43595F50415253455281
:1014A00000434153455F4C494748545F42524947C6
:1014B00048544E45535300544F47474C455F4C49A1
:1014C0004748545300534F4654574152455F504F7D
:1014D000574552004255494C445F50455243454E92
:1014E00054004C4556454C494E475F4441544100D9
:1014F0005A5F50524F42450052554E4F555400418D
:1015000055544F4C4556454C005052494E545F4A35
:101510004F420050524F4752455353004155544F8C
:101520005245504F52545F54454D5000564F4C5504
:101530004D455452494300454550524F4D00424994
:101540004E4152595F46494C455F5452414E5346B5
:1015500045520053455249414C5F584F4E5F584FDA
:101560004646004649524D574152455F4E414D4512
:101570003A4D61726C696E20322E302E375F4457BF
:10158000372E3320544D33442053534D4442422090
:101590002841707220323420323032312031393AD1
:1015A00035353A33342920534F555243455F434F25
:1015B00044455F55524C3A68747470733A2F2F67E4
:1015C00069746875622E636F6D2F496E73616E6901
:1015D00074794175746F6D6174696F6E2F4D6172AE
:1015E0006C696E2F747265652F437265616C6974E6
:1015F000794477696E5F322E302050524F544F43FA
:101600004F4C5F56455253494F4E3A312E30204D84
:10161000414348494E455F545950453A544D33442F
:101620002043522D582045585452554445525F434B
:101630004F554E543A3220555549443A63656465D6
:10164000326132662D343161322D343734382D39E0
:101650006231322D6335356336326633363766662E
:101660000A0050726F6265204F6666736574205A77
:101670000050726F6265204F6666736574205A0071
:10168000290A0020746F20003F5A206F7574206F64
:10169000662072616E6765202800290A0020746F39
:1016A00020003F59206F7574206F662072616E674D
:1016B0006520282D00290A0020746F20003F582043
:1016C0006F7574206F662072616E676520282D002B
:1016D00050726F6265204F666673657420580043D0
:1016E000616E6E6F74206F70656E207375626469D1
:1016F0007220002569730025696D20256973002516
:1017000069682025696D2025697300256964202595
:1017100069682025696D2025697300256979202570
:101720006964202569682025696D20256973003D5D
:101730003D4477696E20496E697420436F6D706C0B
:101740006574653D3D002A2A2A4E6F7A7A6C65548D
:10175000656D705374617475735B325D203D003D3F
:101760003D48656174696E6720446F6E652043680B
:10177000616E67652046696C616D656E743D3D0004
:101780002020737461727470726F67726573732056
:10179000003D3D7761697477617920353D3D003DBD
:1017A0003D7761697477617920343D3D003D3D7737
:1017B00061697477617920333D3D003D3D77616912
:1017C0007477617920313D3D003D3D6F6E50726907
:1017D0006E7454696D657253746F707065643D3DCD
:1017E000003D3D6F6E466163746F7279526573653B
:1017F000743D3D00270A0A0000272027002027000B
:101800002D006E6F74696669636174696F6E200084
:1018100063616E63656C005072696E742041626F23
:1018200072746564004469736D697373005549206F
:1018300041626F7274656400726573756D65002A2C
:101840002A2A43506C617920546F6E652A2A2A0037
:101850005761726E696E673A20436C65616E204312
:101860006972636C65207265717569726573205861
:10187000590A005761726E696E673A205261646955
:101880007573204F7574206F662052616E67650A0C
:10189000004E6F7A7A6C6520746F6F20636F6C6492
:1018A000202D20536B697070696E672077697065B1
:1018B0000A003D3D6F6E5072696E7454696D6572B9
:1018C0005061757365643D3D00486F6D696E6720BA
:1018D0004661696C6564006F70656E0054524947DB
:1018E0004745524544003A20007A5F6D696E0079A1
:1018F0005F6D696E00785F6D696E005265706F7222
:1019000074696E6720656E6473746F7020737461A0
:101910007475730A0000809D4300009A430000C85C
:101920004300000000000000000000000020746F71
:101930006F206C6F6E6720657874727573696F6E57
:101940002070726576656E7465640A0020636F6C42
:101950006420657874727573696F6E207072657635
:10196000656E7465640A00486F6D65202573257384
:101970002573204669727374005761726E696E67D1
:101980003A20486F6D696E672042756D702044691A
:101990007669736F72203C20310A00020204000055
:1019A0000000000000000000000000809D430000D7
:1019B0009A430000C84300000041000000410000BD
:1019C0000040FFFFFF000000010000000100008058
:1019D00000555555000000400033333300AAAA2AB1
:1019E000004992240000002000C7711C0099991939
:1019F00000D1451700555515003BB113002449127D
:101A00000011111100000010000F0F0F00E3380E3D
:101A10000043790D00CCCC0C00C3300C00E8A20BC5
:101A20000064210B00AAAA0A00703D0A009DD80993
:101A300000427B090092240900DCD3080088880852
:101A4000001042080000000800F0C1070087870767
:101A50000075500700711C07003EEB0600A1BC0694
:101A6000006990060066660600703E060061180672
:101A70000017F4050074D105005BB00500B29005B5
:101A800000627205005555050078390500B81E053D
:101A900000050505004EEC040087D40400A1BD0438
:101AA0000090A7040049920400C17D0400EE69047F
:101AB00000C7560400444404005C320400082104BA
:101AC0000041100400000004003FF00300F8E003B0
:101AD0000026D20300C3C30300CCB503003AA80319
:101AE000000A9B0300388E0300C08103009F75032A
:101AF00000D0690300505E03001D53030034480307
:101B000000913D03003333030016290300381F03FF
:101B10000097150300300C0300030303000BFA02C7
:101B20000049F10200BAE802005CE002002DD80290
:101B3000002DD0020059C80200B0C0020031B90225
:101B400000DAB10200AAAA0200A0A30200BC9C0213
:101B500000FA9502005C8F0200DF88020082820298
:101B600000457C02002776020027700200436A02CB
:101B7000007C640200D05E02003F590200C853029C
:101B800000FFFDFCFAF8F6F4F2F0EEECEAE9E7E526
:101B9000E3E1E0DEDCDAD9D7D5D4D2D0CFCDCBCAE1
:101BA000C8C7C5C3C2C0BFBDBCBAB9B7B6B4B3B26B
:101BB000B0AFADACAAA9A8A6A5A4A2A1A09E9D9CC9
:101BC0009A99989795949392908F8E8D8B8A898805
:101BD000878684838281807F7E7D7B7A7978777621
:101BE0007574737271706F6E6D6C6B6A696867661D
:101BF0006564636261605F5E5D5C5B5A595858570B
:101C000056555453525150504F4E4D4C4B4A4A49E1
:101C100048474646454443424241403F3E3E3D3CA4
:101C20003B3B3A3938383736353534333232313058
:101C3000302F2E2E2D2C2B2B2A29292827272625FD
:101C40002524232322212120201F1E1E1D1C1C1B96
:101C50001B1A191918181716161515141313121222
:101C60001111100F0F0E0E0D0D0C0C0B0A0A0909A5
:101C7000080807070606050504040303020201001D
:101C80000020746F6F206C6F6E67206578747275BA
:101C900073696F6E2070726576656E7465640A0094
:101CA00020636F6C6420657874727573696F6E2041
:101CB00070726576656E7465640A003D3D6F6E50A6
:101CC00072696E7454696D6572537461727465647F
:101CD0003D3D003D3D6F6E53746F72655365747486
:101CE000696E67733D3D003D3D6F6E436F6E666983
:101CF0006775726174696F6E53746F72655772693C
:101D00007474656E3D3D0053657474696E6773202D
:101D100053746F726564000A20696E6974207A706A
:101D2000726F62655F7A6F6666736574203D20002E
:101D30003D3D6F6E436F6E66696775726174696F62
:101D40006E53746F7265526561643D3D0045455048
:101D5000524F4D20496E697469616C697A65640AF5
:101D6000003B20003A0A0020204D3630332000543A
:101D70006F6F6C2D6368616E67696E673A002055FE
:101D8000005431204C002055005430204C0046694E
:101D90006C616D656E74206C6F61642F756E6C6F15
:101DA0006164206C656E677468733A00204B002094
:101DB000204D3930302054004C696E6561722041ED
:101DC0006476616E63653A0020204D3835312058C5
:101DD000005A2D50726F6265204F666673657400FD
:101DE00020204D343133205300506F7765722D4CD5
:101DF0006F7373205265636F766572793A00204481
:101E00000020490020204D33303420500020440071
:101E100020490020204D33303120500050494420CB
:101E200073657474696E67733A00204A0020204716
:101E30003239205720490020204D343230205300C1
:101E40004175746F20426564204C6576656C696EDF
:101E5000673A0020204D323036205800486F6D65BB
:101E6000206F66667365743A002058002053002086
:101E7000204D323035204200416476616E636564E6
:101E80003A20423C6D696E5F7365676D656E745F85
:101E900074696D655F75733E20533C6D696E5F6656
:101EA000656564726174653E20543C6D696E5F7453
:101EB000726176656C5F66656564726174653E200B
:101EC000583C6D61785F785F6A65726B3E20593C63
:101ED0006D61785F795F6A65726B3E205A3C6D6117
:101EE000785F7A5F6A65726B3E20453C6D61785F12
:101EF000655F6A65726B3E0020540020520020200E
:101F00004D323034205000416363656C65726174FA
:101F1000696F6E2028756E6974732F7332293A20A9
:101F2000503C7072696E745F616363656C3E2052F1
:101F30003C726574726163745F616363656C3E20BB
:101F4000543C74726176656C5F616363656C3E00DE
:101F500020204D3230312058004D6178696D756D0B
:101F600020416363656C65726174696F6E202875CA
:101F70006E6974732F7332293A0020204D3230334A
:101F80002058004D6178696D756D206665656472D5
:101F9000617465732028756E6974732F73293A0014
:101FA00053746570732070657220756E69743A00A1
:101FB00020204D32303020530020440020204D326C
:101FC00030302054002044697361626C65640A00FB
:101FD00046696C616D656E742073657474696E67B3
:101FE000733A0020286D6D290020204732312020CF
:101FF00020203B20556E69747320696E206D6D0042
:102000003D3D6F6E4C6F616453657474696E6773A8
:102010003D3D000000FA430000FA4300002041006B
:102020000096420000A0420000A0420000C8430009
:1020300000BE42DC050000DC050000640000004B2F
:1020400000000024F4D43050C38E20C2A240178276
:102050008B7011127A910D816CD90AA861E108C7C1
:10206000586607615143061E4B5D05C145A7041A1A
:10207000411104093D9803713931034036DB026593
:10208000339102D4305402802E1D02632CEE017570
:102090002AC501B028A001102781018F2564012BDA
:1020A000244B01E0223401AC211F018D200D018061
:1020B0001FFC00841EED00971DDF00B81CD200E657
:1020C0001BC600201BBC00641AB200B219A8000A8B
:1020D00019A0006A189900D117910040178B00B51C
:1020E00016840031167E00B31579003A157300C7C7
:1020F000146F0058146A00EE1366008813630025FD
:10210000135E00C7125B006C12570015125400C119
:1021100011510070114F0021114B00D61049008D54
:102120001047004610440002104200C00F400080DB
:102130000F3E00420F3C00060F3B00CB0E380093D1
:102140000E37005C0E3500270E3400F30D3200C14F
:102150000D3100900D3000600D2E00320D2D000568
:102160000D2C00D90C2B00AE0C2900850C29005C2D
:102170000C2700350C27000E0C2600E80B2400C4A9
:102180000B2400A00B23007D0B23005A0B210039E8
:102190000B2100180B2000F80A1F00D90A1E00BBF3
:1021A0000A1E009D0A1D00800A1D00630A1C0047CC
:1021B0000A1B002C0A1B00110A1A00F7091A00DD7D
:1021C000091900C4091900AB091900920917007B0D
:1021D000091800630917004C09160036091600207B
:1021E0000916000A091500F5081500E0081400CCCE
:1021F000081400B8081400A4081400900813007D07
:102200000812006B08130058081200460812003428
:10221000081100230811001208110001081100F034
:10222000071000E0071000D0071000C0071000B032
:10223000070F00A107100091070E0083070F00741D
:10224000070F0065070E0057070E0049070E003BF9
:10225000070D002E070E0020070D0013070D0006C6
:10226000070D00F9060C00ED060D00E0060C00D489
:10227000060C00C8060C00BC060C00B0060C00A43E
:10228000060B0099060C008D060B0082060B0077EA
:10229000060B006C060B0061060A0057060B004C8B
:1022A000060A0042060A0038060A002E060A002422
:1022B000060A001A060A001006090007060A00FDB1
:1022C000050900F4050900EB050900E2050900D93C
:1022D000050900D0050900C7050900BE050900B5BC
:1022E000050800AD050800A50509009C0508009437
:1022F0000508008C050800840508007C05080074AA
:102300000508006C050700650508005D0507005617
:102310000508004E0507004705070040050800387E
:10232000050700310507002A050700230507001CE3
:10233000050600160507000F050700080506000240
:10234000050700FB040600F5040700EE040600E89C
:10235000040600E2040700DB040600D5040600CFF3
:10236000040600C9040600C3040600BD040600B745
:10237000040600B1040500AC040600A6040600A093
:102380000405009B04060095040500900406008ADD
:1023900004050085040500800406007A0405007524
:1023A000040500700405006B040500660405006167
:1023B0000405005C04050057040500520405004DA7
:1023C00004050048040500430405003E0404003AE7
:1023D00004050035040500300404002C0405002722
:1023E000040400230405001E0404001A040400165B
:1023F000040500110404000D040400090405000490
:1024000004040000040400FC030400F8030400F4C6
:10241000030400F0030400EC030400E8030400E4F8
:10242000030400E0030400DC030400D8030400D428
:10243000030400D0030400CC030400C8030300C558
:1024400003030024F404D9201BC40C5C0E9804C4BC
:10245000095F0265077101F405F900FB04B3004848
:10246000048700C10369005803550003034500BEFB
:10247000023A008402310053022A00290225000496
:10248000022000E4011C00C8011900AF01170098E8
:10249000011400840113007101100061011000514A
:1024A000010E0043010D0036010B002B010B002033
:1024B000010B00150109000C01090003010800FBD4
:1024C000000800F3000800EB000700E4000600DE4F
:1024D000000600D8000600D2000600CC000500C7A8
:1024E000000500C2000500BD000400B9000400B5ED
:1024F000000400B1000400AD000400A9000400A520
:10250000000300A20003009F0004009B000300984A
:102510000003009500020093000300900003008D6B
:102520000002008B00030088000200860002008485
:10253000000300810002007F0002007D0002007B9A
:1025400000020079000200770001007600020074AA
:1025500000020072000100710002006F0002006DB5
:102560000001006C0002006A0001006900020067BF
:1025700000010066000100650001006400020062C5
:1025800000010061000100600001005F0002005DC9
:102590000001005C0001005B0001005A00010059CD
:1025A00000010058000100570001005600010055CD
:1025B00000010054000100530000005300010052CC
:1025C00000010051000100500001004F0001004EC9
:1025D0000000004E0001004D0001004C0001004BC6
:1025E0000000004B0001004A0001004900010048C2
:1025F00000000048000100470001004600000046BE
:1026000000010045000000450001004400010043B6
:1026100000000043000100420000004200010041B0
:1026200000000041000100400001003F0000003FA9
:102630000001003E0000003E0001003D0000003DA2
:102640000001003C0000003C0000003C0001003B99
:102650000000003B0001003A0000003A0001003990
:102660000000003900010038000000380000003888
:10267000000100370000003700010036000000367E
:102680000000003600010035000000350000003574
:102690000001003400000034000000340001003369
:1026A000000000330000003300010032000000325F
:1026B0000000003200010031000000310000003154
:1026C0000001003000000030000000300001002F49
:1026D0000000002F0000002F0000002F0001002E3E
:1026E0000000002E0000002E0001002D0000002D33
:1026F0000000002D0000002D0001002C0000002C27
:102700000000002C0000002C0001002B0000002B1A
:102710000000002B0000002B0001002A0000002A0E
:102720000000002A0000002A000100290000002902
:1027300000000029000000290000002900010028F5
:1027400000000028000000280000002800000028E9
:1027500000010027000000270000002700000027DC
:1027600000000027000100260000002600000026CF
:1027700000000026000000260001002500000025C2
:1027800000000025000000250000002500000025B5
:1027900000010024000000240000002400000024A8
:1027A000000000240001002300000023000000239B
:1027B000000000230000002300000023000000238D
:1027C0000001002200000022000000220000002280
:1027D0000000002200000022000100210000002172
:1027E0000000002100000021000000210000002165
:1027F0000000002100010020000000200000002057
:102800000000002000000020000000200000002048
:10281000000000200001001F0000001F0000001F3A
:102820000000001F0000001F0000001F0000001F2C
:102830000001001E0000001E0000001E0000001E1F
:10284000000000232C0000B8220000561800003AB7
:102850000F0000B8080000B1040000710200003E43
:1028600001000020436F756E7420583A00236465A0
:1028700066696E652044454641554C545F000062D0
:102880006564004B6420004B6920004B70200050B1
:102890004944204175746F74756E652066696E6970
:1028A00073686564212050757420746865206C61BC
:1028B0007374204B702C204B6920616E64204B6434
:1028C00020636F6E7374616E74732066726F6D2017
:1028D00062656C6F7720696E746F20436F6E6669F6
:1028E0006775726174696F6E2E680A0050494420E2
:1028F0004175746F74756E65206661696C656421DD
:102900002074696D656F75740A00504944204175E3
:10291000746F74756E65206661696C6564212054FE
:10292000656D706572617475726520746F6F206873
:102930006967680A00204B643A2000204B693A20FE
:1029400000204B703A200020436C61737369632050
:10295000504944200A00204E6F206F7665727368DC
:102960006F6F740A002054753A2000204B753A208E
:1029700000206D61783A2000206D696E3A200020B9
:10298000643A200020626961733A20005049442073
:102990004175746F74756E652073746172740A008A
:1029A000504944204175746F74756E652066616985
:1029B0006C6564212054656D706572617475726513
:1029C00020746F6F20686967680A0042656400457B
:1029D0003100626564002C2073797374656D207317
:1029E000746F7070656421204865617465725F4919
:1029F000443A200048656174696E67204661696CDD
:102A000065640048656174696E67206661696C651C
:102A100064004D3131322053687574646F776E00F5
:102A20001000C90210012C0140012201700118019F
:102A3000B0010E01F00104015002FA00B002F000F2
:102A40003003E600D003DC009004D2007005C8001B
:102A5000A006BE000008B400B009AA00D00BA00078
:102A6000600E960060118C0000158200201978001D
:102A7000C01D6E00A0226400B0275A00902C5000A8
:102A800000314600E0343C0010383200903A280013
:102A9000603C1E00A03D1400803E0A00203F000064
:102AA000544845524D414C2052554E4157415900D2
:102AB000546865726D616C2052756E617761790042
:102AC0004572723A204D415854454D50004D415881
:102AD00054454D502074726967676572656400459E
:102AE00072723A204D494E54454D50004D494E5456
:102AF000454D502074726967676572656400202FC8
:102B0000002042403A0020403A0020573A00205727
:102B10003A00496E76616C696420657874727564F8
:102B200065720A0041637469766520457874727530
:102B30006465723A2000486F74656E6420746F6F2C
:102B400020636F6C640A007C3C3E5E2B3D3F2F5B34
:102B50005D3B2C2A225C0043616E6E6F74206F70A7
:102B6000656E207375626469722000534420496E5B
:102B70006974204661696C0053442063617264206B
:102B80006F6B0A006F70656E526F6F7420666169BB
:102B90006C65640A00766F6C756D652E696E69747C
:102BA000206661696C65640A004E6F20534420639F
:102BB0006172640A000A4D3234004D3233202573AD
:102BC000002E0A006F70656E206661696C65642C6A
:102BD0002046696C653A200046696C652073656C17
:102BE00065637465640A002053697A653A2000467B
:102BF000696C65206F70656E65643A2000454E44CF
:102C000020535542524F5554494E450A00222070D8
:102C10006F73002220706172656E743A2200535502
:102C200042524F5554494E452043414C4C2074610B
:102C3000726765743A220053756263616C6C204F51
:102C4000766572666C6F7700457863656564656468
:102C5000206D617820535542524F5554494E4520BE
:102C600064657074683A002E0A0044656C65746986
:102C70006F6E206661696C65642C2046696C653AEC
:102C8000200046696C652064656C657465643A0073
:102C90005344207072696E74696E6720627974653E
:102CA00020004E6F74205344207072696E74696EF8
:102CB000670A0057726974696E6720746F206669CD
:102CC0006C653A2000667265736800646F696E67B0
:102CD000002066696C653A20004E6F7720002F61F6
:102CE00075746F25632E67002020506C616E6E65D1
:102CF0007242756666657242797465733A20002087
:102D000046726565204D656D6F72793A2000436F9C
:102D10006D70696C65643A204170722032342032E3
:102D20003032310A00204C61737420557064617434
:102D300065643A20323032312D30342D3138207CE8
:102D400020417574686F723A2054696E794D6163E1
:102D500068696E657333440A00322E302E375F4443
:102D600057372E330A004D61726C696E0020536F25
:102D70006674776172652052657365740A00205726
:102D800061746368646F672052657365740A00201C
:102D900042726F776E206F75742052657365740A86
:102DA000002045787465726E616C2052657365749D
:102DB0000A00506F77657255700A007374617274FF
:102DC0000A004732385859004D31303031006572B1
:102DD000726F722077726974696E6720746F2066F3
:102DE000696C650A00446F6E6520736176696E6771
:102DF0002066696C652E0A004D323900456E647399
:102E0000746F70730025532025632025632025638C
:102E100020256300205A3A0020593A0020583A00F1
:102E2000656E6473746F7073206869743A20007003
:102E3000012C0190012701B0012201C0011D01F008
:102E40000118011002130130020E01600209019005
:102E5000020401C002FF000003FA004003F50080F5
:102E600003F000D003EB002004E6007004E100E072
:102E700004DC004005D700C005D2004006CD00D0DC
:102E800006C8008007C3003008BE00F008B900C0C3
:102E900009B400B00AAF00B00BAA00D00CA5000026
:102EA0000EA000500F9B00C0109600501291000021
:102EB000148C00C0158700B0178200B0197D00D0B7
:102EC0001B7800001E730040206E0090226900F005
:102ED00024640040275F0090295A00E02B55001021
:102EE0002E500020304B0010324600E0334100905D
:102EF000353C001037370070383200A0392D00B053
:102F00003A2800A03B2300603C1E00103D190090B1
:102F10003D1400103E0F00703E0A00C03E05000048
:102F20003F0000403FFBFF803FF6FFC03FF1FF0046
:102F3000000A0B02090C0D0E080703040100000033
:102F40000000000000000000000000000000000081
:102F5000000000000000000000000012111000003E
:102F60000000000000000000000000000000000061
:102F7000000000000050726F62696E672046616950
:102F80006C656400205A3A200020593A20004265BE
:102F90006420583A20003D3D6F6E55736572436F53
:102FA0006E6669726D52657175697265643D3D004A
:102FB000220A00556E6B6E6F776E20636F6D6D61C8
:102FC0006E643A2022002042002050006F6B0020E7
:102FD0004500205A00205900204D39322058002049
:102FE000453A00205A3A0020593A00583A004361C5
:102FF0006E6E6F7420656E7465722073756264699D
:10300000723A20004D323520500A4D32340052655C
:1030100073756D65005549205061757365004E6F7D
:10302000204D61746368203A005067557000506706
:10303000446F776E0049732046696C6520004973C0
:10304000204469722000476F5570446972004861DE
:1030500073204D656469610046696C656E616D65DC
:103060002053656C6563746564004D3130303043C6
:10307000004D313030300046696C616D656E7420F2
:10308000537461742030202D20330046696C616DCB
:10309000656E7420537461742030202D20320046F8
:1030A000696C616D656E7420537461742030202DDD
:1030B0002031002046696C616D656E742052657325
:1030C000706F6E7365204E6F00526573756D65206D
:1030D00059657320647572696E67207072696E74C9
:1030E000000A204E6F2046696C616D656E74004960
:1030F0006E76616C6964204F7074696F6E004D3537
:1031000030300053746F72652053657474696E6754
:1031100073004265642050494420537461727465A1
:1031200064004D3939390A4D323830503053313618
:103130003000424C546F75636820526573657400AB
:103140004D3530320A4D35303000496E69742045B6
:103150004550524F4D00486F74656E64205049448D
:10316000205374617274656400456E676C6973689E
:1031700020416C726561647920536574004368690D
:103180006E657365204E6F7420537570706F727426
:10319000656400496E4C616E6743686F69636500E2
:1031A0000A202A2A2A7265636461742E646174613C
:1031B0005B305D203D004732380A473120463130D0
:1031C0003030205A313000556E737570706F7274E4
:1031D0006564204F7074696F6E2053656C6563740D
:1031E00065640047323652323535004D313930533F
:1031F00035350A4732380A4732390A4D3430300AF9
:103200004D313034533231350A4732380A4D31307E
:1032100039533231350A4D34323053310A4731583F
:103220003130305931303046353030300A47315A3C
:10323000300A4D3530300A4D313137205365742016
:103240005A204F666673657400473120463130302E
:1032500030205A302E30004732380A47312046316C
:10326000303030205A302E30004D353030005A206A
:103270004F6666736574203A202573004D353030F3
:10328000005A204F6666736574203A202573004704
:1032900032380A473146313530305A302E30004707
:1032A00032385A0A473146313530305A302E3000E4
:1032B0004D383400473146313030305A302E3000EE
:1032C0004732380A473146313030305A302E3000DC
:1032D0004D616E75616C53657454656D70005A2054
:1032E0004F6666736574203A2025730053746F70BF
:1032F000205472696767657265640053746F70204B
:103300004E6F0053746F705072696E740048616E36
:10331000646C6520446174612041646A7573742033
:10332000322053657474696E672053637265656EED
:10333000200048616E646C652044617461205072A5
:10334000696E7446696C6520332053657474696EC8
:10335000672053637265656E200048616E646C651A
:103360002044617461205072696E7446696C6520F6
:10337000322053657474696E672053637265656E9D
:1033800020004D38340048616E646C6520446174DF
:1033900061205072696E7446696C6520506F737459
:1033A0000048616E646C65204461746120507269EC
:1033B0006E7446696C652050726500426567696E7F
:1033C000537769746368003D3D20436865636B6BA8
:1033D00065793D3D007265636461742E6164647259
:1033E000203D3D007265636461742E646174615BAD
:1033F000305D203D3D0077616974776179203D3D06
:103400000020202A2A2A2A2A2A2A5254535F486155
:103410006E646C65446174612A2A2A2A2A2A2A2A3F
:103420002000526573656E643A200000002200257A
:103430000028002B002E003100340002010000059E
:103440000108010B0100002100240027002A002DA3
:10345000003000330001010000040107010A0105EA
:10346000050505070508080808020202020A0A08FD
:103470000804040404010101010101010103030323
:103480000303030303040707070C0C0C0C0C0C0CC0
:103490000C0202020206060606060606060B0B0BC7
:1034A0000B0B0B0B0B010210202008081020401002
:1034B00020408002010201080402010102040810F8
:1034C0002040808040201008040201800402018016
:1034D000402010080402010804020101020408103F
:1034E0002040800102040810204080436F6F6C6907
:1034F0006E672E2E2E0048656174696E672E2E2E23
:10350000004520255300544D33442043522D58206C
:1035100052656164792E005072696E74696E672E0F
:103520002E2E005072696E742050617573656400B0
:103530006E6F74696669636174696F6E20005049CB
:10354000442054756E652046696E69736865640031
:103550004D3234002801E00011241FBECFEFD1E22C
:10356000DEBFCDBF00E00CBF14E0A0E0B2E0E2E5BA
:10357000F7E802E00BBF02C007900D92AC32B10732
:10358000D9F727E1ACE2B4E001C01D92A831B2073F
:10359000E1F71AE1CBEADAE100E006C02197010980
:1035A000802FFE010F94D63FCA3AD10780E008076A
:1035B000A9F70F94E82C0D9497430C940000282F42
:1035C0009091CD0B833021F495FD0FC094FD0FC079
:1035D000892F90E0B0E0A0E004C0B695A79597953C
:1035E00087952A95D2F78170089581E0089580E04B
:1035F0000895CF92DF92EF92FF92CF93DF93EC0189
:10360000CC80DD80EE80FF8027E137EB41ED58EB89
:10361000C701B6010F943F4287FD23C023E030E08D
:103620004AE953E4C701B6010F940F391816CCF0DC
:10363000C880D980EA80FB8027E137EB41ED58EB69
:10364000C701B6010F943F4287FD0BC0C1E023E0E4
:1036500030E84DE953E4C701B6010F940F3918164D
:103660000CF4C0E08C2FDF91CF91FF90EF90DF90B2
:10367000CF900895129A479A0895269A2E9A0895FF
:10368000CF92DF92EF92FF921F93CF93DF93182F89
:10369000662351F010921405109210051092110536
:1036A00010921205109213050F9423106B017C01E8
:1036B0008091100590911105A0911205B09113050C
:1036C000A7019601281B390B4A0B5B0BDA01C901D4
:1036D000B7FD3DC02091140517FD13C0412F012EE9
:1036E000000C550B4C5F5F4F822F022E000C990B84
:1036F0004817590764F184EF91E0A0E0B0E021178A
:1037000024F488EE93E0A0E0B0E08C0D9D1DAE1D8A
:10371000BF1D8093100590931105A0931205B093DF
:1037200013052170C22F30E0D32F84E28C9FB001AB
:103730008D9F700D7C1B112460597C4F82E390E0BB
:103740000E9476A0809114058F5F80931405DF910D
:10375000CF911F91FF90EF90DF90CF9008952F921F
:103760003F924F925F926F927F928F929F92AF9211
:10377000BF92CF92DF92EF92FF920F931F93CF935E
:10378000DF93CDB7DEB760970FB6F894DEBF0FBEFC
:10379000CDBF8B876C87042F122F282F30E03E87F8
:1037A0002D87462F50E05A87498785E0982E929EB4
:1037B000C001939E900D1124988B8F87FA01E80F1A
:1037C000F91FEE0FFF1FEE0FFF1FE959F44F608145
:1037D0007181828193819B01AC010F94D142882336
:1037E00009F445C14B85400F6C85610F949EC00163
:1037F0001124E985FA85E80FF91FEE0FFF1FEE0F80
:10380000FF1FE959F44FC080D180E280F380040F9C
:10381000909EA0011124E985FA85E40FF51FEE0FB3
:10382000FF1FEE0FFF1FE959F44F00819180828046
:103830007380262F30E0EF85F889E20FF31FEE0F3B
:10384000FF1FEE0FFF1FE959F44F2080718179832C
:1038500072817A8373817B83610F70E0EF85F889D1
:10386000E60FF71FEE0FFF1FEE0FFF1FE959F44F92
:10387000F88BEF87F081FC83EF85F889F181FD8378
:10388000EF85F889F281FE83EF85F889F381FF8364
:10389000FC01E20FF31FEE0FFF1FEE0FFF1FE959B0
:1038A000F44F20812887A180B2806380FA01E60F5F
:1038B000F71FEE0FFF1FEE0FFF1FE959F44F408077
:1038C000518032801381202F392D482D572D602FA4
:1038D000792D882D972D0F94D142882321F000E077
:1038E000912C812C712C9601A701B601C7010F9470
:1038F000D142882321F0C02ED92CE82CF72C2C8122
:103900003D814E815F816C817D818E819F810F948D
:10391000D142882321F01C821D821E821F82222D0B
:1039200039814A815B81622D79818A819B810F94E3
:10393000D142882339F02C803D8139834E814A83DE
:103940005F815B839201432D512FB201832D912F13
:103950000F94D142882321F0412C512C312C10E0BE
:1039600028853A2D4B2D562D68857A2D8B2D962D39
:103970000F94D142882321F04886A52CB32C612EC8
:1039800085E02D853E85829FF001839FF00D1124F7
:1039900049855A85E40FF51FEE0FFF1FEE0FFF1F3D
:1039A000E959F44FFA87E9879601A701B601C701E3
:1039B0000F94DF3F202F392D482D572D0F94DE3FD8
:1039C0006B017C01222D39814A815B81622D7981D5
:1039D0008A819B810F94DF3F2C813D814E815F81E5
:1039E0000F94DE3F9B01AC01C701B6010F94DF3F8E
:1039F0006B017C0128853A2D4B2D562D68857A2D3B
:103A00008B2D962D0F94DF3F9201432D512F0F9454
:103A1000DE3F9B01AC01C701B6010F94DF3F20E000
:103A200030E040E450E40F94D940E985FA856083A2
:103A30007183828393836C858B8560960FB6F8942F
:103A4000DEBF0FBECDBFDF91CF911F910F91FF90D1
:103A5000EF90DF90CF90BF90AF909F908F907F902E
:103A60006F905F904F903F902F900D94670A6096F3
:103A70000FB6F894DEBF0FBECDBFDF91CF911F917F
:103A80000F91FF90EF90DF90CF90BF90AF909F90FD
:103A90008F907F906F905F904F903F902F90089500
:103AA0000F931F93CF93DF9300D01F92CDB7DEB754
:103AB0009C010BE41BE090E1E2E6FDE0D8010190FF
:103AC0000D929A95E1F7F90120813181428153816C
:103AD000F80160857185828593850F94DF3FF80139
:103AE000608771878287938780E090E0A0EAB0E4E6
:103AF00089839A83AB83BC83CE0101960E94BF8FDA
:103B00000F900F900F900F90DF91CF911F910F9119
:103B100008952F923F924F925F926F927F928F9271
:103B20009F92AF92BF92CF92DF92EF92FF921F933C
:103B3000CF93DF93CDB7DEB72C970FB6F894DEBFE7
:103B40000FBECDBF7A011901DC012D913D914D9140
:103B50005C912D833E834F835887FB0140805180C9
:103B6000628073808090620D9090630DA090640DD0
:103B7000B090650DA50194016D817E818F8198853E
:103B80000F940F3981110EC011E0A30192016091D1
:103B9000660D7091670D8091680D9091690D0F947D
:103BA0000F39811110E0D1012D913D914D915C9122
:103BB00029873A874B875C87F701C080D180E280F4
:103BC000F38020910B0230910C0240910D02509134
:103BD0000E02C701B6010F940F39882309F44EC0B5
:103BE000C0920B02D0920C02E0920D02F0920E02F3
:103BF00080916E0D90916F0DA091700DB091710D2F
:103C00004091660D5091670D6091680D7091690D3E
:103C100080924B0B90924C0BA0924D0BB0924E0B9E
:103C200040934F0B5093500B6093510B7093520B7A
:103C3000C092530BD092540BE092550BF092560B5E
:103C40008093570B9093580BA093590BB0935A0B3A
:103C500020E030E040E05FE360912E0D70912F0D89
:103C60008091300D9091310D0F94753969837A836D
:103C70008B839C83CE0101960E94BF8F2D813E8154
:103C80004F81588520934B0B30934C0B40934D0B39
:103C900050934E0B40924F0B5092500B6092510B31
:103CA0007092520BD1012D913D914D915C9160919B
:103CB000570B7091580B8091590B90915A0B0F94A0
:103CC000DF3F6093570B7093580B8093590B909381
:103CD0005A0B11112FC020E030E0A90169857A85C7
:103CE0008B859C850F940F39811133C060E070E0A3
:103CF00088EC92E469837A838B839C83CE0101965E
:103D00000E94BF8F2C960FB6F894DEBF0FBECDBFBA
:103D1000DF91CF911F91FF90EF90DF90CF90BF90F8
:103D2000AF909F908F907F906F905F904F903F905B
:103D30002F9008952AEF3EE74AE25FE36091320D4B
:103D40007091330D8091340D9091350D0F9475392C
:103D5000D1CF60E070E080EA91E4CCCFCF93DF93E5
:103D600000D01F92CDB7DEB780E090E0A0EAB0E4CB
:103D700089839A83AB83BC8361E0CE0101960E9464
:103D800046910F900F900F900F90DF91CF91089573
:103D900080912E0590912F05009731F04AE050E078
:103DA00070E060E00D942A3760E070E0CB01089588
:103DB0000F931F93CF93DF9300D000D01F921F92D9
:103DC000CDB7DEB78B01FC0123A5211102C00F94F2
:103DD0006E0E1D821E821F82188620E030E040E0B9
:103DE0005FE360916A0D70916B0D80916C0D909105
:103DF0006D0D0F94DF3F69837A838B839C839E01D3
:103E00002B5F3F4FAE014F5F5F4F66E67DE082E67E
:103E10009DE00E94891D1D821E821F82188620E05F
:103E200030E040E05FE3F80160857185828593852D
:103E30000F94DF3F69837A838B839C83B8016C5F27
:103E40007F4F9E012B5F3F4FAE014F5F5F4FC80119
:103E50000E94891D28960FB6F894DEBF0FBECDBF15
:103E6000DF91CF911F910F91089580912E05909130
:103E70002F05009731F04AE050E070E060E00D94CB
:103E8000FC3560E070E0CB0108950E94351F97FD7E
:103E90000CC00E94351F6F3F71058105910509F027
:103EA00034F40E94351F862F089580E008958FEF27
:103EB0000895CF92DF92EF92FF920F931F93CF93CB
:103EC000DF936B017A01EC01CC53DB4F28813CE09E
:103ED000389F8001399F100D112427FF24C0FB015A
:103EE0001182108288818F5F888388819801280FD2
:103EF000311D87FD3A95C90120915613F601281707
:103F0000190629F024F088818C300CF43CC08081A3
:103F10009181049680349C4908F475C0F601808133
:103F20009181049672C088819801280F311D87FD08
:103F30003A95C901209156132817190699F294F25F
:103F40008881A801480F511D87FD5A95FA01EE0F8F
:103F5000FF1FE40FF51FE25FFC4E808187FFC2CF99
:103F60008881F801E80FF11D87FDFA95CF01EE0F6A
:103F7000FF1FE80FF91FE25FFC4E808160E08F7742
:103F80000F948E0EAFCF808191812881A801420FBE
:103F9000511D27FD5A959A01FA01EE0FFF1FE20FFE
:103FA000F31FE25FFC4E21813281820F931FF701E4
:103FB0009183808388819801280F311D87FD3A9570
:103FC000F901EE0FFF1FE20FF31FE25FFC4E80814D
:103FD00087FF20C08881080F111D87FD1A95F80101
:103FE000EE0FFF1FE00FF11FE25FFC4E808161E0EA
:103FF0008F77DF91CF911F910F91FF90EF90DF901E
:10400000CF900D948E0E80E49CE9F701918380831C
:104010008FEF8883DF91CF911F910F91FF90EF90E9
:10402000DF90CF9008950F931F93CF93DF93C82F06
:10403000D0E0FE01EE0FFF1FE25CFD4F7183608355
:10404000CC0FDD1FCC0FDD1F8E01025E1D4F072E32
:10405000000C880B990B0F9416392AE037ED43E2D8
:104060005CE30F947539C655DA4F288139814A814E
:104070005B810F947539F801608371838283938328
:10408000DF91CF911F910F910895FC01659175917A
:1040900085919491089580915B0B882319F080E0BD
:1040A0000E940B9480E008954F925F926F927F92EE
:1040B0008F929F92AF92BF92CF92DF92EF92FF9238
:1040C000CF93DF9300D000D01F921F92CDB7DEB701
:1040D0005C01DB01CD90DD90ED90FC90E0916613EA
:1040E000F0916713FE83ED8384819581A681B7816A
:1040F00089839A83AB83BC839C01AD01C701B60160
:104100000F94DE3F2B013C01F50180809180A2805D
:10411000B380AD81BE818D919D910D90BC91A02DFC
:104120008D839E83AF83B88727E137EB41ED58EB52
:10413000C301B2010F943F4287FDD1C023E030E0BC
:104140004AE953E4C301B2010F940F3918160CF475
:10415000C6C02D813E814F815885C501B4010F94A1
:10416000DE3F2B013C0127E137EB41ED58EB0F948B
:104170003F4287FDB4C023E030E84DE953E4C3017A
:10418000B2010F940F3918160CF4A9C020E030E0EA
:10419000A9016D817E818F8198850F94DF3F2B016E
:1041A0003C0120E030E040E450E40F940F3987FFF9
:1041B00005C0412C512C30E4632E762C27E137EBDF
:1041C00041ED58E3C301B2010F94DE3F9B01AC0106
:1041D000C501B4010F943F4287FD81C020E030E863
:1041E0004DE953E46D817E818F8198850F94DF3F87
:1041F0002B013C0120E030E844E953E40F943F42B6
:1042000018163CF4412C20E8522E24E9622E23E4B7
:10421000722E27E137EB41ED58E3C301B2010F9451
:10422000DF3F9B01AC01C501B4010F940F39181693
:104230000CF455C020E030E0A90169817A818B81BE
:104240009C810F94DF3F4B015C0120E030E040E9AE
:1042500051E40F940F3987FF06C0812C912C90E90F
:10426000A92E91E4B92E27E137EB41ED58E3C501C2
:10427000B4010F94DE3F9B01AC01C701B6010F945E
:104280003F4287FD2CC020E030E04AE953E46981D9
:104290007A818B819C810F94DF3F4B015C0120E090
:1042A00030E04DE853E40F943F42181634F4812C6B
:1042B000912C8DE8A82E83E4B82E27E137EB41ED51
:1042C00058E3C501B4010F94DF3F9B01AC01B1E09D
:1042D000B983C701B6010F940F3918160CF419826F
:1042E000898128960FB6F894DEBF0FBECDBFDF914F
:1042F000CF91FF90EF90DF90CF90BF90AF909F90C5
:104300008F907F906F905F904F9008958F929F92C3
:10431000AF92BF92CF92DF92EF92FF92CF93DF9353
:10432000EC018090B00C9090B10CA090B20CB090C9
:10433000B30C20E030E0A901C501B4010F940F399E
:10434000882309F454C0C880D980EA80FB80A70183
:104350009601C501B4010F940F3918160CF04CC02A
:104360002091A80C3091A90C4091AA0C5091AB0C53
:10437000C701B6010F940F39882331F1C092A80C00
:10438000D092A90CE092AA0CF092AB0C2091AC0C4C
:104390003091AD0C4091AE0C5091AF0C6881798199
:1043A0008A819B810F9475399B01AC0160E070E0BC
:1043B00080E89FE30F94DE3F60930F02709310023A
:1043C000809311029093120260910F02709110027B
:1043D0008091110290911202DF91CF91FF90EF90A6
:1043E000DF90CF90BF90AF909F908F90089560E046
:1043F00070E080E89FE3F0CF60E070E0CB01ECCFAD
:104400009B01AC01485F5F4FBC016C5F7F4F0C9418
:10441000891D2F923F924F925F926F927F928F925F
:104420009F92AF92BF92CF92DF92EF92FF920F9343
:104430001F93CF93DF93CDB7DEB7A6970FB6F8944F
:10444000DEBF0FBECDBF8C011B015A87498740904C
:10445000620D5090630D6090640D7090650D8090BA
:10446000660D9090670DA090680DB090690DDB010E
:104470008D919D910D90BC91A02D8B8B9C8BAD8BC4
:10448000BE8B9C01AD01C301B2010F94DE3F6B01F5
:104490007C01D10114968D919D910D90BC91A02D20
:1044A0008F8B988FA98FBA8F9C01AD01C501B40184
:1044B0000F94DE3F6B8F7C8F8D8F9E8FA985BA8581
:1044C0008D919D910D90BC91A02D8B879C87AD8780
:1044D000BE879C01AD01C301B2010F94DE3F6F8F17
:1044E00078A389A39AA3A985BA8514968D919D91E5
:1044F0000D90BC91A02D8F87988BA98BBA8B9C01B6
:10450000AD01C501B4010F94DE3F6BA37CA38DA365
:104510009EA3A7019601C701B6010F9475396B01DF
:104520007C012B8D3C8D4D8D5E8DCA01B9010F94A0
:1045300075399B01AC01C701B6010F94DF3F4B01F8
:104540005C012B893C894D895E896B857C858D85D5
:104550009E850F94DE3F2B013C012F89388D498DBC
:104560005A8D6F85788989899A890F94DE3F6B010E
:104570007C01A3019201C301B2010F9475392B0193
:104580003C01A7019601C701B6010F9475399B0143
:10459000AC01C301B2010F94DF3F0F948D426B0158
:1045A0007C012F8D38A149A15AA1CA01B9010F94EC
:1045B00075392B013C012BA13CA14DA15EA1CA0183
:1045C000B9010F9475399B01AC01C301B2010F947D
:1045D000DF3F9B01AC01C501B4010F943F421816A7
:1045E000B4F520E030E0A901C701B6010F943F42C5
:1045F00087FF2AC0C701B601905820E030E040EAAA
:1046000050E40F943F42181614F5A10169857A858C
:10461000C8010E940922A6960FB6F894DEBF0FBE0D
:10462000CDBFDF91CF911F910F91FF90EF90DF9061
:10463000CF90BF90AF909F908F907F906F905F9042
:104640004F903F902F900895C701B601D6CF20E03C
:1046500030E040E050E4C501B4010F943F42181629
:1046600024F4B101C8010E94D81E19821A821B824B
:104670001C82BE016F5F7F4FC1010E9400222DECA2
:104680003CEC4CEC5CE3C701B6010F9475399B011F
:10469000AC01F80160817181828193810F94753939
:1046A0006D837E838F839887D8019B968C919B978F
:1046B0008823C9F02AE939E949E95FE314966D9145
:1046C0007D918D919C9117970F94753969837A83A9
:1046D0008B839C83BE016F5F7F4F8BE49BE00E94C6
:1046E0000022F80113A6BE016B5F7F4F89859A8572
:1046F0000E94002290CF3F924F925F926F927F92E2
:104700008F929F92AF92BF92CF92DF92EF92FF92E1
:104710000F931F93CF93DF93CDB7DEB76C970FB690
:10472000F894DEBF0FBECDBFDB010C91142F100F2C
:10473000153008F067C11196DC90C22ECD0CB4E0A4
:10474000BC1508F45FC1ED2DF0E0EB5DFA4F808001
:10475000912CB12CA12C002E04C0B694A794979450
:1047600087940A94D2F780FE4DC1EC2DF0E0EB5D0A
:10477000FA4F8080912CB12CA12C012E04C0B6944C
:10478000A794979487940A94D2F780FE3BC1322E67
:10479000642F7C0140905F0950906009609061092E
:1047A000709062098091670990916809A0916909E8
:1047B000B0916A09898F9A8FAB8FBC8F660F770B88
:1047C000072E000C880B990B0F9416394B015C01D6
:1047D000602F000F770B880B990B0F941639298DDA
:1047E0003A8D4B8D5C8D0F947539A30192010F9416
:1047F000DF3FA50194010F94DF3F6D877E878F8790
:10480000988B612F110F770B880B990B0F9416392A
:10481000298D3A8D4B8D5C8D0F947539A3019201D2
:104820000F94DF3FA50194010F94DE3F69837A83E3
:104830008B839C8340906309509064096090650964
:104840007090660980916B0990916C09A0916D0937
:10485000B0916E09898F9A8FAB8FBC8F632D660FD5
:10486000770B072E000C880B990B0F9416394B0110
:104870005C016D2DDD0C770B880B990B0F941639AD
:10488000298D3A8D4B8D5C8D0F947539A301920162
:104890000F94DF3FA50194010F94DF3F698B7A8B62
:1048A0008B8B9C8B6C2DCC0C770B880B990B0F94FE
:1048B0001639298D3A8D4B8D5C8D0F947539A30176
:1048C00092010F94DF3FA50194010F94DE3F6D83A9
:1048D0007E838F839887F70180859185A285B38534
:1048E00089879A87AB87BC878D8B9E8BAF8BB88F60
:1048F00043E351E061E070E0CE0141960E94C2DEE8
:1049000043E351E061E070E0CE0105960E94C2DE13
:104910004AE351E061E070E0CE010D960E94C2DEF4
:104920004AE351E061E070E0CE0101960E94C2DEF0
:1049300089889A88AB88BC8827E137EB41ED58EB32
:10494000C501B4010F943F4287FD5CC023E030E015
:104950004AE953E4C501B4010F940F3918160CF459
:1049600051C08D849E84AF84B88827E137EB41ED38
:1049700058EBC501B4010F943F4287FD43C023E0CB
:1049800030E84DE953E4C501B4010F940F3918160E
:10499000CCF18D809E80AF80B88427E137EB41ED6C
:1049A00058EBC501B4010F943F4287FD2BC023E0B3
:1049B00030E04AE953E4C501B4010F940F391816E9
:1049C0000CF189809A80AB80BC8027E137EB41ED08
:1049D00058EBC501B4010F943F4287FD13C023E09B
:1049E00030E84DE953E4C501B4010F940F391816AE
:1049F0004CF0AE014F5F5F4FBE01635F7F4FC70159
:104A00000E9409226C960FB6F894DEBF0FBECDBF90
:104A1000DF91CF911F910F91FF90EF90DF90CF909A
:104A2000BF90AF909F908F907F906F905F904F90CE
:104A30003F9008958C38910514F08CE890E09093A5
:104A40006212809361120C948ADB80912E05909102
:104A50002F05892B41F00E94451F91E0811101C073
:104A600090E0892F089591E0FCCF0E94351FCB0183
:104A700008950F931F93CF9380912E0590912F054A
:104A80000097E9F0FC018F01C1912C2F2F7D81F05F
:104A9000C53411F0C536B9F7F801108270E060E056
:104AA0000F949E34F801C083CF911F910F91089508
:104AB00070E060E0CF911F910F910D949E3460E003
:104AC00070E0CB01F1CF2FEB280F2A3108F047C05F
:104AD000E22FF0E080915D0590915E05A0915F0569
:104AE000B091600504C0B695A795979587952A95CE
:104AF000D2F780FD02C081700895E15CFA4FE08139
:104B0000EE2341F180915D0B90915E0BE80FF92F40
:104B1000F11D808190ED980F9A3030F08E3251F473
:104B2000818180538A3098F4F0932F05E0932E050D
:104B300081E008958D3211F08B3249F4818190ED3E
:104B4000980F9A3088F38E3211F48281EACFF0E028
:104B5000E0E0EACF10922F0510922E05E9CF80E019
:104B600008950E946325882341F081E020912E055D
:104B700030912F05232B09F480E00895CF93DF9324
:104B8000EB010E94B125882319F00E94351FEB012B
:104B9000CE01DF91CF910895CF93DF93EB010E9477
:104BA000B125882321F0DF91CF910C943525CE01DA
:104BB000DF91CF910895CF93C62F0E94B12588230E
:104BC00019F0CF910C94451F8C2FCF910895CF925F
:104BD000DF92EF92FF926A017B010E94B125882348
:104BE00031F0FF90EF90DF90CF900C943925C70102
:104BF000B601FF90EF90DF90CF9008954F925F92B3
:104C00006F927F928F929F92AF92BF92CF92DF92DC
:104C1000EF92FF921F93CF93DF9300D01F92CDB7F7
:104C2000DEB719821A821B821C82CE0101964C01CA
:104C30008BE4C82E8BE0D82E92E6E92E9DE0F92E6B
:104C400024EBA22E2CE0B22E10E088E5810F0E940A
:104C5000B125F40181934F01882309F4E0C00E943B
:104C600039252B013C01812F0E94DF1A882309F48A
:104C7000CCC0F7012081318142815381C301B2014F
:104C80000F94DF3FF60160837183828393831F5FFC
:104C9000F4E0CF0ED11C84E0E80EF11C94E0A90EE4
:104CA000B11C133091F685E40E94B1258C838823D2
:104CB00009F4C0C00E9439256B017C0183E00E9489
:104CC000DF1A882371F020916E0D30916F0D4091A5
:104CD000700D5091710DC701B6010F94DF3F6B014C
:104CE0007C01C092570BD092580BE092590BF09276
:104CF0005A0B80915E09882359F18091371582FF04
:104D000027C08C81882321F18981811103C08A8188
:104D10008823F1F02DEC3CEC4CE45DE36091FA0B60
:104D20007091FB0B8091FC0B9091FD0B0F94DF3F7A
:104D30009B01AC0160916A0D70916B0D80916C0DBF
:104D400090916D0D0F943F42181614F40F949B0927
:104D500040E050E0BA0186E40E94E72520E030E020
:104D6000A9010F943F42181684F40E94392520E0CF
:104D700030E040E752E40F94D940609353027093BF
:104D8000540280935502909356028091CC0B83FD80
:104D900028C08091680A882321F120916E0D3091FE
:104DA0006F0D4091700D5091710D6091570B709186
:104DB000580B8091590B90915A0B0F94DE3F209124
:104DC000750A3091760A4091770A5091780A0F94CB
:104DD000DF3F6093750A7093760A8093770A909309
:104DE000780A0F900F900F900F90DF91CF911F9145
:104DF000FF90EF90DF90CF90BF90AF909F908F90FB
:104E00007F906F905F904F900895F50120813181E0
:104E100042815381C301B2010F94DE3F33CFF701CA
:104E200080819181A281B381F60180839183A283E5
:104E3000B3832DCF80916E0D90916F0DA091700D69
:104E4000B091710D8093570B9093580BA093590B11
:104E5000B0935A0B4ECFCF93DF93C82FD62F0E941B
:104E6000B125882321F0DF91CF910C9425258C2F3B
:104E70000E946325811101C08D2FDF91CF9108958C
:104E8000E1EFFBE087EBDF011D928A95E9F70895DA
:104E900080915E09811104C00E9440270C94F2D1D8
:104EA0008091371582FD0D949B0908958091F10B37
:104EB000882361F09091A70C891308C08091371561
:104EC00083FF04C084E39CE00C94BCD080E0089590
:104ED000FC01238121110C94F1CC08954F925F9233
:104EE0006F927F928F929F92AF92BF92CF92DF92FA
:104EF000EF92FF920F931F93CF93DF93EC012091DA
:104F00005F0930916009409161095091620968819F
:104F100079818A819B810F94DE3F6B017C01209116
:104F200063093091640940916509509166096C816B
:104F30007D818E819F810F94DE3F4B015C01A70133
:104F40009601609103027091040280910502909194
:104F500006020F940F39882309F450C0C09203024F
:104F6000D0920402E0920502F09206022091080518
:104F70003091090540910A0550910B05C701B60112
:104F80000F9475392B013C010F9481416B017C0119
:104F900020E030E0A9010F940F3987FD70C020E0B8
:104FA00030E040E450E4C701B6010F943F421816C8
:104FB0002CF4C12CD12CC0E4EC2EFE2CA7019601C0
:104FC000C301B2010F94DE3F6093000570930105A9
:104FD0008093020590930305C701B6010F944B41DE
:104FE0006093FE04062E000C770B6F5F7F4F6430DA
:104FF000710514F064E070E06093FC04D09101024C
:105000001091FE04A50194016091070270910802BD
:105010008091090290910A020F940F39811133C0D7
:10502000D11381C02091E4043091E5044091E6045D
:105030005091E7046091000570910105809102058F
:10504000909103050F9475392091E8043091E9049B
:105050004091EA045091EB040F94DF3FDF91CF9130
:105060001F910F91FF90EF90DF90CF90BF90AF9086
:105070009F908F907F906F905F904F900895C12C7C
:10508000D12C76019BCF8092070290920802A092C9
:105090000902B0920A0220910C0530910D05409151
:1050A0000E0550910F05C501B4010F9475394B01E0
:1050B0005C010F9481416B017C0120E030E0A9018B
:1050C0000F940F3987FDF3C020E030E040E450E456
:1050D000C701B6010F943F4218162CF4C12CD12CF5
:1050E000B0E4EB2EFE2CA7019601C501B4010F948C
:1050F000DE3F609304057093050580930605909349
:105100000705C701B6010F944B416093FF04062EBB
:10511000000C770B6F5F7F4F6430710514F064E013
:1051200070E06093FD04C091FF04D11305C080912D
:1051300002028C1709F470C08091FE049091FF0464
:1051400090930202809301020C2E000CDD0B25E0EF
:105150001203C0011124FC01EC0FFD1FEE0FFF1F15
:10516000EE0FFF1FE959F44F2081318142815381B5
:105170002093F8043093F9044093FA045093FB040D
:105180000091FD04002E000C110BFC01E00FF11F3B
:10519000EE0FFF1FEE0FFF1FE959F44F6081718181
:1051A000828193810F94DE3F6093F4047093F50441
:1051B0008093F6049093F7042091FC0435E02303D8
:1051C000F0011124CE0FDF1FCC0FDD1FCC0FDD1F30
:1051D000C959D44F288139814A815B812093F004D9
:1051E0003093F1044093F2045093F304E00FF11F65
:1051F000EE0FFF1FEE0FFF1FE959F44F6081718121
:10520000828193810F94DE3F6093EC047093ED04F0
:105210008093EE049093EF04809004059090050530
:10522000A0900605B09007052091F4043091F50494
:105230004091F6045091F704C501B4010F947539FB
:105240002091F8043091F9044091FA045091FB0444
:105250000F94DF3F6B017C01C092E804D092E90417
:10526000E092EA04F092EB042091EC043091ED041A
:105270004091EE045091EF04C501B4010F947539CB
:105280002091F0043091F1044091F2045091F30424
:105290000F94DF3FA70196010F94DE3F6093E40473
:1052A0007093E5048093E6049093E704BBCEC12C91
:1052B000D12C760118CF1F93CF93DF93CDB7DEB7F4
:1052C0002C970FB6F894DEBF0FBECDBF182F8823E2
:1052D00079F020E030E0A9016091670970916809D8
:1052E0008091690990916A090F940F398823F9F028
:1052F0008091010D8117D9F00E9403888CE0E5E8C8
:10530000F2E0DE01119601900D928A95E1F7CE014F
:1053100001960E946E278091010D882391F082E60C
:105320009DE00E9426881092010D0E946C922C969E
:105330000FB6F894DEBF0FBECDBFDF91CF911F91A6
:10534000089581E08093010D82E69DE00E945387DD
:10535000ECCF8F929F92AF92BF92EF92FF920F93FA
:105360001F93CF93DF9380E00E945B291092630923
:1053700010926409109265091092660910925F09F3
:1053800010926009109261091092620910926B09E3
:1053900010926C0910926D0910926E0910926709B3
:1053A000109268091092690910926A0907E61BE0D9
:1053B000C0E0812C912C80ECA82E8FE7B82E7801CC
:1053C000D0E0F70181929192A192B1927F016D2F6D
:1053D0008C2F0F94670ADF5FD53099F7CF5F0C5E93
:1053E0001F4FC53061F7DF91CF911F910F91FF9053
:1053F000EF90BF90AF909F908F9008958F929F9263
:10540000AF92BF92CF92DF92EF92FF92C090670966
:10541000D0906809E0906909F0906A0920E030E0D6
:10542000A901C701B6010F940F398823E1F1A70143
:10543000960160E070E080E89FE30F94D9406B0133
:105440007C0180906B0990906C09A0906D09B090E0
:105450006E0920E030E0A901C501B4010F940F39B5
:10546000882329F1A501940160E070E080E89FE3C2
:105470000F94D940C0920805D0920905E0920A0520
:10548000F0920B0560930C0570930D0580930E054B
:1054900090930F05FF90EF90DF90CF90BF90AF906B
:1054A0009F908F900895C12CD12C7601CACF60E0D7
:1054B00070E0CB01DFCFEFE6F0E080818260808397
:1054C00008958091161290911712892B79F480918A
:1054D000161290911712892B49F4209116123091CF
:1054E000171281E0232B19F480E0089581E00895DC
:1054F000CF92DF92EF92FF926B017C0183E3C8169B
:10550000D104E104F10470F082E3C81AD108E10883
:10551000F10862E370E080E090E00F94F00F0E94E9
:1055200004DFECCFC701B6010F94F00FFF90EF90AE
:10553000DF90CF900C9404DF80910112882341F01A
:10554000813041F064E670E080E090E00C94782ACD
:10555000129AF8CF479AF6CF5F9A8091000D8E7F0E
:105560008093000D8A9A8091000D8D7F8093000DAD
:105570008091080180958170809306018091000DD3
:105580008B7F8093000D0C943A1B9091371593FB01
:10559000882780F993FF06C081E090919E169111B3
:1055A00001C080E0089581E00C9443A770E060E0C2
:1055B00080E00E9444E370E060E081E00C9444E30A
:1055C00081E00895DC01EC918E2F90E0FC01EE0F5C
:1055D000FF1FE80FF91FE25FFC4E80818F77808309
:1055E00008958F929F92AF92BF92CF92DF92EF92E7
:1055F000FF920F93CF93DF931F92CDB7DEB75C017D
:105600007B0149016B01C40ED51EF501808191819A
:105610000F942D3F8983002311F0F7018083BE0191
:105620006F5F7F4FC4010F942E00F501808191813F
:10563000019691838083FFEFEF1AFF0AEC14FD04BB
:1056400021F780E00F90DF91CF910F91FF90EF90C5
:10565000DF90CF90BF90AF909F908F90089500976C
:1056600081F41092900082E0809391001092950056
:1056700010929400C19A80917100826080937100B1
:105680000895019761F41092A00082E08093A10038
:105690001092A5001092A40089BB80937200089517
:1056A0007F928F929F92AF92BF92CF92DF92EF92B2
:1056B000FF920F931F93CF93DF93EC017B018881BF
:1056C000883108F0C3C090E0FC01EE0FFF1FE80F27
:1056D000F91FE25FFC4E80818F770F94AF0619822D
:1056E0001A8288812CE0622F0F94B63F829FB0010E
:1056F000112430E020E0AB01420F531FFA01EE0FFE
:10570000FF1FE40FF51FE25FFC4E908197FD08C07C
:105710002F5F3F4F2C30310571F790E00E942F2B07
:105720007880072D10E06801CC0CDD1CF601E00F3D
:10573000F11FE25FFC4E80818068808377FC86C029
:1057400080E2E81682E0F8060CF03FC08A8128E586
:1057500032E0281B310987FD3395220F331F220FBA
:10576000331F032E000C440B550B898178E8872EDC
:10577000912C881A910887FD9394880C991C880CA9
:10578000991C092C000CAA08BB0860E070E0CB0152
:10579000F7FC0AC0B701653B710514F064EB70E0DB
:1057A000072E000C880B990B281939094A095B0947
:1057B0000F94433F24EB30E040E050E00F94753FFE
:1057C000820E931EA41EB51E740187E18715D8F0C2
:1057D000298188E890E0821B910927FD9395880F25
:1057E000991F880F991FE816F90604F502972FB73D
:1057F000F894E601C00FD11FC25FDC4E880F991FDD
:105800009A8389832FBF62E370E080E090E0DF91AC
:10581000CF911F910F91FF90EF90DF90CF90BF90AD
:10582000AF909F908F907F900C94782A2A8188E582
:1058300092E0821B910927FD9395880F991F880F8D
:10584000991FE816F90694F6C701D0CFDF91CF91E2
:105850001F910F91FF90EF90DF90CF90BF90AF908E
:105860009F908F907F900895CF93DF93EB01682FE7
:1058700070E087E593E10E94502B688179818A81ED
:105880009B81643F21E072078105910520F464EF5C
:1058900071E080E090E00E94782A89B183FB88273C
:1058A00080F9DF91CF910895CF93DF9300D01F92BD
:1058B000CDB7DEB78EEE92E0A0E0B0E089839A83A8
:1058C000AB83BC83BE016F5F7F4F8AE50E94342C9F
:1058D0000F900F900F900F90DF91CF910895CF937D
:1058E000DF9300D01F92CDB7DEB78EEE92E0A0E03E
:1058F000B0E089839A83AB83BC83BE016F5F7F4F27
:105900008AE00E94342C0F900F900F900F90DF913F
:10591000CF910895CF93DF9300D01F92CDB7DEB71C
:1059200084EF91E0A0E0B0E089839A83AB83BC83ED
:10593000BE016F5F7F4F80EA0E94342C0F900F9062
:105940000F900F90DF91CF9108951F920F920FB695
:105950000F9211240BB60F922F933F934F935F93A7
:105960006F937F938F939F93AF93BF93EF93FF9327
:1059700048EA50E064EA70E081E090E00E94591F3C
:10598000FF91EF91BF91AF919F918F917F916F9117
:105990005F914F913F912F910F900BBE0F900FBED3
:1059A0000F901F9018951F920F920FB60F9211240F
:1059B0000BB60F922F933F934F935F936F937F9309
:1059C0008F939F93AF93BF93EF93FF9348E950E07A
:1059D00064E970E090E080E00E94591FFF91EF9130
:1059E000BF91AF919F918F917F916F915F914F91F7
:1059F0003F912F910F900BBE0F900FBE0F901F90F5
:105A000018959091D10095FD0CC09091D00095FF14
:105A100008C08093D6008091D00080648093D0002D
:105A20000895209142042F5F2F770FB607FC27C0FF
:105A300090914304921328C09091D00095FF1EC00E
:105A40009091430440914204941306C09091D10078
:105A50009F7D9093D10012C0E92FF0E0EE5BFB4FE9
:105A600032819F5F9F773093D600909343043091AB
:105A7000D00030643093D000491741F3D9CF9091D2
:105A80004304921301C0FBCFE0914204F0E0EE5BCF
:105A9000FB4F8283209342048091D10080628093E7
:105AA000D10008951F920F920FB60F9211240BB6DA
:105AB0000F922F938F939F93EF93FF9380914304C3
:105AC00020914204821306C08091D1008F7D809383
:105AD000D10012C0E82FF0E0EE5BFB4F92818F5FA8
:105AE0008F779093D600809343049091D000906478
:105AF0009093D000281741F3FF91EF919F918F91E0
:105B00002F910F900BBE0F900FBE0F901F90189506
:105B10001F920F920FB60F9211240BB60F920F9394
:105B20001F932F933F934F935F936F937F938F9325
:105B30009F93AF93BF93CF93DF93EF93FF93C09166
:105B4000D60000916505D091640511E01D0F1F730B
:105B500090914104913108F09FC0E92FF0E088272F
:105B6000EB54F24D8F4F0D94D63FC62DF52D042EDC
:105B7000132E1A2E4C2E1E2E4C2E222E262E4C2E3E
:105B80002A2E2E2E322E392E4C2E442EC03229F0A3
:105B900028F5CA3011F0CD3031F5011731F0ED2F75
:105BA000F0E0EC59FA4FC283D12FD0936405FF91F6
:105BB000EF91DF91CF91BF91AF919F918F917F91A5
:105BC0006F915F914F913F912F911F910F910F9086
:105BD0000BBE0F900FBE0F901F901895CD3481F023
:105BE00081E0CE3471F080E10CC0CA3338F4C033A8
:105BF000A0F6C03291F2CD32B1F7CFCFCD3499F7C4
:105C000082E080934104C9CFC13359F018F4C03207
:105C100021F2E9CF88E0C433A1F38BE0C83389F3E4
:105C2000E2CF83E0EECF84E0C03359F386E0C133A6
:105C300041F3D9CF85E0C833B1F6E3CF87E0C23373
:105C400091F6DFCF89E0C13371F6DBCF8AE0C03354
:105C500051F6D7CF8CE0C73331F6D3CF8DE0C633C2
:105C600011F6CFCFC03209F498CF8EE0C33549F298
:105C7000BACF80ED8C0F8A3008F08FCF9FE09093E1
:105C800041048093400489CFCA3019F0CD3009F027
:105C900084CF1092410481CFCA3019F0CD3009F081
:105CA0007CCF80912B158823A1F3973079F038F4BD
:105CB000953079F710924E021092DC12EACF9A30AA
:105CC00049F09F3031F70F941B00E3CF81E08093C0
:105CD000AE09DFCF81E08093AD09DBCF9091C000AA
:105CE00095FFFCCF8093C6000895CF92DF92EF928C
:105CF000FF92CF936B017C01C42F4A3069F4F7FE09
:105D00000BC0F094E094D094C094C11CD11CE11C51
:105D1000F11C8DE20E946E2E4C2FC701B601CF916F
:105D2000FF90EF90DF90CF900C942AC4CF93DF9335
:105D3000EC01FE0184912196882319F00E946E2EB9
:105D4000F8CFDF91CF9108952F923F924F925F92BB
:105D50006F927F928F929F92AF92BF92CF92DF927B
:105D6000EF92FF920F931F93CF93DF93CDB7DEB7E0
:105D7000C059D1090FB6F894DEBF0FBECDBF0E9447
:105D800056278823B9F183E50E946325882309F407
:105D90004BC08DED9EE00E94962E8AE00E946E2EF2
:105DA0008EEF8093A70581E0809378021092A6057C
:105DB00081E09AE59093CE148093CD148CE490E02A
:105DC0009093D0148093CF1487E08093C11482E81D
:105DD0008093C41484E890E0A0E0B0E08093C51400
:105DE0009093C614A093C714B093C81481E794E1AC
:105DF0000E94389EC057DF4F0FB6F894DEBF0FBE2B
:105E0000CDBFDF91CF911F910F91FF90EF90DF9069
:105E1000CF90BF90AF909F908F907F906F905F904A
:105E20004F903F902F90089583E40E94632588232C
:105E300049F00E9440270E94F2D10E9447D10E945F
:105E4000F0A6D8CF20909D0C30909E0C40909F0CD7
:105E50005090A00C8091A60C80FF05C09091CC0BB7
:105E600098609093CC0B869581708093CB0B81EAE0
:105E70009FE00E94BDBD80912C0C90912D0C9E0145
:105E80002F5F3F4F7901009799F09F938F9388E997
:105E90009FE09F938F933F932F930F94A638C70152
:105EA0000E948FBD0F900F900F900F900F900F904A
:105EB00080912A0C90912B0C009799F09F938F93CF
:105EC0008FE89FE09F938F93FF92EF920F94A638F5
:105ED000C7010E948FBD0F900F900F900F900F90F1
:105EE0000F906E0131E8C30ED11C6091040C7091CB
:105EF000050C8091060C9091070C860123E041E08F
:105F00000F94DC339F938F938DE79FE09F938F9344
:105F1000FF92EF920F94A638C7010E948FBD85E7CC
:105F20009FE00E94BDBD87E08093000D8093E5094E
:105F300092E2692E9CE0792E0F900F900F900F90B7
:105F40000F900F90B12CA12C28E6822E2FE0922EDC
:105F5000F30161917191819191913F01860123E05B
:105F600041E00F94DC339F938F93BF92AF929F9247
:105F70008F92FF92EF920F94A638C7010E948FBDB7
:105F80000FB6F894DEBF0FBECDBFAA94AB2809F0C0
:105F900065C18091210C811115C08091200C1F9248
:105FA0008F938CE59FE09F938F93FF92EF920F94D6
:105FB000A638C7010E948FBD0F900F900F900F90D1
:105FC0000F900F908091200C1F928F9386E59FE099
:105FD0009F938F93FF92EF920F94A638C7010E9470
:105FE0008FBD80912E0C0F900F900F900F900F90FF
:105FF0000F908823A1F01F928F931F921F9289E424
:106000009FE09F938F93FF92EF920F94A638C70162
:106010000E948FBD0FB6F894DEBF0FBECDBF80913A
:106020002F0C8823A9F01F928F931F9281E08F93EA
:1060300089E49FE09F938F93FF92EF920F94A6388D
:10604000C7010E948FBD0FB6F894DEBF0FBECDBF53
:106050008090300C9090310CA090320CB090330CAA
:1060600020E030E0A901C501B4010F940F3981117E
:1060700004C08091A60C82FF20C0860121E041E08F
:10608000C501B4010F94DC339F938F938091A60CCC
:1060900082FB882780F91F928F938CE39FE09F9368
:1060A0008F93FF92EF920F94A638C7010E948FBD85
:1060B0000FB6F894DEBF0FBECDBF88E39FE00E940D
:1060C000BDBD6091F60B7091F70B8091F80B90912C
:1060D000F90B8E010F581F4F23E041E00F94DC3382
:1060E000B82EA92E6091F20B7091F30B8091F40BF6
:1060F0009091F50B860123E041E00F94DC33AF92E1
:10610000BF929F938F9387E29FE09F938F93FF921D
:10611000EF920F94A638C7010E948FBD6091FA0BD1
:106120007091FB0B8091FC0B9091FD0B23E041E003
:106130000F94DC338CE19FE00E94BDBDDF92CF92D3
:1061400082E19FE09F938F93FF92EF920F94A63886
:10615000C7010E948FBD8091030C8F938091020C28
:106160008F938BE09FE09F938F93FF92EF920F941A
:10617000A638C7010E948FBD6091FE0B7091FF0B86
:106180008091000C9091010C23E041E00F94DC33EE
:106190009F938F9381E09FE09F938F93FF92EF9265
:1061A0000F94A638C7010E948FBD8CE0E8E0FCE0A8
:1061B000A5EEBBE001900D928A95E1F78CE0E4E159
:1061C000FCE0A9EDBBE001900D928A95E1F780E03B
:1061D0000E94B48B81E00E94B48B82E00E94B48B59
:1061E0008091A50C8093CD0B81E080935E090E9485
:1061F000482784E39CE09F938F938AEB9BE29F93D5
:106200008F93FF92EF920F94A6380FB6F894DEBFEB
:106210000FBECDBFC7010E948FBD8091A40C8F938C
:106220008091A30C8F938091A20C8F938091A10CED
:106230008F935F924F923F922F9283EF9EE09F93B6
:106240008F93FF92EF920F94A638C7010E948FBDE3
:106250000FB6F894DEBF0FBECDBFCCCDAA24A39459
:10626000B12C76CE80915D05827149F480915F05F5
:106270008C7829F480916005837009F475C082E4FC
:106280000E946325882351F00E94C81E6093120D5E
:106290007093130D8093140D9093150D83E50E9458
:1062A0006325882351F00E9439256093420D709335
:1062B000430D8093440D9093450D84E50E94632522
:1062C000882351F00E9439256093460D7093470D45
:1062D0008093480D9093490D88E50E94632588239B
:1062E00051F00E943925609373097093740980936B
:1062F00075099093760989E50E946325882351F0FA
:106300000E94392560937709709378098093790901
:1063100090937A098AE50E9463258823B1F00E9450
:10632000392560937B0970937C0980937D09909354
:106330007E092DEC3CEC4CEC5DE30F940F39181604
:1063400024F085E39EE00E94962E85E40E9463255A
:10635000882351F00E94392560937F09709380094A
:1063600080938109909382090895AF92BF92CF9252
:10637000DF92EF920F931F93CF93DF935B01EA01BC
:106380006901882309F463C08EE29EE00E94962E84
:10639000F501608171818281938146E00E9420D461
:1063A000E1100BC085E29EE00E94962E6881798103
:1063B0008A819B8146E00E9420D48EE19EE00E946B
:1063C000962EF601608171818281938143E00E9463
:1063D00020D487E19EE00E94962EF80160817181B1
:1063E0008281938143E00E9420D48EE09EE00E944F
:1063F000962EF6012081318142815381F80160811E
:106400007181828193810F94DE3F43E00E9420D40A
:10641000EE20F9F08AE00E946E2E89EF9DE00E9446
:10642000962E688179818A819B8146E00E9420D4E2
:106430008AE00E946E2E8AE0DF91CF911F910F912A
:10644000EF90DF90CF90BF90AF900C946E2EE11044
:10645000E4CFDF91CF911F910F91EF90DF90CF901C
:10646000BF90AF9008950F931F93CF938C01C62FC9
:1064700084E298E00E94962EC8010E94962ECC23BA
:1064800031F08AE0CF911F910F910C946E2ECF9135
:106490001F910F910895CF92DF92EF92FF920F9389
:1064A0001F93CF93DF9300D01F92CDB7DEB77C014F
:1064B0006B018A0161E08FED98E00E94333245E282
:1064C00058E166EE78E085E00F946302909118122F
:1064D00081E0890F809318128091371582FF06C0E2
:1064E0008B7F809337159E5F909318120E94AF9F09
:1064F00080E1E2E6FDE0A5E1B5E001900D928A952C
:10650000E1F70E94038881E00F94740B20E030E0F3
:10651000A901F70160817181828193810F940F3904
:106520008823F1F08091CB0B81110CC08091420245
:106530009091430201972091C9123091CA122817F5
:10654000390774F080E090E0A0E7B2E489839A8391
:10655000AB83BC83BE016F5F7F4FC7010E94B391C5
:1065600087E00E94D48B811103C0B6010E94CC97B2
:1065700020E030E0A901F80160817181828193817E
:106580000F940F39882319F0C8010F94BA0B0E9499
:106590009C2A81E00F900F900F900F90DF91CF9188
:1065A0001F910F91FF90EF90DF90CF90089560E0E2
:1065B0008DEF98E00E9433328EE298E00E94962E92
:1065C0008AE00C946E2EEF92FF920F931F93CF935D
:1065D0007C018B01C42F60E08DEF98E00E94333284
:1065E000C7010E94962E80E20E946E2EC8010E9472
:1065F000962ECC2319F08C2F0E946E2E8AE0CF911C
:106600001F910F91FF90EF900C946E2EDF92EF92FE
:10661000FF920F931F93CF93DF93D82E7B018A01B4
:10662000E9010E94D732D092DD1240E0B70181E14A
:1066300099E00E94E3320115110531F040E0B80104
:106640008AE099E00E94E332209731F040E0BE01F9
:106650008AE099E00E94E33260E08DEF98E00E94CA
:10666000333285E099E00E94962E8AE0DF91CF9147
:106670001F910F91FF90EF90DF900C946E2EAF92D0
:10668000BF92CF92DF92EF92FF920F931F93CF931F
:10669000DF9381E997E00E94962EC0E0D7E0D150C9
:1066A00021F080E20E946E2EFACF8C2F0F949C0076
:1066B000CF5FC53099F78AE00E946E2E07E61BE097
:1066C000C0E080E20E946E2E8C2F0F949C00580137
:1066D000D5E080E20E946E2EF501C080D180E2807C
:1066E000F380A7019601C701B6010F94D142882318
:1066F00069F180E20E946E2E8DE30E946E2E8DE382
:106700000E946E2E8DE30E946E2E8DE30E946E2EEF
:106710008DE30E946E2ED150F4E1AF0EB11CD11169
:10672000D8CF8AE00E946E2ECF5F0C5F1F4FC5301E
:1067300041F68AE0DF91CF911F910F91FF90EF908A
:10674000DF90CF90BF90AF900C946E2E20E030E0A1
:10675000A901C701B6010F943F4287FD03C08BE238
:106760000E946E2E43E0C701B6010E9420D4D3CF11
:10677000CF93DF93EB010E94962ECE01DF91CF9154
:106780000D945A01CF93C62F0E94962E8C2FCF9135
:106790000D949C00CF92DF92EF92FF926A017B01F1
:1067A0000E94962E42E0C701B601FF90EF90DF9065
:1067B000CF900C9420D4CF92DF92EF92FF926A0197
:1067C0007B010E94962E4AE0C701B601FF90EF9030
:1067D000DF90CF900C94752ECF93DF93EB010E9446
:1067E000962ECE01DF91CF910D94A3008111B0C000
:1067F00087E69EE00E94962E4091C0095091C10903
:106800006091C2097091C3098FE89EE00E94CA336B
:106810004091C8095091C9096091CA097091CB098A
:1068200086EC9FE20E94CA334091C4095091C50989
:106830006091C6097091C7098FEC9FE20E94CA332C
:106840006091CC097091CD09072E000C880B990B33
:106850000F941639AB01BC0189EC9FE20E94CA3348
:106860006091CE097091CF09072E000C880B990B0F
:106870000F941639AB01BC018CE89EE00E94CA332C
:106880006091D0097091D109072E000C880B990BEB
:106890000F941639AB01BC0189E89EE00E94CA330F
:1068A0006091D4097091D50986E89EE00E94EC338E
:1068B0006091D6097091D70983E89EE00E94EC337D
:1068C0006091F00970E080E89EE00E94EC336091F6
:1068D000EF0970E090E080E00F941439AB01BC0147
:1068E0008DE79EE00E94CA336091D80970E090E085
:1068F00080E00F941439AB01BC018AE79EE00E944E
:10690000CA334091D9095091DA096091DB0970913D
:10691000DC0989E69EE10E94CA334091DD0950916D
:10692000DE096091DF097091E00985ED9FE20E9428
:10693000CA334091E1095091E2096091E3097091F5
:10694000E40982ED9FE20E94CA338AE00C946E2E25
:1069500083E79EE04FCF8F929F92AF92BF92CF92EC
:10696000DF92EF92FF920F931F93CF93DF9300D0AC
:1069700000D01F921F92CDB7DEB781E50E9463253C
:10698000882309F464C120E030E0A9016091C409C2
:106990007091C5098091C6099091C7090F943F4233
:1069A00018160CF041C18091CB0B81110DC0809164
:1069B00042029091430201972091CB123091CC1268
:1069C000281739070CF430C180E1E2E6FDE0ABE4C2
:1069D000BBE001900D928A95E1F78091E5098770FF
:1069E000F12C873009F089C0F090D809FF2009F414
:1069F00084C02091E1093091E2094091E30950916E
:106A0000E40960916A0D70916B0D80916C0D90910D
:106A10006D0D0F94DF3F60936A0D70936B0D809343
:106A20006C0D90936D0D80906D0290906E02A09011
:106A30006F02B0907002A50194010F943F421816A6
:106A400044F480926A0D90926B0DA0926C0DB092FE
:106A50006D0D20E030E040E05FE360912E0D70911D
:106A60002F0D8091300D9091310D0F947539698300
:106A70007A838B839C83CE0101960E942A900E9488
:106A800003888091D9099091DA09A091DB09B0912E
:106A9000DC098093620D9093630DA093640DB09315
:106AA000650D8091DD099091DE09A091DF09B0911B
:106AB000E0098093660D9093670DA093680DB093E5
:106AC000690DE090011280E090E0A8ECB2E48983C7
:106AD0009A83AB83BC83A12CB12C65018E010F5F1F
:106AE0001F4F2EE63DE04AE65DE066E67DE082E689
:106AF0009DE00E945C880E9403886091CC0970919F
:106B0000CD09072E000C880B990B0F94163920E045
:106B100030E040E752E40F94D9406D837E838F8349
:106B200098872091C4093091C5094091C6095091B8
:106B3000C7096091C0097091C1098091C209909103
:106B4000C3090F94DF3F69837A838B839C83BE01E3
:106B50006B5F7F4FCE0101960E94B391FF2021F120
:106B60008091660D9091670DA091680DB091690DAF
:106B70004091620D5091630D6091640D7091650DAF
:106B800040934B0B50934C0B60934D0B70934E0BFB
:106B900080934F0B9093500BA093510BB093520BDB
:106BA0008EE29DE00E94BF8F6091D0097091D10963
:106BB000072E000C880B990B0F94163920E030E05B
:106BC00040E752E40F94D9406D837E838F8398878A
:106BD00020E030E0A9016091C8097091C909809155
:106BE000CA099091CB090F94DF3F69837A838B8325
:106BF0009C83BE016B5F7F4FCE0101960E94B391D3
:106C00008091570B9091580BA091590BB0915A0B52
:106C100080936E0D90936F0DA093700DB093710DD6
:106C20008EE69DE00E94C18928960FB6F894DEBFDB
:106C30000FBECDBFDF91CF911F910F91FF90EF90CD
:106C4000DF90CF90BF90AF909F908F90089583E595
:106C50000E94B1258823F1F00E9439256B017C0147
:106C600020E030E0A9010F940F3987FD3FC120E0FB
:106C700030E84BE354E4C701B6010F943F421816C5
:106C80000CF438C1C092C009D092C109E092C20987
:106C9000F092C30982E40E94B1258823F9F00E9492
:106CA00039256B017C0120E030E040E251EC0F948B
:106CB0000F3987FD27C120E030E040E251E4C701F1
:106CC000B6010F943F4218160CF423C1C092C809B4
:106CD000D092C909E092CA09F092CB0985E40E94DA
:106CE000B1258823F1F00E9439256B017C0120E059
:106CF00030E0A9010F940F3987FD12C120E030E880
:106D00004BE354E4C701B6010F943F4218160CF44C
:106D10000BC1C092C409D092C509E092C609F09295
:106D2000C70980E50E94B125882399F00E94392582
:106D30000F944B41693185E1780714F068E175E102
:106D40006A30710514F46AE070E07093CD096093C5
:106D5000CC0982E50E94B125882399F00E9439254B
:106D60000F944B41693185E1780714F068E175E1D2
:106D70006A30710514F46AE070E07093CF09609393
:106D8000CE0985E50E94B125882399F00E94392516
:106D90000F944B41693185E1780714F068E175E1A2
:106DA0006A30710514F46AE070E07093D109609361
:106DB000D00987E50E94B125882369F00E94392512
:106DC00011E020E030E0A9010F940F39811101C0DA
:106DD00010E01093D80988E50E94B1258823D1F0EE
:106DE0000E9439250F944B4177FDA6C06C3381E09A
:106DF000780714F06BE371E0072E000C880B990BF9
:106E00000F9416396093D9097093DA098093DB09DE
:106E10009093DC0989E50E94B1258823D1F00E9476
:106E200039250F944B4177FD8BC0653381E078079E
:106E300014F064E371E0072E000C880B990B0F949B
:106E400016396093DD097093DE098093DF09909312
:106E5000E0098AE50E94B125882351F00E94392576
:106E60006093E1097093E2098093E3099093E40948
:106E70001092EE098CE40E94B125882379F00E94DB
:106E800035258230910550F48093EF0991E02091EF
:106E90000112281708F090E09093F00981E40E9415
:106EA0006325882321F00E9425258093F00984E53D
:106EB0000E946325882309F449C080912E05909192
:106EC0002F05892B09F446C00E9435258230910593
:106ED000D8F52091011228171906B1F18F5F809320
:106EE000EE090E94CFDA1092EE099ECEC12CD12C71
:106EF0007601C8CEC12C30E8D32E3BE3E32E34E438
:106F0000F32EC0CEC12CD12C20E2E22E21ECF22EA9
:106F1000DDCEC12CD12C90E2E92E91E4F92ED6CE13
:106F2000C12CD12C7601F5CEC12C80E8D82E8BE374
:106F3000E82E84E4F82EEDCE60E070E0CB0162CF65
:106F400060E070E0CB017DCF1092EE0980E00E94FE
:106F5000F6336ACE0E94CFDA67CE2F923F924F92DD
:106F60005F926F927F928F929F92AF92BF92CF92D9
:106F7000DF92EF92FF920F931F93CF93DF93CDB7E2
:106F8000DEB7CB54D1090FB6F894DEBF0FBECDBF2C
:106F90002DB73EB739AF28AF87E00E943BBD8111C6
:106FA0000BC061E086E50E94DB258DA3853060F093
:106FB00084ED9DE00E94962EA8ADB9AD0FB6F89471
:106FC000BEBF0FBEADBF3DC33DA1332321F084EB57
:106FD0009DE00E94962E6AE080E50E94DB25182F36
:106FE0008CEF810F8F3218F080E99DE0E3CF60E0F5
:106FF00085E40E942B27882309F448C081E08FABE9
:10700000E0906613F0906713D7012D913D914D915B
:107010005C916091620D7091630D8091640D90910F
:10702000650D0F94DF3FAB01BC0188E50E94E725A9
:1070300069877A878B879C87F70124813581468110
:1070400057816091660D7091670D8091680D9091E8
:10705000690D0F94DF3FAB01BC0189E50E94E72574
:107060006D877E878F87988BBE01635F7F4FCE01D0
:1070700009960E945420382E81110BC063E68CE7DC
:107080009DE00E9408A384E69DE094CF92E09FAB30
:10709000B7CF8CE40E946325082F882309F431C1FF
:1070A0000E94451F8EA3803118F08DE39DE082CFB2
:1070B000FEA1F13009F427C160E083E50E942B278F
:1070C0008AAF882321F0011102C037E03EA38DA1D1
:1070D000833020F083E29DE00E94962E9091010D76
:1070E0009DAF80E00E945B290E94A08F1D8A1E8AAE
:1070F0001F8A188E198E1A8E1B8E1C8E83EF9FE4AA
:10710000A3ECB7E48D8F9E8FAF8FB8A383EF9FE47E
:10711000A3ECB7EC89A39AA3ABA3BCA3A12FB0E0C7
:10712000BCA7ABA7EDB7FEB724E0129FE019F109A9
:1071300011240FB6F894FEBF0FBEEDBF8DB79EB7FA
:1071400001969CAF8BAF2DA14FA9BE01635F7F4F0E
:10715000CE0109960F94810C9B01AC010F94D14292
:1071600081115FC20F94231061157105810591058E
:1071700011F00F949534212C1BAA1CAA1DAA1EAA3B
:10718000AEA1A150BB0B2C96BFAFAEAF2C97E22D9A
:10719000F0E0F8A7EFA32BA53CA5E217F3070CF04E
:1071A00071C23196FEA7EDA73F932F93FF93EF9304
:1071B0008FE09DE09F938F9389E19DE09F938F9354
:1071C0001F920F940D048DB79EB709960FB6F894D1
:1071D0009EBF0FBE8DBF9EA1992309F455C10F9488
:1071E00046342AE030E040E050E00F94753F0F94C1
:1071F000163920E030E040EA50E40F943F420FEFB0
:107200001FEF181614F001E010E00F94463428E642
:1072100031E040E050E00F94753F0F9416392B0198
:107220003C010F94463420E230E040E050E00F94FF
:10723000753F6B5F7F4F8F4F9F4F0F9416394B01F8
:107240005C01ADA1A430D1F4BC01A40181E09DE0BA
:107250000E94CA33B301A20189EF9CE00E94CA33A5
:1072600083EF9CE00E94962E0130110519F483E40F
:107270000E946E2E8FEE9CE00E94962E312CC8014B
:10728000110FAA0BBB0B2A968CAF9DAFAEAFBFAF51
:107290002A972C96AEADBFAD2C973A161B060CF074
:1072A000F3C02A966CAD7DAD8EAD9FAD2A970F943D
:1072B00016396B017C01BAADBB2341F1AC019B01D6
:1072C0000F94DF3F20E030E040E952E40F9475393D
:1072D0009B01AC01C301B2010F94DF3F2B013C01C4
:1072E00020E030E044EB53E40F943F421816FCF4E6
:1072F00020E030E044EB53E4C301B2010F94DE3FE1
:10730000EDCF1EA2D9CE22E02EA3D6CE0F944634C6
:1073100024E130E040E050E00F94753F675E7F4F1E
:107320008F4F9F4F0F941639A7019601CFCF20E0C2
:1073300030E0A901C301B2010F940F3987FF0BC0E0
:1073400020E030E044EB53E4C301B2010F94DF3F8F
:107350002B013C01ECCF0091661310916713F801EB
:1073600024813581468157816D857E858F859889F9
:107370000F94DE3F22966CAF7DAF8EAF9FAF22970A
:107380002BED3FE049E450E4C301B2010F9475399D
:1073900020E030E044E353E40F94D9406B017C01DA
:1073A0000F94D4406FA778AB89AB9AABD8012D91DD
:1073B0003D914D915C9169857A858B859C850F9473
:1073C000DE3F26966CAF7DAF8EAF9FAF2697A501AF
:1073D00094016FA578A989A99AA90F9475399B0181
:1073E000AC0126966CAD7DAD8EAD9FAD26970F940A
:1073F000DF3F69837A838B839C83C701B6010F9437
:107400007F42A50194010F94753922962CAD3DADB4
:107410004EAD5FAD22970F94DF3F6D837E838F83E8
:1074200098874BE351E070E060E0CE0101960E9446
:10743000C2DE44E351E070E060E0CE0105960E94B8
:10744000C2DEBDA1B43099F449815A816B817C813F
:1074500083EE9CE00E94CA334D815E816F81788506
:1074600085ED9FE20E94CA338AE00E946E2E198A3F
:107470001A8A1B8A1C8ABE016F5E7F4FCE0101965D
:107480000F94680E339405CF20E04FA9BE01635FCF
:107490007F4FCE0109960F94810C4B015C01312C7A
:1074A000AC019B010F94D142811102C0332433946B
:1074B000A5019401C501B4010F94D1428111E2C02C
:1074C000EFA1F8A5EE0FFF1FEE0FFF1F2BAD3CAD98
:1074D000E20FF31F80829182A282B382A501940100
:1074E0006D8D7E8D8F8D98A10F943F42181624F4D8
:1074F0008D8E9E8EAF8EB8A2A501940169A17AA14E
:107500008BA19CA10F940F3987FF04C089A29AA276
:10751000ABA2BCA2A50194016BA97CA98DA99EA9CF
:107520000F94DF3F6BAB7CAB8DAB9EABADA5BEA527
:10753000BD01BB0F880B990B0F9416396FA378A769
:1075400089A79AA79B01AC016BA97CA98DA99EA9CB
:107550000F94D9402B013C014D8A5E8A6F8A788E48
:10756000EBADFCADF8ABEFA710E0C12CD12C760150
:10757000AFA5B8A96D917D918D919D91B8ABAFA745
:10758000A30192010F94DE3F9B01AC010F9475396A
:107590009B01AC01C701B6010F94DF3F6B017C0179
:1075A0001F5F211628F72FA138A549A55AA50F94CA
:1075B000D9400F948D42698F7A8F8B8F9C8FBDA19C
:1075C000B23068F18DA59EA50F94A3006BA57CA594
:1075D0008EED9CE00E94EC3388ED9CE00E94962E9C
:1075E00043E0C501B4010E9420D480E20E946E2EC7
:1075F00081E0EDA1E3300CF480E0E12C8E010F5D21
:107600001F4F9E01235E3F4FAE01475E5F4FBE019D
:107610006B5E7F4F0E94B5318AE00E946E2E2394EC
:10762000B6CD0E944B200E94878F8DAD0E945B29B2
:107630000E949D9288AD99AD0FB6F8949EBF0FBE83
:107640008DBFE8ADF9AD0FB6F894FEBF0FBEEDBF2C
:10765000C55BDF4F0FB6F894DEBF0FBECDBFDF9125
:10766000CF911F910F91FF90EF90DF90CF90BF903F
:10767000AF909F908F907F906F905F904F903F90D2
:107680002F9008950E944B20332069F28DEC9CE0EE
:107690000E94962E81E0FDA11F160CF080E0EE24E2
:1076A000E3948E010F5D1F4F9E01235E3F4FAE019D
:1076B000475E5F4FBE016B5E7F4F0E94B531698DA3
:1076C0007A8D8B8D9C8D0052110926E042E00F943B
:1076D000DC339F938F938CEB9CE09F938F9386EC8E
:1076E0009CE09F938F931F920F940D042DB73EB78C
:1076F000295F3F4F0FB6F8943EBF0FBE2DBF93CF0B
:107700002F923F924F925F926F927F928F929F92B1
:10771000AF92BF92CF92DF92EF92FF920F931F939F
:10772000CF93DF93CDB7DEB7CC58D1090FB6F8941D
:10773000DEBF0FBECDBF8DEA9BE00E94962E87E094
:107740000E943BBD81116EC084E50E94B125882353
:1077500029F00E94352560E00E942FD880E090E05B
:10776000A0E8BFE389839A83AB83BC838D839E8328
:10777000AF83B8878DEC9CECACE4BEE389879A8735
:10778000AB87BC8780E090E0A0E2B1E48D879E8764
:10779000AF87B88B8CE390E09A8B898B8DEC90E06F
:1077A0009C8B8B8B8DEC9CECACECBEE38D8B9E8B21
:1077B000AF8BB88F80E090E0A0EEBFE3898F9A8F07
:1077C000AB8FBC8F1BA61CA64AE959E969E97EE389
:1077D0008FE40E94E7256D8F7E8F8F8F98A360E0E6
:1077E00083E40E942B2789A360E08BE40E942B276F
:1077F0008AA382E40E94B125882381F10E94352565
:10780000009761F19C01285231092536310520F19C
:107810006CE870E08FE79BE00E94EC338AE79BE026
:107820000E94962EC457DF4F0FB6F894DEBF0FBEEE
:10783000CDBFDF91CF911F910F91FF90EF90DF901F
:10784000CF90BF90AF909F908F907F906F905F9000
:107850004F903F902F9008959A8B898B8CE40E94D3
:10786000B1258823E1F00E9439256B017C01C9868E
:10787000DA86EB86FC8620E030E0A9010F943F42D7
:1078800087FD0AC020E030E040E050E4C701B601C7
:107890000F940F3918161CF482E59BE0C1CF81E5E7
:1078A0000E946325882331F180912E0590912F0548
:1078B000892BE9F00E9439256B017C01CD82DE82A3
:1078C000EF82F8862DEC3CEC4CE45DE30F943F42F4
:1078D00087FD0AC020E030E040E751E4C701B6016F
:1078E0000F940F39181634F481E29BE099CF86EF9C
:1078F0009AE096CF83E50E94B1258823E9F00E94A3
:1079000039256B017C01CD8ADE8AEF8AF88E2DEC59
:107910003CEC4CEC5DE30F943F4287FD0AC020E055
:1079200030E040E050E4C701B6010F940F3918165B
:107930001CF48FEC9AE074CF80E50E9463258823C5
:1079400041F180912E0590912F05892B19F487E93B
:107950009AE066CF8BA58F5F8BA70E9439256B01BC
:107960007C01CD86DE86EF86F88A20E030E0A90132
:107970000F943F4287FD0AC020E030E048EC51E41C
:10798000C701B6010F940F3918161CF48FE69AE060
:1079900047CF86E40E94B1258823E9F00E9439256B
:1079A0006B017C01C98EDA8EEB8EFC8E20E030E01C
:1079B00040E85FE30F943F4287FD0AC020E030E0DB
:1079C00040E850E4C701B6010F940F3918161CF4B3
:1079D00086E49AE025CFC98CDA8CEB8CFC8C8D8800
:1079E0009E88AF88B88CA7019601C701B6010F9495
:1079F00075399B01AC0160E070E084E490E40F9481
:107A0000D94029813A814B815C810F9475392B01D2
:107A10003C01A5019401C501B4010F947539A7017A
:107A200096010F9475392CEE31E548EB5DE30F9428
:107A3000D9409B01AC01C301B2010F947539698330
:107A40007A838B839C8388E40E94B125882379F014
:107A50000E943525009759F09C01255A3109283894
:107A6000310518F088E19AE0DBCE9C8B8B8B85E5A5
:107A70000E9463258823C9F00F94231061157105B6
:107A80008105910511F00F94953480912E05909108
:107A90002F05892B91F00E94392560932A05709358
:107AA0002B0580932C0590932D0582E50E9463257C
:107AB000811108C084EE99E0B3CE60E070E088E404
:107AC00092E4EBCF80912E0590912F05892B61F0E8
:107AD0000E943525AD969FAF8EAFAD97181619064B
:107AE0004CF080EB99E09CCE2AE130E0AD963FAFC0
:107AF0002EAFAD9789E50E94B125882381F10E94C0
:107B000039252091B80C3091B90C4091BA0C5091A4
:107B1000BB0C0F94DE3F6B017C0188E50E94B12510
:107B2000882331F10E9439252091B40C3091B50C95
:107B30004091B60C5091B70C0F94DE3F6BA37CA321
:107B40008DA39EA3CFA2D8A6E9A6FAA6CE018396BE
:107B50000E94F91A811115C086E899E061CEC090A3
:107B6000660DD090670DE090680DF090690DD5CF4F
:107B70006091620D7091630D8091640D9091650D1F
:107B8000DDCF84E40E94632591E089270E945B2970
:107B900080E090E0A0EAB0E48DA79EA7AFA7B8ABC5
:107BA00060E0CE018D960E9446913091D80BCD5762
:107BB000DF4F3883C358D0401092D80B0E94C08842
:107BC00085E699E00E94962E89899A898A319105E5
:107BD0000CF046C08B899C890E94858761E080916A
:107BE00001120E94AFD6811143C06FEF8AE799E07E
:107BF0000E9408A38CA5811104C0CE0101960F94A8
:107C00006E0E80E090E0A0EAB0E48093530B909376
:107C1000540BA093550BB093560B1DA61EA61FA682
:107C200018AABE01635D7F4F8BE49BE00E94002297
:107C3000CD57DF4F5881C358D0405093D80B0E9486
:107C4000C0888AA18111EECD109262121092611249
:107C50000E948ADB8091011290E00E948587E2CD2C
:107C60000E941A2581E00E9437D58111B3CFBDCF84
:107C700010926E0D10926F0D1092700D1092710D8A
:107C80008EE69DE00E94C1898BA5882309F452C02D
:107C900020E030E040E751E46091320D7091330D07
:107CA0008091340D9091350D0F94D9406DA77EA72A
:107CB0008FA798AB80E1E2E6FDE0ABE4BBE001908A
:107CC0000D928A95E1F72D853E854F855889609103
:107CD000570B7091580B8091590B90915A0B0F9440
:107CE000DF3F6093570B7093580B8093590B909321
:107CF0005A0BCE018D960E94BF8F2D853E854F85F4
:107D000058896091570B7091580B8091590B909145
:107D10005A0B0F94DE3F6093570B7093580B809370
:107D2000590B90935A0B8CA5811104C0CE0101967A
:107D30000F946E0EE5E2F5E085E0DF011D928A9575
:107D4000E9F780E1E2E6FDE0ABE4BBE001900D92F3
:107D50008A95E1F789859A85AB85BC858093530B1D
:107D60009093540BA093550BB093560B1DA61EA6D3
:107D70001FA618AABE01635D7F4F8BE49BE00E94A3
:107D80000022BE01635E7F4F8BE49BE00E940022D5
:107D900089A1882309F41CC42091620D3091630DE0
:107DA0004091640D5091650DE5962CAF3DAF4EAFFF
:107DB0005FAFE5978091660D9091670DA091680D7A
:107DC000B091690DE1968CAF9DAFAEAFBFAFE197BB
:107DD000312C212C9FEFA4969FAFA497AFEFA896CC
:107DE000AFAFA897BFEFC158DF4FB883CF57D04090
:107DF000EFE4C058DF4FE883C058D040F3ECCF57D2
:107E0000DF4FF883C158D04027E4CE57DF4F288397
:107E1000C258D04081E090E0A0E0B0E0022C04C065
:107E2000880F991FAA1FBB1F0A94D2F7CC57DF4FA8
:107E300088839983AA83BB83C458D040A5E2B5E068
:107E4000E796BFAFAEAFE79710E000E09101032CDB
:107E5000000C440B550BC857DF4F288339834A83E6
:107E60005B83C858D040C457DF4F2882CC58D040DD
:107E7000E796AEADBFADE7978D91E796BFAFAEAFDA
:107E8000E79790E0B0E0A0E0CC57DF4F2881398140
:107E90004A815B81C458D04082239323A423B52315
:107EA000892B8A2B8B2B09F024C1C857DF4F68819F
:107EB00079818A819B81C858D0400F9416392091CE
:107EC0006709309168094091690950916A090F94D6
:107ED000753920915F093091600940916109509195
:107EE00062090F94DF3FEB966CAF7DAF8EAF9FAF13
:107EF000EB97B801012E000C880B990B0F941639E3
:107F000020916B0930916C0940916D0950916E0977
:107F10000F94753920916309309164094091650986
:107F2000509166090F94DF3F6B017C01EB962CADFD
:107F30003DAD4EAD5FADEB97E5966CAD7DAD8EADD5
:107F40009FADE5970F94DE3F2B013C01A701960101
:107F5000E1966CAD7DAD8EAD9FADE1970F94DE3FA8
:107F60004B015C01A3019201C301B2010F94753969
:107F70002B013C01A5019401C501B4010F94753991
:107F80009B01AC01C301B2010F94DF3F0F948D42FE
:107F90004B015C01EB962CAD3DAD4EAD5FADEB976B
:107FA0006BA17CA18DA19EA10F94DE3F2B013C0112
:107FB000A70196016FA178A589A59AA50F94DE3F28
:107FC0006B017C01A3019201C301B2010F947539C9
:107FD0002B013C01A7019601C701B6010F94753929
:107FE0009B01AC01C301B2010F94DF3F0F948D429E
:107FF00020E030E040E751E40F94D940A50194011E
:108000000F94DF3F6B017C0180902A0590902B0537
:10801000A0902C05B0902D0520E030E040E85FE313
:10802000C501B4010F943F421816F4F4C501B40120
:108030000F944B414B015C0160E070E0CB011814E0
:1080400019041A041B0434F40F944634A501940156
:108050000F94753F0F9416399B01AC01B601C7010F
:108060000F94DF3F6B017C01C158DF4F2881CF5750
:10807000D040C058DF4F3881C058D040CF57DF4F75
:108080004881C158D040CE57DF4F5881C258D040A8
:10809000B601C7010F940F3987FF2BC0A4960FAF0D
:1080A000A497C457DF4F3881CC58D040A8963FAF33
:1080B000A897EC96CFAEEC97ED96DFAEED97EE96E7
:1080C000EFAEEE97EF96FFAEEF97C158DF4FC88245
:1080D000CF57D040C058DF4FD882C058D040CF577C
:1080E000DF4FE882C158D040CE57DF4FF882C258E8
:1080F000D0400F5F1F4F0530110509F0B9CE4FEF8B
:10810000241A340A55E02516310409F083CEA496CA
:108110008FADA497E82FF0E0EB5DFA4F208181E06E
:1081200090E0A0E0B0E0A8960FACA89704C0880F3C
:10813000991FAA1FBB1F0A94D2F7822B8083A8968F
:108140009FADA8976A969FAF6A97A496AFADA49784
:108150006B96AFAF6B97EC968FADEC97ED969FADAE
:10816000ED97EE96AFADEE97EF96BFADEF976F96AA
:108170008CAF9DAFAEAFBFAF6F97A896BFADA897BE
:10818000BF3F09F409C2A496EFADA497EF3F09F4ED
:1081900003C26B2FBB0F770B880B990B0F9416390B
:1081A00020916709309168094091690950916A09E5
:1081B0000F94753920915F093091600940916109F0
:1081C000509162090F94DF3F162F072F382E292E6A
:1081D000862F902FA32DB22D65968CAF9DAFAEAF9D
:1081E000BFAF6597A496FFADA4976F2FFF0F770BD6
:1081F000880B990B0F94163920916B0930916C09FB
:1082000040916D0950916E090F9475392091630961
:108210003091640940916509509166090F94DF3FE0
:108220006B017C016996CCAEDDAEEEAEFFAE699718
:10823000CE018F5A9F4F0E94F91A882309F4B0C1CA
:1082400020E030E040EA50E4612F702F832D922D22
:108250000F94DF3F4B015C01CB01D50121968CAF20
:108260009DAFAEAFBFAF21972596CCAEDDAEEEAEE3
:10827000FFAE2597A8962FADA8972111E3C1A4962C
:108280003FADA4973111B3C120E030E040EA50E4A3
:10829000C701B6010F94DF3F6B017C01A4964FAD7F
:1082A000A497442309F4C5C1A4968FADA497843044
:1082B0000CF0BFC122ED422E23E5522E2BE7622E99
:1082C00021E4722E21968CAC9DACAEACBFAC219754
:1082D00025968CAD9DADAEADBFAD2597A7968CAF65
:1082E0009DAFAEAFBFAFA7979C01AD0169966CADD6
:1082F0007DAD8EAD9FAD69970F94DE3FAB966CAFB1
:108300007DAF8EAF9FAFAB97A501940165966CAD25
:108310007DAD8EAD9FAD65970F94DE3F2D966CAF12
:108320007DAF8EAF9FAF2D97AB962CAD3DAD4EADD3
:108330005FADAB9761962CAF3DAF4EAF5FAF61972E
:10834000A50194016091620D7091630D8091640D9F
:108350009091650D0F94DE3F4B015C01A7962CAD0B
:108360003DAD4EAD5FADA7976091660D7091670D05
:108370008091680D9091690D0F94DE3FA7966CAFC8
:108380007DAF8EAF9FAFA797812F902FA32DB22DDA
:108390008DA79EA7AFA7B8ABC9AADAAAEBAAFCAA79
:1083A000C984DA84EB84FC84CDAADEAAEFAAF8AEF5
:1083B0002DEC3CEC4CEC5CE3C301B2010F9475393D
:1083C00029813A814B815C810F94753920916E0D22
:1083D00030916F0D4091700D5091710D0F94DF3FF2
:1083E00069AF7AAF8BAF9CAFA5019401C501B40111
:1083F0000F9475394B015C01A7962CAD3DAD4EAD88
:108400005FADA797CA01B9010F9475399B01AC0103
:10841000C501B4010F94DF3F20E030E040E050E4BC
:108420000F943F421816ACF420E030E040E05FE3E8
:10843000C701B6010F94DF3F29966CAF7DAF8EAFB9
:108440009FAF2997BE01635C7F4FCE0101960E94CA
:10845000D81E89859A85AB85BC8529968CAF9DAF42
:10846000AEAFBFAF2997A3961CAE1DAE1EAE1FAE1A
:10847000A397BE01615A7F4FCE01CD960E94002284
:108480008CA58823C1F02AE939E949E95FE36D81C8
:108490007E818F8198850F947539A3966CAF7DAFDF
:1084A0008EAF9FAFA397BE01615A7F4F8BE49BE0D5
:1084B0000E9400221CA6E0902A0DF0902B0D009146
:1084C0002C0D10912D0DA090260DB090270DC09071
:1084D000280DD090290D9501A601B701C8010F9470
:1084E0003F42181614F47501860180905302909053
:1084F0005402A0905502B09056022DEC3CEC4CEC8E
:108500005DE3B701C8010F9475396093530270930E
:108510005402809355029093560240E0BE01675B7F
:108520007F4FCE018D960F94722780E1E2E6FDE049
:10853000ABE4BBE001900D928A95E1F78092530283
:1085400090925402A0925502B092560220E04FEF52
:10855000BE01675A7F4FCE0101960E947B2320E027
:1085600041E0BE01675A7F4FCE0101960E947B23F6
:108570002FEF40E0BE01675A7F4FCE0101960E9467
:108580007B2321E040E0BE01675A7F4FCE01019678
:108590000E947B230E9403888091720D8093730D4B
:1085A000AD964EAD5FADAD9741505109AD965FAF01
:1085B0004EAFAD97452B09F418CB6A968FAD6A97ED
:1085C00087FD13CB6B968FAD6B9787FFE1CB0DCB00
:1085D0002BA13CA14DA15EA1E5962CAF3DAF4EAFC6
:1085E0005FAFE5978FA198A5A9A5BAA5EBCB812F81
:1085F000902FA32DB22D21968CAF9DAFAEAFBFAF04
:10860000219720E030E040EA50E4C701B6010F9422
:10861000DE3F25966CAF7DAF8EAF9FAF2597A496BA
:108620005FADA49754300CF42FCE182D092D3A2CA1
:108630002B2C92ED492E93E5592E9BEF692E90E459
:10864000792E40CEA8969FADA89794300CF452C0D6
:10865000A496AFADA497A4300CF120E030E040EA3E
:1086600050E4612F702F832D922D0F94DE3F2196C1
:108670006CAF7DAF8EAF9FAF219720E030E040EA36
:1086800050E4C701B6010F94DE3F6B017C01A49654
:10869000EFADA497E4300CF40DCECBCF812F902F0B
:1086A000A32DB22D21968CAF9DAFAEAFBFAF21975A
:1086B00020E030E040EA50E4C701B6010F94DF3F0C
:1086C00025966CAF7DAF8EAF9FAF2597A496BFADBB
:1086D000A497B111D2CF20E030E040EA50E4612FFE
:1086E000702F832D922D0F94DE3F162F072F382EDB
:1086F000292E9FCFA496FFADA497F1110DC020E0C5
:1087000030E040E251E4B401C5010F94DE3F162F82
:10871000072F382E292ECECDA4962FADA497243026
:108720009CF020E030E040E251E4B401C5010F9438
:10873000DE3F21966CAF7DAF8EAF9FAF2197182D96
:10874000092D3A2C2B2CB6CD182D092D3A2C2B2C7B
:1087500082ED482E83E5582E8BEF682E81E4782E2B
:10876000B1CD8AE897E00C94962E84E897E00C94BB
:10877000962ECF9384E50E94B125C09101128823E3
:10878000D9F00E94451FC82F8230B4F00E94B54333
:108790008DE40E946E2E80915A0590915B050F9496
:1087A0005A016C2FCC0F770B8CEA9FE00E94EC33C0
:1087B0008AE00E946E2ECFEF8C2FCF9108954F92BA
:1087C0005F926F927F928F929F92AF92BF92CF9261
:1087D000DF92EF92FF921F93CF93DF9300D000D0F0
:1087E0001F921F92CDB7DEB70E94B943D82E87FDE6
:1087F000B2C08AE50E94B125812C912C20E2A22EE4
:1088000021E4B22E882341F040E050E0BA018AE52D
:108810000E94E7254B015C0110910112ED2C0D2CFB
:10882000000CFF081E151F0421F060E08D2D0E9432
:108830002FD820E030E0A901C501B4010F943F42D8
:1088400018167CF580E090E0A0EAB0E48D839E836A
:10885000AF83B88720916A0D30916B0D40916C0DFC
:1088600050916D0DC501B4010F94DF3F2B013C0108
:1088700020E030E048EC53E40F940F3987FD06C048
:10888000412C512C98EC692E93E4792E49825A821E
:108890006B827C82BE016B5F7F4FCE0101960E948E
:1088A000279184E50E94B12581116BC0809101124E
:1088B000882321F060E080E00E942FD880914E094B
:1088C00090914F09A0915009B0915109B0588983F6
:1088D0009A83AB83BC83CE0101960F94BA0B20E040
:1088E00030E0A901C501B4010F943F4218165CF5B0
:1088F00080E090E0A0EAB0E48D839E83AF83B887E8
:10890000A501940160916A0D70916B0D80916C0DC1
:1089100090916D0D0F94DE3F6B017C0120E030E003
:10892000A9010F943F4218161CF0C12CD12C7601DE
:10893000C982DA82EB82FC82BE016B5F7F4FCE017F
:1089400001960E94279180910112811721F060E029
:10895000812F0E942FD828960FB6F894DEBF0FBE45
:10896000CDBFDF91CF911F91FF90EF90DF90CF901F
:10897000BF90AF909F908F907F906F905F904F903F
:10898000089585E50E9463258823D1F00E9439254A
:108990006B017C0120E030E0A901C701B6010F9412
:1089A0003F4287FF04C0F7FAF094F7F8F094F7FA23
:1089B000F094F7F8F094C982DA82EB82FC828BCFD4
:1089C000F70183E0EE0FFF1F8A95E1F7E25BF64FB8
:1089D000C080D180E280F380DDCFAF92BF92CF9292
:1089E000DF92EF92FF920F931F93CF93DF936091EB
:1089F000011270E084E50E94CC258230C0F08FE344
:108A00000E946E2E84E50E946E2E8FEB9EE00E94E7
:108A1000962E84EB9EE0DF91CF911F910F91FF90F6
:108A2000EF90DF90CF90BF90AF900C94962E992747
:108A3000EC01CC0FDD1FCC0FDD1FFE01EA51F64F1C
:108A4000A080B180C280D3808BE40E94B1258823AE
:108A500039F10E9439257B018C0120E030E0A90129
:108A60000F943F4287FD0AC020E030E040E251E42D
:108A7000B701C8010F940F391816A4F48FE30E94B0
:108A80006E2E8BE40E946E2E8FEB9EE00E94962E3F
:108A900087EB9EE00E94962E84EB9EE00E94962E2D
:108AA000750186019501A601B701C8010F940F3920
:108AB000882351F00E940388CA51D64FA701B801FC
:108AC000488359836A837B8380915D0590915E051D
:108AD000A0915F05B0916005892B8A2B8B2BD9F56E
:108AE0000E94B54383ED9EE00E94962E80E20E9494
:108AF0006E2E80E30E946E2E8AE30E946E2E60919D
:108B0000E6097091E7098091E8099091E90942E04E
:108B10000E9420D480E20E946E2E81E30E946E2E7D
:108B20008AE30E946E2E6091EA097091EB098091B0
:108B3000EC099091ED0942E00E9420D48AE0DF9197
:108B4000CF911F910F91FF90EF90DF90CF90BF904A
:108B5000AF900C946E2EDF91CF911F910F91FF90EB
:108B6000EF90DF90CF90BF90AF9008954F925F92BB
:108B70006F927F928F929F92AF92BF92CF92DF922D
:108B8000EF92FF92CF93DF93CDB7DEB72C970FB65E
:108B9000F894DEBF0FBECDBF4090B40C5090B50C22
:108BA0006090B60C7090B70C2091590230915A0227
:108BB00040915B0250915C02C301B2010F94DF3F10
:108BC00069837A838B839C838090B80C9090B90CD6
:108BD000A090BA0CB090BB0C20915D0230915E0267
:108BE00040915F0250916002C501B4010F94DF3FD4
:108BF0006D837E838F839887C090BC0CD090BD0C12
:108C0000E090BE0CF090BF0C2091610230916202A6
:108C10004091630250916402C701B6010F94DF3F97
:108C200069877A878B879C872091650230916602DD
:108C30004091670250916802C301B2010F94DF3F77
:108C40002B013C012091690230916A0240916B0234
:108C500050916C02C501B4010F94DF3F4B015C01E0
:108C600020916D0230916E0240916F02509170021E
:108C7000C701B6010F94DF3F6B017C010E94B54331
:108C800084EA9EE00E94962E83E50E946325882355
:108C900021F00E942525809357028091570281116F
:108CA00051C084EA93E10E94962E8CE99EE00E94D6
:108CB000962E49815A816B817C8189E69EE10E94D2
:108CC000CA334D815E816F81788585ED9FE20E9478
:108CD000CA3349855A856B857C8582ED9FE20E9467
:108CE000CA338AE99EE00E94962E82E99EE00E94A5
:108CF000962EB301A20189E69EE10E94CA33B50116
:108D0000A40185ED9FE20E94CA33B701A60182ED5E
:108D10009FE20E94CA338AE02C960FB6F894DEBF19
:108D20000FBECDBFDF91CF91FF90EF90DF90CF903E
:108D3000BF90AF909F908F907F906F905F904F907B
:108D40000C946E2E88EA93E1AECF2F923F924F9211
:108D50005F926F927F928F929F92AF92BF92CF92CB
:108D6000DF92EF92FF920F931F93CF93DF93CDB7D4
:108D7000DEB76A970FB6F894DEBF0FBECDBF83E5AE
:108D80000E946325182F3090010D882319F00E944E
:108D90002525382E4090620D5090630D6090640D33
:108DA0007090650D8091660D9091670DA091680D92
:108DB000B091690D8B8B9C8BAD8BBE8B80916A0DB6
:108DC00090916B0DA0916C0DB0916D0D8F8B988F64
:108DD000A98FBA8F112329F0311003C080E00E94BF
:108DE0005B2986E50E9463258A8B20E030E0A9019B
:108DF00060916709709168098091690990916A0989
:108E00000F940F39882309F4C9C083E40E946325B5
:108E1000882309F49DC00E9439256B017C01A7E6D7
:108E2000BBE0B987A887BF83AE83F5E0FD831D86CD
:108E30001E8628EC2F8702EC1A86212C88EC8B8763
:108E400092E49C87AE81BF81B98BA88B15E0E8893D
:108E5000F98981909190A190B190F98BE88B2A8546
:108E6000322D4B855C85C501B4010F940F3987FF06
:108E700004C08A86292CAB86BC862D853E854F850D
:108E8000502FC501B4010F943F42181624F48D866B
:108E90009E86AF860B2D1150D1F6FD81F150FD83DA
:108EA0008E819F8144969F838E83F111CBCF2D8538
:108EB0003E854F85502F6A85722D8B859C850F943A
:108EC000DF3F20E030E040E05FE30F947539A70119
:108ED00096010F94DF3F4B015C012DEB37E346E831
:108EE00055EB0F943F4287FD0AC02DEB37E346E870
:108EF00055E3C501B4010F940F3918164CF580E005
:108F00000E945B2910E0E884F98400E0D7016D91AC
:108F10007D918D919D917D016D01B4E0CB1AD108B9
:108F2000A50194010F94DE3FF60160837183828373
:108F30009383602F812F0F94670A0F5F053031F7FD
:108F40001F5F888599854496998788871530D9F65B
:108F5000AA89AA2381F020E030E0A9016091670985
:108F6000709168098091690990916A090F940F398D
:108F700081110E943F338AE50E946325882351F0C6
:108F80000E94392569837A838B839C83CE01019665
:108F90000F941D09832D0E945B290BC0311003C063
:108FA0009A89992341F30E94B5438DEF9BE00E947B
:108FB000962E332051F08091010D811106C00E9440
:108FC000B1438EED9BE00E94962E0E94B54380ED4A
:108FD0009BE00E94962E8091010D811172C084EA5F
:108FE00093E10E94962E8AE00E946E2E0E94B54365
:108FF00083EC9BE00E94962EC090B00CD090B10CF8
:10900000E090B20CF090B30C20E030E0A901C70171
:10901000B6010F943F4218160CF056C042E0C7014B
:10902000B6010E9420D48DE00E946E2E8AE00E943C
:109030006E2EA30192016091620D7091630D80917B
:10904000640D9091650D0F940F3981111FC02B890C
:109050003C894D895E896091660D7091670D8091A4
:10906000680D9091690D0F940F3981110FC02F89F0
:10907000388D498D5A8D60916A0D70916B0D80917C
:109080006C0D90916D0D0F940F3981110E949D927E
:109090006A960FB6F894DEBF0FBECDBFDF91CF91B9
:1090A0001F910F91FF90EF90DF90CF90BF90AF9006
:1090B0009F908F907F906F905F904F903F902F90F8
:1090C000089588EA93E18DCF8EEB9BE00E94962E67
:1090D000B0CF0E94B7DB0E94D32A80E00F94740BBC
:1090E0008091BE0A8130A1F40E94B1438DE097E0E7
:1090F0000E94962E60E083E097E00E9408A36EE550
:1091000071E080E090E00E94782A88E08093BE0AB7
:109110000895CF92DF92EF92FF921F93CF93DF9348
:1091200000D01F92CDB7DEB78EEEC82E82E0D82ECB
:10913000E12CF12CC982DA82EB82FC82BE016F5FE6
:109140007F4F8AE50E94342C81110EC010E0812FE0
:109150000F900F900F900F90DF91CF911F91FF9084
:10916000EF90DF90CF9008950E948A2CC982DA8216
:10917000EB82FC82BE016F5F7F4F8AE50E94342C38
:10918000182F882319F30E94B14387EE97E00E94BD
:10919000962E0E946948DBCFCF92DF92EF92FF922A
:1091A0001F93CF93DF9300D01F92CDB7DEB78EEE23
:1091B000C82E82E0D82EE12CF12CC982DA82EB8213
:1091C000FC82BE016F5F7F4F8AE00E94342C8111C8
:1091D0000EC010E0812F0F900F900F900F90DF9135
:1091E000CF911F91FF90EF90DF90CF9008950E9454
:1091F0008A2C0E94542C0E946F2C0E94542CC982ED
:10920000DA82EB82FC82BE016F5F7F4F8AE00E94B0
:10921000342C182F8823E9F20E94B1438AEA97E0A0
:109220000E94962E0E946948D5CF5F926F927F92DE
:109230008F929F92AF92BF92CF92DF92EF92FF9266
:109240000F931F93CF93DF931F92CDB7DEB77C01AF
:1092500039018B015B01A40EB51ED12CC12CA016C7
:10926000B10609F450C0F70180809180F801519057
:109270008F015982C4010F942D3F5816B9F1652D05
:10928000C4010F94353FFFEFCF1ADF0AC6018F7775
:109290009927892B21F162E070E080E090E00F9443
:1092A000F00FC4010F942D3F99818917F9F00E94A6
:1092B000B5438FE694E00E94962E81E00F90DF91F7
:1092C000CF911F910F91FF90EF90DF90CF90BF90C3
:1092D000AF909F908F907F906F905F90089562E025
:1092E00070E080E090E00E94782ADBCFBE016F5FE3
:1092F0007F4FC3010F942E00F70180819181019669
:1093000091838083ACCF80E0D9CFCF93DF93CDB76B
:10931000DEB7A8970FB6F894DEBF0FBECDBF8C01A5
:10932000F42E0E94B7DB0E94B14383EE96E00E94C8
:10933000962E0115110511F40AED16E08091A8058D
:1093400080FD79C081608093A80586EC96E00E943C
:10935000962E8AE00E946E2ECC24C3948AE5D82EE5
:10936000D092CE14C092CD148FE090E09093D014A0
:109370008093CF1497E0792E7092C11422E8E22EE8
:10938000E092C41434E8832E912CA12CB12C80924D
:10939000C5149092C614A092C714B092C81481E765
:1093A00094E10E94389ED092CE14C092CD1488E5EC
:1093B00090E09093D0148093CF147092C114E092F7
:1093C000C4148092C5149092C614A092C714B0928F
:1093D000C81481E794E10E94389E8AE289838A83D7
:1093E0008B838C83F801DE011596BE016F5F7F4F82
:1093F000CD01861B970B2491319621110CC0FB01E6
:10940000E80FF91F8AE29F01261B370B283231052E
:1094100024F48193F8CF2D93EBCF20E630E140E0A8
:1094200050E081E794E10F9449006AE070E080E049
:1094300090E00E94F99D61E081ED96E00E94333258
:1094400089EE93E030E6019729F0232F2A9500005A
:10945000E9F7F9CFF89489EE93E038EE019729F017
:10946000232F2A950000E9F7F9CF0E94B7DBFF20F0
:1094700031F00E94AC2A0E943D1BA895FECF0E94AD
:109480003A1BF9CF8091720D9091730D2FEF3FEF42
:10949000981751F0E92FF0E0EE58F24F228130E0BA
:1094A0009F5F9F779093730DC90108951F920F924C
:1094B0000FB60F9211240F900FBE0F901F901895AA
:1094C0001F920F920FB60F9211240BB60F920F93AB
:1094D0001F932F933F934F935F936F937F938F933C
:1094E0009F93AF93BF93CF93DF93EF93FF93C0917D
:1094F000C6000091730DD091720D11E01D0F1F7702
:1095000090913F04913108F09FC0E92FF0E0882747
:10951000E357F54B8F4F0D94D63F9E4ACD4ADC4A18
:10952000EB4AF24A244BF64A244BFA4AFE4A244BB1
:10953000024B064B0A4B114B244B1C4BC03229F0FB
:1095400028F5CA3011F0CD3031F5011731F0ED2F8B
:10955000F0E0EE58F24FC283D12FD093720DFF91FD
:10956000EF91DF91CF91BF91AF919F918F917F91BB
:109570006F915F914F913F912F911F910F910F909C
:109580000BBE0F900FBE0F901F901895CD3481F039
:1095900081E0CE3471F080E10CC0CA3338F4C033BE
:1095A000A0F6C03291F2CD32B1F7CFCFCD3499F7DA
:1095B00082E080933F04C9CFC13359F018F4C03220
:1095C00021F2E9CF88E0C433A1F38BE0C83389F3FB
:1095D000E2CF83E0EECF84E0C03359F386E0C133BD
:1095E00041F3D9CF85E0C833B1F6E3CF87E0C2338A
:1095F00091F6DFCF89E0C13371F6DBCF8AE0C0336B
:1096000051F6D7CF8CE0C73331F6D3CF8DE0C633D8
:1096100011F6CFCFC03209F498CF8EE0C33549F2AE
:10962000BACF80ED8C0F8A3008F08FCF9FE09093F7
:109630003F048093400489CFCA3019F0CD3009F03F
:1096400084CF10923F0481CFCA3019F0CD3009F099
:109650007CCF80912B158823A1F3973079F038F4D3
:10966000953079F710924E021092DC12EACF9A30C0
:1096700049F09F3031F70F941B00E3CF81E08093D6
:10968000AE09DFCF81E08093AD09DBCF8EBD0DB495
:1096900007FEFDCF08958FEF8EBD0DB407FEFDCF01
:1096A0008EB50895909164009B7F90936400982FED
:1096B000906A96959CBD80FD03C091E0863009F4C8
:1096C00090E09DBD0895CF93DF93EB010E94962E0D
:1096D000CE01DF91CF910C94EFC82F923F924F9221
:1096E0005F926F927F928F929F92AF92BF92CF9232
:1096F000DF92EF92FF920F931F93CF93DF9300D0EF
:1097000000D000D01F921F92CDB7DEB7B82E809147
:109710006F0E843008F0D1C10F9423106B017C01CF
:1097200080916F0E811108C08091720D9091730D20
:10973000891B8F7709F4FDC581E6A82E13C08A30F6
:1097400019F08D3009F0F6C010925A0E8091F80D84
:109750009091F90DFC01EC50F24F1682892BF1F437
:109760000E9404DF80916F0E843008F0ECC080917D
:10977000720D9091730D891B8F7709F4E4C00E94DC
:10978000424A97FFDCCF0E94B14385EB95E00E94EF
:10979000962E8091720D8093730DE4CF1092F90D87
:1097A0001092F80D0AEF1DE0F8018191803209F462
:1097B00046C08E3409F0A9C060EB75E0C8010F9473
:1097C0008C384C01892B41F06EE470E0C80104969E
:1097D0000F942D43009709F4C8014AE050E070E06F
:1097E00060E001960F94FC352B013C018091F40D53
:1097F0009091F50DA091F60DB091F70D0196A11D78
:10980000B11D481659066A067B0629F060E08DE70F
:1098100095E0892851F16AE270E0C8010F945C4339
:109820009C01009729F1982F901B912C992349F0C6
:109830009150F801E90FF11D80819826F7CF8F0133
:10984000B3CF4AE050E070E060E0C90101960F94A8
:10985000FC35292D30E050E040E0621773078407A3
:10986000950751F060E08EE595E00F9414077ACFEC
:1098700060E084E395E0F9CF4092F40D5092F50D4D
:109880006092F60D7092F70D8091BE0A8130E1F082
:1098900067E470E0C8010F942D430097A9F04AE0F7
:1098A00050E070E060E001960F94FC356430710583
:1098B0008105910548F483E994E00E94962E60E0CA
:1098C00089E894E00E9408A3C0925F0BD092600BDD
:1098D000E092610BF092620B8091FA0D8B3309F4E8
:1098E00041CF80916F0E843008F03CCF8091710E93
:1098F0008A9DC00111246AEF7DE08E58914F0F942C
:10990000384380E00F94CE062DCF8091371580FF2D
:10991000BBCF68EF7DE2C8010F948C38009731F01F
:10992000FC01838180538A3008F0AECF60E08AE08A
:1099300095E09BCF28EF3DE04AEF5DE06AE57EE0F1
:109940000E94D5B80FCF8091371582FFB6C01A821A
:10995000198271E6F72EE0E1EE2EF9E6DF2E809116
:109960006F0E843008F0A9C00E940DB98111A5C006
:1099700041E050E0BE016B5F7F4F8BE996E10E94B2
:1099800044CB0D8110E0019711F00FEF1FEF809194
:10999000A3169091A416A091A516B091A616809337
:1099A000331590933415A0933515B09336150E9456
:1099B0000DB90F3F100749F4811107C00E94B14350
:1099C00083ED95E00E94962ECACF4091710E242F10
:1099D00030E00A3061F00D3051F0882309F45FC0A7
:1099E00089819A81009719F001969A838983109250
:1099F000C60489819A81F29EF001F39EF00D112434
:109A0000E159F14FE80FF91F1382892B69F50E9484
:109A100004DF0E940DB9882309F4A1CF0E940388B6
:109A20008BE996E10E94F1CC80912E15882391F16B
:109A3000815080932E158D9DC001112462E08A50C3
:109A4000964F0E9446D2E0912E1524E0E29FF0014D
:109A50001124EE50F64F60817181828193810E94C2
:109A6000C7B80E94F9C47BCF1A82198281E00F9493
:109A7000CE068091331590913415A0913515B09193
:109A8000361580936B0E90936C0EA0936D0EB09371
:109A90006E0EBFCF0E94FACCE092BE0A60CF4F9DFF
:109AA000A00111244E58514F9E012F5F3F4F66EC8D
:109AB00074E0802F0E94D5B852CF0F9423106B0111
:109AC0007C01B11004C080911812882351F0C0921B
:109AD0001212D0921312E0921412F0921512BB24BB
:109AE000B39480913A0590913B05A0913C05B091CB
:109AF0003D050097A105B105B1F0409112125091BA
:109B000013126091141270911512840F951FA61FE5
:109B1000B71FA7019601281B390B4A0B5B0BDA0113
:109B2000C901B7FF92C18091140290911502A091D2
:109B30001602B0911702892B8A2B8B2B09F099C141
:109B40000F9423104B015C018091DC12811108C03D
:109B500020916B1390916C1381E0291301C080E078
:109B60002091C9123091CA1291E089272A3A310511
:109B70000CF480E091E04091CB045091CC046091D2
:109B8000CD047091CE04452B462B472B09F490E071
:109B9000981789F0882309F4BDC1D501C401805606
:109BA0009444A24FBF4F8093CB049093CC04A093D6
:109BB000CD04B093CE0440906E0D50906F0D609028
:109BC000700D7090710D2091C7043091C8044091C0
:109BD000C9045091CA04C301B2010F940F398823FC
:109BE00019F18091CB049091CC04A091CD04B09157
:109BF000CE044092C7045092C8046092C904709287
:109C0000CA04892B8A2B8B2B09F449C0D501C401C6
:109C100080569444A24FBF4F8093CB049093CC04C2
:109C2000A093CD04B093CE048091CB049091CC044A
:109C3000A091CD04B091CE040097A105B10579F1B2
:109C4000881A990AAA0ABB0AB7FC29C01092CB0449
:109C50001092CC041092CD041092CE0483E396E0CF
:109C60000E94962E60E08FE196E00E9408A380910A
:109C7000CB129091CC121816190624F490E080E0D3
:109C80000E948587809161129091621218161906C0
:109C900034F410926212109261120E948ADB809159
:109CA000D3049091D404A091D504B091D604460178
:109CB0005701881A990AAA0ABB0AD501C401B7FD3F
:109CC000B9C120916B1390916C1380913402409133
:109CD0003502291323C19091CE0B899FC001112415
:109CE000880F892F881F990B91958D838091CF0BB9
:109CF000489FC0011124880F892F881F990B9195C7
:109D00008E830F94231069837A838B839C8340E036
:109D1000BE016F5F7F4FCE0105960E9443896D8122
:109D200070E089E00F941A0F41E0BE016F5F7F4F32
:109D3000CE0105960E9443896E8170E087E00F9402
:109D40001A0F8091BB09882309F467C100911C0296
:109D500010911D02C80102972091CB123091CC12B4
:109D6000281739070CF459C180906C138F8218861C
:109D700019861A861B8680916B139F80891509F4BA
:109D8000E7C0892D90E038E6A32EA89EF001A99E99
:109D9000F00D1124EE53FA4F458956896789708D6D
:109DA000452B462B472B81F4418D528D638D748D4D
:109DB000452B462B472B41F4458D568D678D70A161
:109DC000452B462B472BE1F128E6B22EB89E900199
:109DD000B99E300D1124A9014E535A4F1A01FA01B0
:109DE00061817281838194810F948D424B015C016A
:109DF000F10161A172A183A194A10F9414392B01E7
:109E00003C01F10165A176A187A190A50F941439B9
:109E10009B01AC01C301B2010F94D940A50194018B
:109E20000F9475394B015C01288539854A855B851E
:109E30000F943F42181624F488869986AA86BB861A
:109E40008F818F5F87708F8396CF0E94B14360911F
:109E50005D0B70915E0B82EE95E00E94634B8AE091
:109E60000E946E2E40E070E060E090E080E00E9492
:109E7000854990916B1380916C13981749F0C092AB
:109E80001212D0921312E0921412F092151258CEC0
:109E9000BB2019F01092D70453CE0F9423100091D9
:109EA00012121091131220911412309115128090F9
:109EB000140290901502A0901602B0901702080D9F
:109EC000191D2A1D3B1D601B710B820B930B97FD07
:109ED000E1CF8091D704811133CE81E08093D70404
:109EE0005F9A8091000D8E7F8093000D8A9A8091F9
:109EF000000D8D7F8093000D809108018095817009
:109F0000809306018091000D8B7F8093000D0E944D
:109F10003A1B16CE80E090E0DC0145CE20916C1318
:109F200058E6259F900111242E533A4FF901EE591E
:109F3000FF4F9081899FC0011124880F892F881FAE
:109F4000990B91958D832D593F4FF9018081D0CE8A
:109F500020913A0230913B0240913C0250913D02E7
:109F6000688579858A859B850F9475394B015C01DD
:109F7000B801012E000C880B990B0F9416399B0128
:109F8000AC01C501B4010F94DF3F69837A838B83F1
:109F90009C8340911A0250911B02B801CE01019698
:109FA0000E94C2DE89809A80AB80BC804090CF0442
:109FB0005090D0046090D1047090D204A30192011B
:109FC000C501B4010F940F3987FF16C028E431EEA4
:109FD0004AE75FE3C301B2010F94753920E037ED22
:109FE00043EA5CE30F94DF3FA50194010F947539B8
:109FF00069837A838B839C8369817A818B819C813D
:10A000006093CF047093D0048093D1049093D204D2
:10A010000F944B41CB010E948587F4E6CF0ED11CF3
:10A02000E11CF11CC092D304D092D404E092D50478
:10A03000F092D6040E9404DF8091BE0A882309F4BE
:10A0400039C190910901892F80958170109100028A
:10A050001817C9F020913715206220933715809387
:10A06000000290FD40C164EF71E080E090E00E944A
:10A07000782A0E941CCD8091371583FD7DC1111176
:10A0800034C10E94BAA70F9423106B017C01109178
:10A0900013021123F1F080913E058823D1F0409105
:10A0A000D8045091D9046091DA047091DB04460120
:10A0B0005701841A950AA60AB70AB501A40177FDCB
:10A0C0001AC0833009F430C10CF01FC181300CF08C
:10A0D00024C1212F30E0A8EEB3E00F94A73FC60EB5
:10A0E000D71EE81EF91EC092D804D092D904E0927F
:10A0F000DA04F092DB0480911912813009F073C008
:10A100000F9423106B017C018091E0049091E10495
:10A11000A091E204B091E304A7019601281B390B3A
:10A120004A0B5B0BDA01C901B7FD3AC0D701C60182
:10A13000805F984DAF4FBF4F8093E0049093E10450
:10A14000A093E204B093E30480900609909007097D
:10A15000A0900809B09009090E947F97AB01BC014B
:10A160004093060950930709609308097093090901
:10A1700080916D0A90916E0AA0916F0AB091700A59
:10A1800088199909AA09BB09840F951FA61FB71F33
:10A1900080936D0A90936E0AA0936F0AB093700A31
:10A1A0008091DC049091DD04A091DE04B091DF0485
:10A1B00046015701881A990AAA0ABB0AD501C401A7
:10A1C000B7FD11C020E8C20E2EEED21E26E3E21E1D
:10A1D000F11CC092DC04D092DD04E092DE04F09227
:10A1E000DF040E94FB860E94ED9F0E94CEA8809112
:10A1F0003905882381F10F9423106B017C01809134
:10A20000350590913605A0913705B0913805460186
:10A210005701881A990AAA0ABB0AD501C401B7FDD9
:10A220001AC02091390530E0A8EEB3E00F94A73FA3
:10A23000C60ED71EE81EF91EC0923505D09236050F
:10A24000E0923705F0923805809101120E94C4D443
:10A250008AE00E946E2E80913405882359F10F9474
:10A2600023106B017C018091300590913105A09104
:10A270003205B0913305A7019601281B390B4A0B13
:10A280005B0BDA01C901B7FD15C02091340530E040
:10A29000A8EEB3E00F94A73FC60ED71EE81EF91E26
:10A2A000C0923005D0923105E0923205F09233052C
:10A2B0000E94B7C42B960FB6F894DEBF0FBECDBF79
:10A2C000DF91CF911F910F91FF90EF90DF90CF9092
:10A2D000BF90AF909F908F907F906F905F904F90C6
:10A2E0003F902F9008950E940BCD123008F0CBCEF6
:10A2F0000E94BAA760E080E796E050C08EE796E043
:10A300009093DB128093DA12BECE843009F0E1CE56
:10A310000E94B54385E896E004C00E94B54384EBF3
:10A3200096E00E94962ED5CE0E94B5438DE996E028
:10A33000F8CF80915F0B9091600BA091610BB09171
:10A34000620BA7019601281B390B4A0B5B0BDA0144
:10A35000C901885E9340A109B109B7FDEDC98DEC33
:10A3600095E00E94962EC0925F0BD092600BE09217
:10A37000610BF092620BE0C9123098F488E496E029
:10A380000E94962E8AE00E946E2E0E94149E90E0FB
:10A3900080E00E94A3A060E081E696E00E9408A30E
:10A3A00072CE123009F06FCE0E9476D1882379F0F8
:10A3B00081E00E944CD147EB50E061EF7BE08CE301
:10A3C00095E10E9444CB8CE395E10E94F1CC0E9480
:10A3D0005627811193CF0E9440270E94F2D10E94FC
:10A3E00047D151CE2F923F924F925F926F927F92C0
:10A3F0008F929F92AF92BF92CF92DF92EF92FF9295
:10A400000F931F93CF93DF93CDB7DEB7EE970FB6C1
:10A41000F894DEBF0FBECDBF8091010D888B87E51C
:10A420000E946325882309F423C120E030E0A901BC
:10A4300060916709709168098091690990916A0932
:10A440000F940F39811108C00E94B1438AEA9CE041
:10A450000E94962E10E01FC18AE50E94B125882334
:10A4600039F10E9439252091BC0C3091BD0C4091EE
:10A47000BE0C5091BF0C0F94DE3F6B017C0120E0BD
:10A4800030E040E251ECC701B6010F943F4287FD36
:10A490000AC020E030E040E251E4C701B6010F9469
:10A4A0000F39181674F40E94B1438DE99CE0D0CFA7
:10A4B000C0906A0DD0906B0DE0906C0DF0906D0D1A
:10A4C000DECF40E050E060EC7FE788E50E94E725C2
:10A4D0002091B40C3091B50C4091B60C5091B70C52
:10A4E0000F94DE3F2B013C0140E050E060EC7FE741
:10A4F00089E50E94E7252091B80C3091B90C409174
:10A50000BA0C5091BB0C0F94DE3F4B015C016FEF16
:10A5100089E40E94DB25182F6FEF8AE40E94DB2577
:10A52000082FA3019201C301B2010F94D1428111FE
:10A530006EC0A5019401C501B4010F94D1428111EF
:10A5400066C08BA19CA1ADA1BEA18BAB9CABADABFA
:10A55000BEAB20915F093091600940916109509133
:10A560006209C301B2010F94DE3F2B013C0120E0E0
:10A5700030E040E05FE36BA97CA98DA99EA90F9410
:10A5800075399B01AC01C301B2010F94DF3F2BA9C8
:10A590003CA94DA95EA90F94D9400F944B41162FA9
:10A5A0004FA058A469A47AA420916309309164094A
:10A5B0004091650950916609C501B4010F94DE3FD1
:10A5C0004B015C0120E030E040E05FE3C301B201F9
:10A5D0000F9475399B01AC01C501B4010F94DF3FA5
:10A5E000A30192010F94D9400F944B41062F812F64
:10A5F000012E000C990B97FD33C005979CF5802F19
:10A60000002E000C990B97FD2FC005977CF5153097
:10A6100008F020CF053008F01DCF80E00E945B29B4
:10A6200095E01902F0011124E00FF11D07FDFA95E4
:10A63000EE0FFF1FEE0FFF1FE959F44FC082D182CA
:10A64000E282F382602F812F0F94670A88890E942B
:10A650005B298889882309F4FDCE0E949D92FACE59
:10A6600010E0CDCF14E0CBCF00E0D1CF04E0CFCFCE
:10A670008AE40E946325182F811127C070E060E0F2
:10A6800086E50E94CC259A838983059708F188E79F
:10A690009CE00E94962E812FEE960FB6F894DEBFB6
:10A6A0000FBECDBFDF91CF911F910F91FF90EF9023
:10A6B000DF90CF90BF90AF909F908F907F906F90E2
:10A6C0005F904F903F902F9008950E94A929C2CE8D
:10A6D00060E084E40E942B278F8740E050E0BA01BD
:10A6E0008AE50E94E7256BA77CA78DA79EA740E07F
:10A6F00050E86BE376E483E50E94E72520E030E054
:10A7000040E752E40F94D94060934F027093500297
:10A710008093510290935202E0906613F090671379
:10A72000D7018D909D90AD90BC9020E030E0A901C4
:10A73000C501B4010F94DF3F6BAF7CAF8DAF9EAF0F
:10A7400020E030E040E450E40F940F3987FF06C06A
:10A750001BAE1CAEB0E4BDAFE0E4EEAF20E030E8ED
:10A760004DE953E4C501B4010F94DF3F662E7BAB86
:10A770008FAB98AF20E030E844E953E40F943F42B8
:10A7800018163CF4612CF0E8FBAB24E92FAB33E462
:10A7900038AFD70114968D909D90AD90BC901797CF
:10A7A00020E030E0A901C501B4010F94DF3FD62EAF
:10A7B000E72EF82E092F20E030E040E951E40F9415
:10A7C0000F3987FF05C0D12CE12CF0E9FF2E01E401
:10A7D00020E030E04AE953E4C501B4010F94DF3FC3
:10A7E000B62EC72E89AF9AAF20E030E04DE853E493
:10A7F0000F943F42181634F4B12CC12CBDE8B9AF08
:10A80000E3E4EAAF88E40E946325882309F416C2D2
:10A810000E9439250F944B411B0177FF02C06F5FE7
:10A820007F4F759567957195619571096A567F4F50
:10A83000072E000C880B990B0F941639762E872E55
:10A84000982EA92E2D2D3E2D4F2D502F0F943F4287
:10A8500018161CF4D72C74010A2D2BAD3CAD4DAD50
:10A860005EAD672D782D892D9A2D0F943F421816D5
:10A8700024F07BAC8CAC9DACAEAC872D982DA92D73
:10A88000BA2D8B8B9C8BAD8BBE8B8D2D9E2DAF2DC2
:10A89000B02F8F8B988FA98FBA8FB101330C880B93
:10A8A000990B0F9416391B012C01AC019B016D2DE6
:10A8B0007E2D8F2D902F0F94DF3FD62EE72EF82E72
:10A8C000092F2B2D3C2D49AD5AAD0F940F3987FF21
:10A8D00004C0BD2CCE2CF9AE0AAFA2019101672DA8
:10A8E000782D892D9A2D0F94DF3FD62EE72EF82E46
:10A8F000092F262D3BA94FA958AD0F940F3987FF7B
:10A9000004C06D2CEBAAFFAA08AF862D9BA9AFA9A6
:10A91000B8AD8B8F9C8FAD8FBE8F8B2D9C2DA9AD2D
:10A92000BAAD8F8F98A3A9A3BAA3BE01695E7F4F6A
:10A93000CE0143960E945420882309F4B0C1BE0181
:10A94000615E7F4FCE014B960E945420E82E8823F3
:10A9500009F4A5C12F89388D498D5A8D6F8D78A145
:10A9600089A19AA10F94DE3F20E030E040E85EE349
:10A970000F9475394B015C012B893C894D895E89A7
:10A980006B8D7C8D8D8D9E8D0F94DE3F20E030E0B1
:10A9900040E85EE30F9475396BA37CA38DA39EA35F
:10A9A0008FA298A6A9A6BAA689819A811816190617
:10A9B00074F486E49CE00E94962E8F85882321F013
:10A9C0008CE39CE00E94962E8AE00E946E2E0E94EC
:10A9D00003880E94A08F80E00E945B2980E090E0C5
:10A9E000A0E2B1E48FA798ABA9ABBAAB60E0CE010F
:10A9F0008F960E9446912091670930916809409195
:10AA0000690950916A096BA17CA18DA19EA10F9447
:10AA10000F39811130C020916B0930916C09409140
:10AA20006D0950916E096FA178A589A59AA50F941B
:10AA30000F39811120C020915F0930916009409148
:10AA40006109509162096B897C898D899E890F9477
:10AA50000F39811110C02091630930916409409130
:10AA60006509509166096F89788D898D9A8D0F944B
:10AA70000F398823A9F00E94A92988E0FE01B39626
:10AA8000A7E6B9E001900D928A95E1F788E0FE0112
:10AA90007396AFE5B9E001900D928A95E1F7188AB7
:10AAA00060E085E40E942B27882309F4FBC0F1E0D5
:10AAB000FBAB1B861C861D861E861A8A9E2C4CE0CC
:10AAC000C42E4CE0D42E5AE1A52E5CE0B52E1A8996
:10AAD00015300CF0F7C06B857C858D859E859B01BC
:10AAE000AC010F94D1428111EDC0992009F4DDC071
:10AAF00031E03FAB35E0232E91E09926F12EFF0C9B
:10AB0000FF0CF10EF394898B19896A89121509F4E7
:10AB1000D5C0062E000C770B880B990B0F941639B5
:10AB20002FA138A549A55AA50F9475392F89388DBD
:10AB3000498D5A8D0F94DF3F2B013C01612F110F7E
:10AB4000770B880B990B0F9416392BA13CA14DA1C3
:10AB50005EA10F9475392B893C894D895E890F94CC
:10AB6000DF3F6B837C838D839E834F82588669860B
:10AB70007A8689819A81892B79F06F2D88E29CE011
:10AB80000E94C23369E170E086E29CE00E94EC33EF
:10AB900083E29CE00E94962E1F9299E19F931F9260
:10ABA000FF92DF92CF92BF92AF921F920F940D044B
:10ABB00029814BA9BE01695F7F4FCE0103960F9497
:10ABC000810C2B013C014B865C866D867E860FB620
:10ABD000F894DEBF0FBECDBFAC019B010F94D142F4
:10ABE000811169C089883A8825E0382D32038001B7
:10ABF0001124030D111D37FC1A95000F111F000FB2
:10AC0000111F0959144FA30192016BA57CA58DA5B5
:10AC10009EA50F94DF3FD8016D937D938D939C93F8
:10AC20001397632D882D0F94670A188A81E00E947C
:10AC30006D4BF3948989BFA98B0F65CF4D2D5E2D88
:10AC40006F2D702F86E40E94E7251B012C014BAD70
:10AC50005CAD6DAD7EAD8CE40E94E7256B8B7C8B8B
:10AC60008D8B9E8B2F8A388E498E5A8E4B2D5C2D64
:10AC700069AD7AAD82E40E94E7256B017C01462D27
:10AC80005BA96FA978AD82E50E94E7256B8F7C8F69
:10AC90008D8F9E8FCF8ED8A2E9A2FAA246CE8CE5E8
:10ACA0009CE0F7CC22E02BAB04CF8FEF8FAB2224BC
:10ACB0002A9484E021CF88890E945B298A898F5F4A
:10ACC0008A8B05CF0F94DE030E944B20882359F016
:10ACD00088890E945B2980E090E0A0ECBFE78B8729
:10ACE0009C87AD87BE876B857C858D859E859B0106
:10ACF000AC010F94D142811159C08F85811126C0BA
:10AD000082E0F82E02E094E0C92E12E0DC2CD11A89
:10AD100021E041E0612F802F0E94AF1B21E04FEF27
:10AD2000612F8F2D0E94AF1B2FEF41E06D2D802FE3
:10AD30000E94AF1B2FEF4FEF6D2D8F2D0E94AF1B89
:10AD4000115020F70150F3940F3FF9F60E943F3362
:10AD50000E94FE298F85811124C08AE69DE00E9411
:10AD600086214B015C0182E69DE00E946E279B01DB
:10AD7000AC01C501B4010F9475399B01AC01609120
:10AD80006A0D70916B0D80916C0D90916D0D0F940B
:10AD9000DE3F60936A0D70936B0D80936C0D909302
:10ADA0006D0D8F858111E888E092010D0E94878FDB
:10ADB0008091010D81110E946C920E94AE1E0E9432
:10ADC0009D926B857C858D859E8511E09B01AC01F4
:10ADD0000F94D14281115FCC3DCB8F929F92AF9265
:10ADE000BF92CF92DF92EF92FF920F931F93CF9378
:10ADF000DF9300D01F92CDB7DEB75C016B017A0103
:10AE0000122F002309F443C00E94B54385E399E063
:10AE10000E94962E61E0812F0E94401B90903E057B
:10AE200083E080933E0581E08093DC120E94D7325C
:10AE300082E08093DD1240E365E279E081E199E010
:10AE40000E94E33240E06DE171E18AE099E00E9406
:10AE5000E33260E08DEF98E00E94333285E099E0C4
:10AE60000E94962E8AE00E946E2E87E199E00E9451
:10AE7000459D8091DC12882341F060E0812F0E9483
:10AE8000401B81E00E946D4BF4CF90923E0520E084
:10AE900030E0A901F50160817181828193810F9475
:10AEA0000F39882371F080E090E0A0ECB0E4898352
:10AEB0009A83AB83BC83BE016F5F7F4FC5010E9445
:10AEC000B39120E030E0A901F601608171818281B7
:10AED00093810F940F39882351F180903A0D90900F
:10AEE0003B0DA0903C0DB0903D0D80E090E0A0E7C0
:10AEF000B1E480933A0D90933B0DA0933C0DB09339
:10AF00003D0D80E090E0A0EAB1E489839A83AB83B1
:10AF1000BC83BE016F5F7F4FC6010E94B3918092D8
:10AF20003A0D90923B0DA0923C0DB0923D0D20E069
:10AF300030E0A901F70160817181828193810F94D2
:10AF40003F42181674F480E090E0A0E4B0E48983F6
:10AF50009A83AB83BC83BE016F5F7F4FC7010E94A2
:10AF6000B3912DE131E14CEE58E066EF78E081E0FD
:10AF70000E9406330E94D73281E00F900F900F900D
:10AF80000F90DF91CF911F910F91FF90EF90DF9085
:10AF9000CF90BF90AF909F908F900895CF93C82F80
:10AFA0008091CC0B83FD14C08091CB0B811110C01C
:10AFB00080914202909143029C01215031094091BD
:10AFC000CB125091CC124217530714F40E9485877C
:10AFD000CC2331F061E080910112CF910C94AFD677
:10AFE0008091CB0B91E0892780934E0280914E0295
:10AFF000882389F08091C9129091CA122091CB12B6
:10B000003091CC12821B930B97FF03C091958195D1
:10B010009109029744F410924E028091CC0B83FF69
:10B0200006C0C1E01AC080E00E946D4BDFCFC09126
:10B03000CB0BC11112C08091420290914302019743
:10B040002091CB123091CC122817390754F70E9467
:10B05000B5438EEC98E00E94962E8C2FCF910895E8
:10B060009F92AF92BF92CF92DF92EF92FF920F9397
:10B070001F93CF93DF93CDB7DEB764970FB6F894E5
:10B08000DEBF0FBECDBF0E94B943D82E87FDC6C01C
:10B090008AE50E94B125882309F4D2C040E050E03F
:10B0A000BA018AE50E94E7257B018C01B09001126C
:10B0B0008D2D0D2C000C990BB816190621F060E0AF
:10B0C0008D2D0E942FD820916A0D30916B0D4091EB
:10B0D0006C0D50916D0D60E070E088EC93E40F947E
:10B0E000DE3F962EA72E6C019701A8010F943F42D8
:10B0F00018161CF0E92CFA2C860120E030E0A9019A
:10B10000B701C8010F943F42181624F4E12CF12C2A
:10B1100000E010E0B701C8010F944B41072E000C6E
:10B12000880B990B0F9416396D837E838F839887D4
:10B1300020E030E0A9010F940F39882321F0CE01DF
:10B1400005960E94501D80E090E0A0EAB1E4898756
:10B150009A87AB87BC871D861E861F86188A8CE45B
:10B160000E946325882309F470C00E9439256B0171
:10B170007C0120E030E0A901C701B6010F943F42F5
:10B1800087FF04C0F7FAF094F7F8F094C98ADA8AD6
:10B19000EB8AFC8A2091CB123091CC1224303105FD
:10B1A00074F08091C9129091CA12821B930B97FF81
:10B1B00003C091958195910901E004970CF400E09A
:10B1C00080E00E94CE57882359F022E0AE01475F0D
:10B1D0005F4FBE016F5E7F4FCE010D960E94ED5610
:10B1E0006D817E818F8198858B019C013058098308
:10B1F0001A832B833C8320E030E0A9010F940F39A0
:10B20000882321F0CE0101960E94501D80910112E9
:10B210008B1521F060E08B2D0E942FD864960FB61D
:10B22000F894DEBF0FBECDBFDF91CF911F910F917C
:10B23000FF90EF90DF90CF90BF90AF909F900895D8
:10B24000E12CF12C00E211E431CFE091011288E011
:10B25000E89FF0011124E25BF64FC480D580E680C0
:10B26000F78087CF7F928F929F92AF92BF92CF92BB
:10B27000DF92EF92FF920F931F93CF93DF9300D053
:10B2800000D01F921F92CDB7DEB76C015B014A015F
:10B29000722E78010091B3090E943C9D8091CB12DF
:10B2A0009091CC128E159F051CF4C7010E948587D2
:10B2B00080E00E94CE57882331F0272DA401B501EC
:10B2C000C6010E94ED561E141F0444F4C7010E94DB
:10B2D000858760E0809101120E94AFD681E00E94D4
:10B2E000CE5780E090E0A0E7B2E489839A83AB83F5
:10B2F000BC8380E090E0A0E8B0EC8D839E83AF83B8
:10B30000B887BE016F5F7F4FCE0105960E94B39153
:10B3100087E00E94D48B811158C080916A0D909172
:10B320006B0DA0916C0DB0916D0D40911905509170
:10B330001A0560911B0570911C05C0901505D090F1
:10B340001605E0901705F0901805C0924B0BD092AF
:10B350004C0BE0924D0BF0924E0B40934F0B5093E1
:10B36000500B6093510B7093520B8093530B90933F
:10B37000540BA093550BB093560B80E090E0A8E4DB
:10B38000B2E489839A83AB83BC83CE0101960E9489
:10B39000BF8F80911D0590911E05A0911F05B09152
:10B3A00020058093530B9093540BA093550BB093AF
:10B3B000560B80E090E0A0EAB0E489839A83AB83E7
:10B3C000BC83CE0101960E94BF8FC12CD12C80E797
:10B3D000E82E82E4F82EC982DA82EB82FC8280E0D9
:10B3E00090E0A0E8B0E48D839E83AF83B887BE0170
:10B3F0006F5F7F4FCE0105960E94B39120E030E051
:10B40000A9016091210570912205809123059091F9
:10B4100024050F940F3987FF0BC0C982DA82EB82B3
:10B42000FC82BE016F5F7F4F81E295E00E94B39185
:10B430008091210590912205A0912305B0912405CA
:10B4400080936E0D90936F0DA093700DB093710D5E
:10B450008093570B9093580BA093590BB0935A0BB2
:10B4600087E59BE00E94C18980915E0981110F945C
:10B470009B0961E084E599E00E94333280911812C3
:10B4800081508093181245E258E16CE579E085E03F
:10B490000F94630280911812882339F00E94F9C436
:10B4A0008091181281508093181280E00F94740BD1
:10B4B00080911912823011F40E94029F0F94DE03D2
:10B4C00028960FB6F894DEBF0FBECDBFDF91CF91A7
:10B4D0001F910F91FF90EF90DF90CF90BF90AF90B2
:10B4E0009F908F907F900895CF92DF92EF92FF927E
:10B4F000CF93DF936B017C01D42FC0913E0583E095
:10B5000080933E0581E08093DC12C114D104E104F4
:10B51000F10431F00F942310C60ED71EE81EF91E59
:10B520008091DC12882389F0C114D104E104F10474
:10B5300021F48D2F0E946D4BF3CF0F9423106C19C3
:10B540007D098E099F0997FDF4CF1092DC12C093FC
:10B550003E05DF91CF91FF90EF90DF90CF9008955F
:10B560000F931F93CF93DF93C82F162F0E94B543DD
:10B57000C11194C0C2E3D8E0CE010E94962E61E0D2
:10B58000812F0E94401B0F942310685370458F4FEA
:10B590009F4F6093AF097093B0098093B109909366
:10B5A000B2091092B30900913E0583E080933E05F5
:10B5B00030E020E04DE151E160EC78E082E00E9473
:10B5C000063380EC98E00E94459D81E08093DC1278
:10B5D0008091DC12882309F464C060E0812F0E940E
:10B5E000401B8091B309882309F454C00E94B543DD
:10B5F00086EA98E00E94962E30E020E040E958E08C
:10B6000067E978E082E00E94063387E998E00E94CB
:10B61000459D41E060E070E0CB010E94745A30E04B
:10B6200020E050E040E063E878E085E00E940633E7
:10B6300083E898E00E94B1A60E943C9D80E00E94B1
:10B64000CE570E94B543CE010E94962E0F94231030
:10B65000685370458F4F9F4F6093AF097093B00947
:10B660008093B1099093B2091092B30930E020E0C1
:10B670004DE151E167E778E082E00E94063386E61B
:10B6800098E00E94459D81E08093DC1261E0812F6B
:10B690000E94401B81E00E946D4B9ACFC7E4D8E026
:10B6A0006BCF00933E05DF91CF911F910F910895CD
:10B6B000BF92CF92DF92EF92FF920F931F93CF939F
:10B6C000DF93CDB7DEB7A0970FB6F894DEBF0FBEFD
:10B6D000CDBF0E94B94387FDE0C0B0900112282F72
:10B6E000082E000C330BB216130619F060E00E940E
:10B6F0002FD885E40E946325882309F4DEC00E94C8
:10B7000039256B017C0120E030E0A9010F943F4214
:10B7100087FF04C0F7FAF094F7F8F094F7FAF09482
:10B72000F7F8F094C98ADA8AEB8AFC8A8CE0E1E9BE
:10B73000F2E0DE01119601900D928A95E1F78AE51B
:10B740000E94B125882351F040E050E0BA018AE51B
:10B750000E94E72569877A878B879C8788E50E9406
:10B76000B125882351F040E050E0BA0188E50E94FD
:10B77000E72569837A838B839C8389E50E94B125C1
:10B78000882351F040E050E0BA0189E50E94E725A6
:10B790006D837E838F83988785E50E946325882348
:10B7A00009F492C00E9439256B017C0120E030E051
:10B7B000A901C701B6010F943F4287FF04C0F7FA01
:10B7C000F094F7F8F094F7FAF094F7F8F094CD8A43
:10B7D000DE8AEF8AF88E198E1A8E1B8E1C8E8CE4F0
:10B7E0000E946325882309F47CC00E9439256B01DF
:10B7F0007C0120E030E0A901C701B6010F943F426F
:10B8000087FF04C0F7FAF094F7F8F094CD8EDE8E3F
:10B81000EF8EF8A262E070E082E40E94CC25F82E60
:10B8200080911812811131C021E0AE014B5E5F4F53
:10B83000BE016F5F7F4FCE0141960E944B3288233D
:10B8400021F16F2D81E00E94B05A82E50E94B1255E
:10B85000882309F453C00E94352540E050E060EA97
:10B8600071E44D875E876F87788B209118122223B1
:10B8700061F08C012F2DAE01435F5F4FBE01635E0F
:10B880007F4FCE0149960E943259809101128B154B
:10B8900021F060E08B2D0E942FD8A0960FB6F8946F
:10B8A000DEBF0FBECDBFDF91CF911F910F91FF90F3
:10B8B000EF90DF90CF90BF900895C12CD12C80E8FD
:10B8C000E82E80E4F82E2ACFE091011288E0E89F6C
:10B8D000F0011124E25BF64FC080D180E280F3805A
:10B8E00065CFE091011288E0E89FF0011124E25B4E
:10B8F000F64FC480D580E680F7807BCF90E080E073
:10B90000ACCFCF92DF92EF92FF920F931F93CF9322
:10B91000DF93CDB7DEB76C970FB6F894DEBF0FBEDE
:10B92000CDBF8CE40E946325882309F4B0C00E9437
:10B9300039256B017C0120E030E0A9010F943F42E2
:10B9400087FF04C0F7FAF094F7F8F094F7FAF09450
:10B95000F7F8F094C98EDA8EEB8EFC8E8CE0E1E97C
:10B96000F2E0DE01119601900D928A95E1F788E5EB
:10B970000E94B1258823A1F040E050E0BA0188E59B
:10B980000E94E7252091B40C3091B50C4091B60C83
:10B990005091B70C0F94DE3F69837A838B839C832D
:10B9A00089E50E94B1258823A1F040E050E0BA016A
:10B9B00089E50E94E7252091B40C3091B50C4091A7
:10B9C000B60C5091B70C0F94DE3F6D837E838F834E
:10B9D00098878AE50E94B125882351F040E050E025
:10B9E000BA018AE50E94E72569877A878B879C8759
:10B9F0001D861E861F86188A80911812811138C0F4
:10BA000020E0AE01435F5F4FBE016F5F7F4FCE010D
:10BA100049960E944B32882359F180915E09811129
:10BA20000F949B0960E080E00E94B05A898D9A8D46
:10BA3000AB8DBC8DB0588D8B9E8BAF8BB88F198A18
:10BA40001A8A1B8A1C8A1D861E861F86188A809168
:10BA50001812882369F010E000E020E0AE014B5E90
:10BA60005F4FBE016F5E7F4FCE010D960E9432592F
:10BA70006C960FB6F894DEBF0FBECDBFDF91CF91AD
:10BA80001F910F91FF90EF90DF90CF900895C12C00
:10BA9000D12C80E8E82E80E4F82E58CF2F923F92E8
:10BAA0004F925F926F927F928F929F92AF92BF92CE
:10BAB000CF92DF92EF92FF920F931F93CF93DF937A
:10BAC000CDB7DEB7E5970FB6F894DEBF0FBECDBF9A
:10BAD0008DAB20913E052CAB81E080933E0580919B
:10BAE0005C058D3409F41EC5843511F40C945B712A
:10BAF000873409F0CFC180915A0590915B058A3156
:10BB0000910509F49CC208F079C18430910508F0D0
:10BB100030C12091BE0A8230910508F4F9C121306C
:10BB200009F0FCC111E0029709F010E00E94FE2527
:10BB300019821A821B821C821D821E821F82188615
:10BB400082E50E94B125882309F4F9C10E943925B4
:10BB50006B017C0120E030E0A9010F940F398823AC
:10BB600009F4EAC04090620D5090630D6090640D3E
:10BB70007090650D8091660D9091670DA091680D94
:10BB8000B091690D8CA79DA7AEA7BFA780904B0B66
:10BB900090904C0BA0904D0BB0904E0B80914F0BA2
:10BBA0009091500BA091510BB091520B88AB99AB77
:10BBB000AAABBBABA5019401C301B2010F940F392D
:10BBC00081110DC028A939A94AA95BA96CA57DA539
:10BBD0008EA59FA50F940F39882309F4ADC0A3014A
:10BBE0009201C501B4010F94DE3F20E030E040E057
:10BBF0005FE30F94753968A779A78AA79BA72CA53F
:10BC00003DA54EA55FA568A979A98AA99BA90F940E
:10BC1000DE3F20E030E040E05FE30F9475392B0118
:10BC20003C0120E030E0A901C701B6010F940F39B3
:10BC3000881F8827881F181709F478C180E090E0D2
:10BC4000A0E8BFEB8CA79DA7AEA7BFA728A539A5E5
:10BC50004AA55BA5CA01B9010F9475394B015C0176
:10BC6000A3019201C301B2010F9475399B01AC018C
:10BC7000C501B4010F94DF3F0F948D424B015C016D
:10BC8000AC019B01C701B6010F94DE3F68AB79ABF5
:10BC90008AAB9BABA5019401C701B6010F94DF3FAE
:10BCA0009B01AC0168A979A98AA99BA90F94753950
:10BCB0006B017C0120E030E0A9010F943F4287FD39
:10BCC0003AC1C701B6010F948D426B017C01C301DB
:10BCD000B2019058A50194010F94D9402CA53DA51F
:10BCE0004EA55FA50F947539A70196010F9475397C
:10BCF00028A539A54AA55BA50F94DF3F69837A8300
:10BD00008B839C83A501940168A579A58AA59BA531
:10BD10000F94D9402CA53DA54EA55FA50F9475396C
:10BD2000A70196010F947539A30192010F94DF3F8B
:10BD30006D837E838F83988720E030E0A90169813D
:10BD40007A818B819C810F940F3981110CC120E085
:10BD500030E0A9016D817E818F8198850F940F3924
:10BD6000811101C10E94B1438FEB9FE00E94962E8A
:10BD7000D5C08C30910509F409C18531910509F4CC
:10BD8000CDC0049709F086C080E50E94B125C12C82
:10BD9000D12C7601882321F00E94C81E6B017C0102
:10BDA00083E50E94B125882361F00E94392520E0B7
:10BDB00030E04AE754E40F9475390F9452416B0117
:10BDC0007C010E94038880911A12811105C060E0F5
:10BDD00085ED9FE00E9408A30F942310C60ED71E86
:10BDE000E81EF91E0F9423106C197D098E099F0916
:10BDF00097FF94C080E00E946D4BF4CF8E31910587
:10BE000009F4C0C108F03EC08C31910509F433C17A
:10BE100008F418C114E00F94231060931212709369
:10BE2000131280931412909315128091010D8111B9
:10BE300086C18EE40E946325882321F081E090E191
:10BE40000E94BDBD87E00E943BBD81117FC10E9461
:10BE5000F251882309F47AC1115009F47EC130E00F
:10BE600020E045E258E16CE270E185E00E94063393
:10BE700061E08FE190E10E94333287E090E10E941F
:10BE8000BDBDC9CF8A35910509F4D5C230F48A9772
:10BE900009F4F2C10F94AC0B41C08B35910509F444
:10BEA000CDC28C359105B1F780915905882309F4ED
:10BEB000C9C2893099F5E9EAAE2EE2E0BE2EF2E67B
:10BEC000CF2EFDE0DF2EE12C00E010E0D5018D91BA
:10BED0005D010E94B125F82E882361F0133011F422
:10BEE000082FFE2C0E943925F6016083718382831E
:10BEF0009383EF2C1F5FF4E0CF0ED11C143031F789
:10BF0000EE2009F4F1C20E946C920E949D9206C03C
:10BF1000213021F40E94FE250E94A28CFDA9F1117E
:10BF20000C945C6A0F941F270C945C6A80E090E08C
:10BF3000A0E8BFE387CEC12CD12C7601C8CE89E41E
:10BF40000E94B125882331F00E94392569837A83C4
:10BF50008B839C838AE40E94B125882309F4ECCE6C
:10BF60000E943925E5CE412FBE016F5F7F4F8BE4E4
:10BF70009BE00F9472270F9423106093121270931A
:10BF800013128093141290931512C8CF87E00E9469
:10BF90003BBD8111C3CF70E060E080E50E94BE250B
:10BFA0008CA365E070E083E50E94BE2588A363E072
:10BFB00070E084E50E94BE258C8F40E050E060ED8B
:10BFC00070E482E50E94E72569837A838B839C83F2
:10BFD00080915F0587FD04C080916005837069F1E1
:10BFE00060E088E50E942B27182F60E089E50E9419
:10BFF0002B2700E0811102E0012B1091010D812F10
:10C000000E945B2960E085E40E942B2791E089274C
:10C01000809358029E01245E3F4FAE014F5F5F4FF9
:10C02000BE01605E7F4FCE0184960E947898109288
:10C030005802812F0E945B2971CF11E0DCCF0E9452
:10C04000803B6CCF87E00E943BBD811167CF8CE0C5
:10C05000EDE9F2E0DE01119601900D928A95E1F78B
:10C0600070E060E080E50E94BE25BE016F5F7F4FFB
:10C070000E94CC9753CF87E00E94D48B811106C0D9
:10C0800060E08FE40E942B27811148CF0E94038833
:10C09000109258026091010D8CE40E942B27E82E2B
:10C0A00080E00E945B290F9423106093121270931A
:10C0B000131280931412909315120E94A08F81E0A6
:10C0C00080937A0A0E94FC938AE50E946325F82EE9
:10C0D000882369F081E00E94D48B182F82E00E94AF
:10C0E000D48B11110C94CE7211E0811101C010E0BB
:10C0F00088E50E94632581110C947C71112311F451
:10C100000C947F71012F10E00C948C7160E070E052
:10C1100080E890E40C949571A3019201C501B401EB
:10C120000C94E27160E080EF9FE00E9408A30E94FF
:10C13000B5438EED9FE00E94962E0C94B77260E09E
:10C140008FE40E942B27882309F473CE0E94D732F4
:10C150008AEC90E10E94BDBDE1CE61E08DEB90E103
:10C160000E94333288E490E10E94BDBD61E080E12D
:10C1700098E10E94333240E070E060E089E390E1B2
:10C180000E9485490091661310916713D8012D9183
:10C190003D914D915C916091620D7091630D809124
:10C1A000640D9091650D0F94DF3FAB01BC0188E5F4
:10C1B0000E94E72569837A838B839C83F80124811D
:10C1C0003581468157816091660D7091670D809130
:10C1D000680D9091690D0F94DF3FAB01BC0189E5BB
:10C1E0000E94E7256D837E838F839887BE016B5FF6
:10C1F0007F4FCE0101960E945420882309F48ECEF1
:10C2000080E00E945B290E94A08F61E085E40E948B
:10C210002B27182F21E0482FBE016B5F7F4FCE01E7
:10C2200001960F94810C6B017C01AC019B010F9472
:10C23000D142811119C049815A816B817C818CEE78
:10C2400090E10E94CA334D815E816F81788587EECF
:10C2500090E10E94CA33B701A60182EE90E10E94EC
:10C26000CA338AE00E946E2E0E94878F11110E94AD
:10C27000AE1E0E949D9252CE8091BE0A813009F07E
:10C280004DCE89E40E94B125082FF12C882319F0A6
:10C290000E943525F82E8AE40E94B125E82E8823D5
:10C2A00041F00E943525182F011106C0153070F09D
:10C2B00006C010E0002351F0F4E0FF1528F484EFED
:10C2C00090E10E94962E2ACEE110F0CF80E1E2E6C6
:10C2D000FDE0ABE4BBE001900D928A95E1F700230D
:10C2E00019F16F2DFF0C770B880B990B0F941639F2
:10C2F00020916709309168094091690950916A0954
:10C300000F94753920915F0930916009409161095E
:10C31000509162090F94DF3F60934B0B70934C0B6D
:10C3200080934D0B90934E0BEE2019F1612F110F5E
:10C33000770B880B990B0F94163920916B0930916C
:10C340006C0940916D0950916E090F9475392091D7
:10C3500063093091640940916509509166090F9411
:10C36000DF3F60934F0B7093500B8093510B909372
:10C37000520B60E080E50E942B278823C1F1002347
:10C38000D1F0E0916613F0916713208131814281F1
:10C39000538160914B0B70914C0B80914D0B9091A0
:10C3A0004E0B0F94DE3F60934B0B70934C0B8093BE
:10C3B0004D0B90934E0BEE20D1F0E0916613F0916F
:10C3C0006713248135814681578160914F0B7091AD
:10C3D000500B8091510B9091520B0F94DE3F609364
:10C3E0004F0B7093500B8093510B9093520B40E086
:10C3F00050E0BA0186E40E94E7256B017C0120E051
:10C4000030E0A9010F943F4218168CF420E030E090
:10C4100040E752E4C701B6010F94D94069837A839B
:10C420008B839C83CE0101960E94BF8F77CD60E005
:10C4300070E0CB01F3CF1092CD0B70CD8FE08093E5
:10C44000CD0B6CCD79EAC72E72E0D72EF12CE12C02
:10C4500000E010E0D6018D916D010E94B125382ECB
:10C460008823D9F10E9439254B015C01133059F022
:10C47000F701EC54F34F20813181428153810F94B5
:10C48000DE3F4B015C01F701EE59F24F2081318113
:10C4900042815381C501B4010F94DE3F2B013C0161
:10C4A0002DEB37E346E855EB0F943F4287FD0AC07A
:10C4B0002DEB37E346E855E3C301B2010F940F3982
:10C4C00018165CF41330C1F480926E0D90926F0DCB
:10C4D000A092700DB092710D032D1F5FB4E0EB0EB2
:10C4E000F11C143009F0B6CF002309F40ECD8EE60E
:10C4F0009DE00E94C18909CDF701E752F44F5F0129
:10C50000A301920160817181828193810F94DF3F49
:10C51000D5016D937D938D939C931397812F0E94EA
:10C52000B48BDBCF80915A0590915B0589379105DB
:10C5300011F40C94A26C08F0E9C18D34910509F452
:10C54000CCC608F0EFC08A31910509F401C608F0A5
:10C5500092C08431910509F444C508F06FC081315F
:10C56000910509F403C508F042C0029708F092CC87
:10C5700080E50E94B125C12CD12C7601882321F0C1
:10C580000E94C81E6B017C0183E50E94B1258823AF
:10C5900061F00E94392520E030E04AE754E40F942E
:10C5A00075390F9452416B017C010E940388809180
:10C5B000610590916205892B09F4D3C40F94520C44
:10C5C00080915A0590915B0565E171E1892B11F429
:10C5D0006DE071E130E020E04DE151E182E00E9448
:10C5E000063340E0C701B6010E94745A97CC4297C7
:10C5F00009F050CC83E50E94B125882311F40C94F6
:10C600004C6B0F942310609312127093131280934B
:10C610001412909315120E94392520E030E04AE769
:10C6200054E40F9475390F9452416093140270933F
:10C630001502809316029093170270CC87319105F2
:10C6400009F404C570F48531910509F4FBC44697DB
:10C6500009F020CC8091371582FD60CC0E940BCD73
:10C660005DCC8831910509F409C5499709F012CCD0
:10C670000E94815C53CC8032910509F4EDC5C0F570
:10C680008D31910509F4D1C570F48B31910509F410
:10C6900072C54C9709F0FECB8091610590916205BF
:10C6A0000E94FDD13BCC8E31910509F4C5C54F9751
:10C6B00009F0F0CB0E947F976C8F7D8F8E8F9F8FBC
:10C6C000BE016F5F7F4FCE014C960E9423B7CE0113
:10C6D00001960F94A6030E94B543BE016F5F7F4F82
:10C6E00081E991E10E94634B8AE00E946E2E16CC94
:10C6F0008934910509F4DDC550F48132910509F4BE
:10C70000D4C5C09709F0C6CB0E94AD3707CC8B3497
:10C71000910509F4DEC58C34910509F0BBCB0E946C
:10C72000AF9FFCCB8C36910509F4F8CB08F083C0A1
:10C730008535910511F40C948F6B90F58235910538
:10C7400009F49AC720F58E34910509F4CAC58135DC
:10C75000910509F09FCB0E94B7DB0E9414880E94CC
:10C76000D32A0E94D62A1092660B1092650B109263
:10C77000640B68EE73E080E090E00E94782A0E94EB
:10C780003D1B60E081E492E10E9408A3C7CB8335A2
:10C79000910509F479C78435910509F42BCF7ACB3B
:10C7A0008936910509F479C688F58C35910509F427
:10C7B000DBC78836910509F06DCB8091CC0B83FDEA
:10C7C000ADCB0E94B943182F87FDA8CB83E50E940B
:10C7D000B1258823C1F00E943525212F110F330B7D
:10C7E000F901EE0FFF1FE454F64F918380834091CF
:10C7F00001124217130609F091CB0E94858761E070
:10C8000080E00F94CF2C0F940F2C88CB8A369105A3
:10C8100009F46EC68B36910509F03CCB609101128C
:10C8200080E50E94DB25823008F078CB70E060E084
:10C830000E9444E373CB8237910511F40C94556C3C
:10C84000A0F58F36910509F47BC6C8F48D369105A5
:10C8500009F4D9C58E36910509F01CCB8EE40E94EF
:10C86000B125882309F45ACB0E94351F6093F40D3B
:10C870007093F50D8093F60D9093F70D4FCB8037A5
:10C88000910509F44BCB8137910509F003CB83E582
:10C890000E94B125882309F49AC60E94451F8D3352
:10C8A00008F090C68093130239CB8637910511F4B6
:10C8B0000C94656CD0F48337910511F40C945D6C85
:10C8C0008537910509F0E6CA80916105909162056E
:10C8D000009711F40C94616CDC012C91222311F46B
:10C8E0000C94616C0F94A60319CB8737910511F452
:10C8F0000C949E6C8837910509F0CCCA81E0809336
:10C900007A0A8093790A0E94FC9308CB8139E1E08E
:10C910009E0711F40C94057008F074C1833D9105D5
:10C9200011F40C94BB6D08F0C4C0883C910511F45F
:10C930000C94AA6CD0F58C38910509F455C628F4EE
:10C940008D37910509F494CEA5CA8B39910509F468
:10C950006CC68E3B910509F09DCA8091CC0B83FD7E
:10C96000DDCA83E50E94B125182F882309F453C638
:10C970000E9435250E941A2560E081E00F94CF2C9B
:10C98000209161123091621280915F129091601239
:10C99000821793070CF446C683E292E160E00E949E
:10C9A00008A3812F0E9437D5B9CA8C3C910511F498
:10C9B0000C943E6D48F5893C910511F40C94146D6E
:10C9C0008B3C910509F066CA0E94B94387FDA6CA4F
:10C9D000B9EAEB2EB2E0FB2E10E000E0D7018D911A
:10C9E0007D010E946325882349F00E943925F801C2
:10C9F000EE5FF24F64A375A386A397A30C5F1F4F4E
:10CA00000031110559F78ACA8D3C910511F40C9437
:10CA1000B76DA5EEEA2EABE0FA2E10E08E3C910544
:10CA200009F038CA88E5810F0E946325882351F0F8
:10CA30000E943925F7016083718382839383812F5C
:10CA40000E94B48B1F5FF4E0EF0EF11C133051F71E
:10CA500080915F0587FD59CA80916005837009F058
:10CA600054CA4091E50B5091E60B6091E70B709131
:10CA7000E80B86E692E10E94CA334091E90B50919F
:10CA8000EA0B6091EB0B7091EC0B85ED9FE20E943D
:10CA9000CA334091ED0B5091EE0B6091EF0B70910A
:10CAA000F00B82ED9FE20E94CA338AE00E946E2E54
:10CAB00035CA8C3221E0920711F40C94926E08F082
:10CAC0005EC08D3D910511F40C94C36D08F04AC011
:10CAD000893D910511F40C94BF6D8C3D910509F0D1
:10CAE000D9C982E40E946325882341F080917102B4
:10CAF00090917202909319028093180282E50E942D
:10CB00006325882341F08091180290911902909337
:10CB100072028093710283E50E94B125882331F06F
:10CB20000E943525909372028093710280915D0579
:10CB300090915E05A0915F05B0916005892B8A2BCD
:10CB40008B2B09F0EBC960917102709172028DE636
:10CB500092E10E94EC3385E20E946E2E8AE00E94F0
:10CB60006E2EDCC98831B1E09B0711F40C94F66D90
:10CB70008232914009F08EC90E94F4BBCFC98F3236
:10CB8000F1E09F0711F40C94C06F78F58D32A1E0AD
:10CB90009A0711F40C94A86E8E32914009F07AC96C
:10CBA00083E50E946325182F882369F00E943525AC
:10CBB0009C01909343028093420291E0232B09F061
:10CBC00090E09093CB0B80E50E946325882311F4BD
:10CBD0000C949E6F2091420230914302232B11F05E
:10CBE0000E9425258093CB0B99C98033E1E09E07F5
:10CBF00011F40C942A6F8039914009F04BC90E94BE
:10CC000003888CC98C3022E0920711F40C94E670F2
:10CC100008F0C5C08C3AB1E09B0711F40C94267063
:10CC200008F08EC08D39F1E09F0711F40C942D713E
:10CC300058F48239A1E09A0711F40C940F708A39E4
:10CC4000914009F46BC926C9843AE1E09E0711F4CA
:10CC50000C941770853A914009F01CC96FEF7FEF73
:10CC600089E40E94CC25082F6FEF7FEF8AE40E94B1
:10CC7000CC25182F8AE50E94B125D12C811108C03E
:10CC800081E50E94B125D82E882311F40C94C67238
:10CC9000C02E81E0800F863010F00C941E70912E13
:10CCA00081E0810F863010F00C941E700E943925AF
:10CCB0002B013C01F02E07FDF12C07FF02C004E020
:10CCC000C02E812E17FD812C17FF02C014E0912E7B
:10CCD000B5E03B2ECF1408F421C9E82C3F9C50014D
:10CCE00011249E1410F40C941B700E2D10E020E003
:10CCF00030E0A901DD2069F0F501E00FF11FEE0F32
:10CD0000FF1FEE0FFF1FE959F44F2081318142814F
:10CD100053810A0D1B1D000F111F000F111F095910
:10CD2000144FC301B2010F94DF3FF8016083718398
:10CD3000828393836E2D8F2D0F94670AE394D1CF56
:10CD4000863F21E0920711F40C94D87068F4843F78
:10CD5000B1E09B0711F40C94D470853F914009F029
:10CD600099C80E94DEFEDAC8873FF1E09F0711F400
:10CD70000C94DC70883F914009F08CC881E080936E
:10CD800083090E94E08610928309882309F4C6C8AB
:10CD90000E94B54389E993E10E94962EBFC88C3664
:10CDA000A3E09A0709F4BAC808F08BC08D3BE2E013
:10CDB0009E0711F40C94117108F075C0883522E0BB
:10CDC000920711F40C94F7708B35924009F062C809
:10CDD0000E94B943082F87FDA1C885E50E946325FD
:10CDE000882369F10E9439254B015C01E02E002E59
:10CDF000000CFF0820E030E0A9010F943F4287FFBC
:10CE000004C0B7FAB094B7F8B09420E030E84BE330
:10CE100054E4C501B4010F943F42970143E0220F4F
:10CE2000331F4A95E1F7225B364F181614F40C9421
:10CE3000FB70D9018D929D92AD92BC9213978CE4B8
:10CE40000E946325882309F469C80E9439256B0173
:10CE50007C01002E000C110B20E030E0A9010F94A2
:10CE60003F4287FF04C0F7FAF094F7F8F09420E00F
:10CE700030E84BE354E4C701B6010F943F429801F8
:10CE800093E0220F331F9A95E1F7225B364F181675
:10CE900014F40C940671D9011496CD92DD92ED92A2
:10CEA000FC9217973BC88E3BB2E09B0711F40C94A1
:10CEB00015718335934011F00C944A5F0E9429B993
:10CEC0002DC8873EF3E09F0711F40C941D71C8F440
:10CED0008438A3E09A0711F40C941971803A9340B6
:10CEE00011F00C944A5F2091610530916205909198
:10CEF0003715926090933715C9010E94FDD10C94AB
:10CF00008E5F883EE3E09E0711F40C945071893ED9
:10CF1000934011F00C944A5F80912D1581110C946F
:10CF200054710E9440270E94F2D10E947F976D3376
:10CF300071058105910520F08CED93E10E94BDBD46
:10CF400088ED93E10E94BDBD84EE8093A90584EC39
:10CF500093E10E94962E80EC93E10E94BDBD0C945B
:10CF60008E5F86E291E10E94459D2ACB80915D050E
:10CF700084FD18C080915F0587FD14C08091600515
:10CF8000837081F460E089E391E10E9408A35F98D7
:10CF90008A98809108018170809306010F940C2C6F
:10CFA0000C948E5F88E50E94632581115F9889E566
:10CFB0000E94632581118A988AE50E94632588234F
:10CFC00029F08091080181708093060185E40E9418
:10CFD0006325882311F40C948E5F0F940C2C0C9411
:10CFE0008E5F8091371583FF25C081E591E10E9416
:10CFF000962E8091371583FF17C087E595E10E9433
:10D0000082CD8BE1E7E5F5E1DE01119601900D920D
:10D010008A95E1F770E060E0CE0101960E9439D375
:10D02000CE0101960E94682782E491E10E94962E2B
:10D030000C948E5F0E94B54382E691E10E94962E89
:10D040000C948E5F0E941CCD0C948E5FE091610564
:10D05000F09162058191882331F08032D9F7DF01A8
:10D0600011971C92F7CF60E0809161059091620565
:10D070000E9446D21092A9050C948E5F83E50E940F
:10D08000B125882321F00E94351F0E94C7B884E58E
:10D090000E94B1258823A9F00E94351F6B017C01F5
:10D0A0000E94B197C0920209D0920309E09204094C
:10D0B000F0920509CD28CE28CF2819F081E0809381
:10D0C0001912809118128823F9F080E090E0A0EA0C
:10D0D000B1E489839A83AB83BC831C8E1D8E1E8E24
:10D0E0001F8E18A219A21AA21BA210E000E020E0D5
:10D0F000AE014F5F5F4FBE01645E7F4FCE018096F1
:10D100000E9432590C948E5F0E94C52A882381F0B8
:10D110000E94F9C40E94029F84E39CE00E94AACC72
:10D1200010926B0E10926C0E10926D0E10926E0E8D
:10D1300061E088E398E10E94333245E258E16CE611
:10D1400071E185E00F9463020F94DE030C948E5F0F
:10D150008091371583FD02C00C948E5F83E50E9499
:10D16000B125882311F40C948E5F0E94351F0E9414
:10D17000C7B80C948E5F83E40E946325882361F115
:10D1800082E891E10E94962E80919E168823F9F004
:10D19000BE016F5F7F4F8BE996E10E943DCCCE01CF
:10D1A00001960E94EFC8CE0101960E94C8CD8091E1
:10D1B0007D12882339F080E20E946E2E8DE792E185
:10D1C0000E94EFC88AE00E946E2E0C948E5F88E762
:10D1D00091E10E94962EF6CF83E50E94B125882327
:10D1E00001F10E94451F182F8C3308F08CE38093C7
:10D1F00034050F9423106B017C01212F30E0A8EE41
:10D20000B3E00F94A73FC60ED71EE81EF91EC092CA
:10D210003005D0923105E0923205F09233050C943E
:10D220008E5F0E94B7C40C948E5F809137158E7FFD
:10D23000809337150C948E5F8091371583FD02C063
:10D240000C948E5F0F94920B809161059091620512
:10D250000E948AD10C948E5F8091371582FD0E94C6
:10D2600003888091371583FD02C00C948E5F60E0C7
:10D2700080E50E942B27182F682F809161059091DF
:10D2800062050E9446D283E50E94B125882321F0E1
:10D290000E94351F0E94C7B80E94F9C411110C9456
:10D2A0008E5F0E94029F0C948E5F0E9402B80C94C5
:10D2B0008E5F80E50E946325882311F40C948E5FB5
:10D2C0000E94451F853608F084E68093A9050C94DA
:10D2D0008E5F0E94029F0C948E5F0E94D32A0C9452
:10D2E0008E5F70E060E083E50E94CC258E3491056E
:10D2F00031F40E9424870F94DE030C948E5F8CEF30
:10D3000091E10E94962E6091690A70916A0A83EFFA
:10D3100091E10E94B83360916B0A70916C0A86EEBD
:10D3200091E10E94B8336091690A70916A0A809114
:10D330006B0A90916C0A681B790B809119128150CD
:10D3400021E030E0823010F030E020E0621B730B0F
:10D350008BED91E10E94B8338AE00E946E2E83ED3E
:10D3600091E10E94962E80916D0A90916E0AA09193
:10D370006F0AB091700A8C8F9D8FAE8FBF8FBE01E8
:10D380006F5F7F4FCE014C960E9423B7BE016F5F47
:10D390007F4F86EC91E10E94634B8091710A9091DE
:10D3A000720AA091730AB091740A8C8F9D8FAE8F10
:10D3B000BF8FBE016F5F7F4FCE014C960E9423B797
:10D3C000BE016F5F7F4F86EB91E10E94634B20E0CF
:10D3D00030E04AE754E46091750A7091760A8091D2
:10D3E000770A9091780A0F94D940AB01BC018EE97D
:10D3F00091E10E94CA338DE60E946E2E8AE00E945F
:10D400006E2E0C948E5F8091CC0B83FF02C00C9427
:10D410008E5F0E94B943182F87FF02C00C948E5F65
:10D4200083E50E94B125082F882389F10E943525C4
:10D43000212F012E000C330BF901EE0FFF1FE454D6
:10D44000F64F91838083409101124217130611F029
:10D450000C948E5F0E94858761E081E00F94CF2C51
:10D460002091CB123091CC128091C9129091CA12A6
:10D470008217930714F0011102C00F9427040F9430
:10D480000F2C602F812F0E94AFD60C948E5F82E507
:10D490000E94B1258111CACFB6C90E94B943182F85
:10D4A00087FD0AC084E092E10E94962E812F0E949F
:10D4B000C4D48AE00E946E2E2CA920933E05E596E6
:10D4C0000FB6F894DEBF0FBECDBFDF91CF911F9195
:10D4D0000F91FF90EF90DF90CF90BF90AF909F9013
:10D4E0008F907F906F905F904F903F902F90089516
:10D4F0006091011280E50E94DB25F82E81E08F15F6
:10D5000010F40C948E5F81E40E9463250FEF10E00D
:10D51000882341F0E0910112F0E0E253F44F608182
:10D52000062F10E083E50E94B125882319F00E94A0
:10D53000351F8B01B8018F2D0E9444E30C948E5F40
:10D5400083E50E946325882331F060E083E50E9433
:10D55000DB258093CC0B0E94B54385E192E10E94CC
:10D56000962E8091CC0B882351F110E000E020E052
:10D570008091CC0B90E0B0E0A0E0002E04C0B69506
:10D58000A795979587950A94D2F780FF12C0FF243C
:10D59000F394F20E222319F08CE20E946E2EF80111
:10D5A000EE0FFF1FE55FFD4E859194910E94962E30
:10D5B0002F2D0F5F1F4F05301105D1F603CE87E0E9
:10D5C00092E107CE8CE3809313020C948E5F0E944D
:10D5D000B543609113028CE192E10E94C2338AE06C
:10D5E0000E946E2E0C948E5F8091CC0B83FF02C044
:10D5F0000C948E5F83E50E94B125882311F40C946E
:10D600008E5F0E9435250E941A2561E080E00F940C
:10D61000CF2C0C948E5F82E50E94B1258111A8C9A0
:10D620000C948E5F82E392E1B9C983E50E94B12533
:10D63000882311F40C948E5F0E94451F182F8C33A1
:10D6400008F08CE3809339050F9423106B017C0163
:10D65000212F30E0A8EEB3E00F94A73FC60ED71EEF
:10D66000E81EF91EC0923505D0923605E0923705C6
:10D67000F09238050C948E5F8091CD0B8F7D806188
:10D680008093CD0B0C948E5F8091CD0B8F7E80624A
:10D690008093CD0B0C948E5F80915D0584FD0CC052
:10D6A00080915F0587FD08C080916005837021F43B
:10D6B0000E9414880C948E5F0E94038888E50E9463
:10D6C0006325882331F05F9A8091000D8E7F8093CF
:10D6D000000D89E50E946325882331F08A9A8091A4
:10D6E000000D8D7F8093000D8AE50E9463258823BD
:10D6F00059F0809108018095817080930601809196
:10D70000000D8B7F8093000D85E40E9463258823A4
:10D7100011F40C948E5F0E943A1B0C948E5F83E58B
:10D720000E946325882311F40C948E5F0F942310BC
:10D730006093121270931312809314129093151227
:10D740000E94392520E030E04AE754E40F9475390F
:10D750000F94524160933A0570933B0580933C05CA
:10D7600090933D050C948E5F0E94B94387FF02C0E1
:10D770000C948E5F80915D0584FD09C080915F05EA
:10D7800087FD05C080916005837009F489C029EA8E
:10D79000C22E22E0D22E32E0E32E3DE0F32E10E046
:10D7A000D6018D916D010E94B125882309F465C0D1
:10D7B000133009F06DC00E9439254B015C0120E057
:10D7C00030E040EA51E40F940F3987FF4EC0A501C5
:10D7D00094016091220D7091230D8091240D909100
:10D7E000250D0F94D9402B013C01AC019B016091A8
:10D7F0007F097091800980918109909182090F942D
:10D80000753960937F0970938009809381099093A3
:10D810008209A30192016091320D7091330D8091C4
:10D82000340D9091350D0F9475396093320D7093CE
:10D83000330D8093340D9093350D6091BE0570913A
:10D84000BF058091C0059091C1050F941439A301C3
:10D8500092010F9475390F9452416093BE057093F5
:10D86000BF058093C0059093C1058092220D9092D0
:10D87000230DA092240DB092250D1F5FF4E0EF0E52
:10D88000F11C143009F08CCF0E94DF870C948E5F5E
:10D890000E943925F701648B758B868B978BEDCFB2
:10D8A00081E00F94390B0C948E5F0F94B80881E9D6
:10D8B00093E10E9459E30C948E5F0E948FBC0C94FC
:10D8C0008E5F0F94DE030C948E5F009161051091C2
:10D8D000620594E0F12C40E09150F9F0F80180816C
:10D8E000282F2B7F213499F421812133B1F4813405
:10D8F00011F1853409F441E098012E5F3F4F890111
:10D900002F5F3F4FF80180818032C9F3E5CF80352A
:10D9100021F4818180538A3078F341110E94B5430C
:10D92000FF2021F080E592E10E94962EC8010E941E
:10D930002ABD0C948E5FFF24F394DECF0E94B8932F
:10D940000C948E5F10927A0A1092790A0E94FC93CE
:10D950000C948E5F0E94B943182F87FF02C00C946D
:10D960008E5FF090D80B84E40E94B125082F8823A5
:10D9700009F456C00E9439256B017C0120E030E09B
:10D98000A9010F940F39882309F44CC024E0120236
:10D99000F0011124E053F44FC082D182E282F3827D
:10D9A00020E030E0A9016091D00B7091D10B809103
:10D9B000D20B9091D30B0F940F3981110CC080E0E2
:10D9C00090E0A0EEBFE38093D00B9093D10BA09397
:10D9D000D20BB093D30B20E030E0A9016091D40BBF
:10D9E0007091D50B8091D60B9091D70B0F940F3976
:10D9F00081110CC080E090E0A0EEBFE38093D40BD7
:10DA00009093D50BA093D60BB093D70B602F83E5E3
:10DA10000E942B278093D80B0E94C0880C948E5FA5
:10DA20000F2DF4CF80E0F6CF0E94B94387FF02C0EC
:10DA30000C948E5F09EA12E082E0E82E8DE0F82E69
:10DA40009DEAC92E92E0D92ED8018D918D010E94B8
:10DA50006325882359F00E9439250F945241F7011C
:10DA600060837183828393830E949187F4E0EF0E39
:10DA7000F11CC016D10641F70C948E5F80915E05B3
:10DA800087FD2DC080915F058E7049F54091360D60
:10DA90005091370D6091380D7091390D86E592E106
:10DAA0000E94CA3340913A0D50913B0D60913C0D5C
:10DAB00070913D0D83E592E10E94CA3340913E0D85
:10DAC00050913F0D6091400D7091410D88EF9EE1A6
:10DAD0000E94CA338AE00E946E2E0C948E5F83E50A
:10DAE0000E94B125882391F00E9439256093360D5C
:10DAF0007093370D8093380D9093390D60933E0DE0
:10DB000070933F0D8093400D9093410D80E50E94EE
:10DB1000B125882351F00E9439256093360D70930A
:10DB2000370D8093380D9093390D82E50E94B12511
:10DB3000882351F00E94392560933A0D70933B0D74
:10DB400080933C0D90933D0D84E50E94B125882380
:10DB500011F40C948E5F0E94392560933E0D7093F2
:10DB60003F0D8093400D9093410D0C948E5F0E9469
:10DB700032310C948E5F0E94B6450C948E5F0E94E9
:10DB8000AB340C948E5F0E94B943082F87FF02C00C
:10DB90000C948E5F83E50E94B125882341F00E949A
:10DBA0003525BC01802F0E9413200C948E5F0E94AB
:10DBB000B543002E000C110B85E40E946E2E80E30D
:10DBC000800F0E946E2E000F111FF801E25CFD4FC6
:10DBD0006081718181E792E10E94EC3385E20E94CD
:10DBE0006E2E8AE00E946E2E0C948E5F80E50E945D
:10DBF0006325882311F40C948E5F0E9435258C01D7
:10DC0000892B09F082C083E50E946325882391F067
:10DC10000E9435258F3F980731F487E593E10E94F4
:10DC2000E22A0C948E5FBC0187E593E10E94502BA1
:10DC30000C948E5F0E94B54370E060E08CE792E147
:10DC40000E94EC338091591358E5C52E52E0D52E31
:10DC5000C81AD10887FDD394CC0CDD1CCC0CDD1C7C
:10DC60000D2C000CEE08FF088091581378E8872EE1
:10DC7000912C881A910887FD9394880C991C880C24
:10DC8000991C092C000CAA08BB088091571390E03E
:10DC90008F3FC9F1FC01EE0FFF1FE80FF91FE25F94
:10DCA000FC4E8181928133E0880F991F3A95E1F70C
:10DCB000B0E0A0E044E0B595A795979587954A9583
:10DCC000D1F702969C012F5F3F4F032E000C440BAF
:10DCD000550B281939094A095B09A4EBB0E00F94E8
:10DCE000943FA7019601281939094A095B090F9445
:10DCF000753FB90189E792E10E94EC338AE00E9406
:10DD00006E2E0C948E5F80E0DDCF0E94B143B8018F
:10DD100083E992E10E94EC3384E892E10E94962E1E
:10DD20000C948E5F64E071E083E50E94BE258C0157
:10DD300068EE73E080E50E94BE258938A3E19A076A
:10DD400010F088E893E1B8010E9476A00C948E5FF1
:10DD500060E085E40E94DB25811174C080E50E94AB
:10DD60006325882351F00E9439256093CE12709369
:10DD7000CF128093D0129093D11289E40E94632530
:10DD8000882381F00E9439252CEA35EC47E25EE3D6
:10DD90000F9475396093D2127093D3128093D4127A
:10DDA0009093D51284E40E946325882381F00E9419
:10DDB00039252CEA35EC47E25EE30F94D9406093B5
:10DDC000D6127093D7128093D8129093D9120E94D2
:10DDD000B5434091CE125091CF126091D012709104
:10DDE000D11282EA92E10E94CA332CEA35EC47E272
:10DDF0005EE36091D2127091D3128091D41290910F
:10DE0000D5120F94D940AB01BC018EE992E10E947A
:10DE1000CA332CEA35EC47E25EE36091D61270918A
:10DE2000D7128091D8129091D9120F947539AB0105
:10DE3000BC018AE992E10E94CA338AE00E946E2EF8
:10DE40000C948E5F0E94B14386EA92E10E94962E66
:10DE50000C948E5F80E50E946325882351F00E9418
:10DE600039256093641270936512809366129093C3
:10DE7000671289E40E946325882381F00E94392576
:10DE80002CEA35EC47E25EE30F9475396093681233
:10DE90007093691280936A1290936B1284E40E94CB
:10DEA0006325882381F00E9439252CEA35EC47E26E
:10DEB0005EE30F94D94060936C1270936D1280935F
:10DEC0006E1290936F120E94B5434091641250916C
:10DED0006512609166127091671280EC92E10E9467
:10DEE000CA332CEA35EC47E25EE360916812709128
:10DEF000691280916A1290916B120F94D940AB0114
:10DF0000BC018CEB92E10E94CA332CEA35EC47E26B
:10DF10005EE360916C1270916D1280916E1290911F
:10DF20006F120F947539AB01BC0188EB92E10E942E
:10DF3000CA338AE00E946E2E0C948E5F11110C94ED
:10DF40008E5F0E94B54380EE92E10E94962E8091F2
:10DF5000CB0B882391F088EC92E10E94962E609181
:10DF60004202709143028FEC92E10E94EC338BEC01
:10DF700092E10E94962E0C948E5F84EC92E1EDCF9C
:10DF800070E060E085E40E94CC25F82EBFEF8B178F
:10DF9000C9F1882341F080E093E10E94962E0F940E
:10DFA0006C020C948E5F04EB10E083E50E94B125B7
:10DFB000882319F00E9435258C0165E070E083E428
:10DFC0000E94CC25E82E60E085E50E942B27D82E04
:10DFD00060E083EF92E10E9408A3B801110F880B63
:10DFE000990B0F94163969837A838B839C832D2D2B
:10DFF0004E2D6F2DCE0101960E946CF20F94DE0320
:10E000000C948E5F06E410E0D0CF80915B0B811101
:10E010000C94855F81E00E940B940C94855F0E94B4
:10E020004B200E94AE1E0E949D920C948E5F0E9417
:10E03000A5460C948E5FF3940C946A660E94B143DB
:10E0400084E493E10E94962E0C948E5F87E00E94F8
:10E050003BBD81110C948E5F6EE9C62E69E1D62E10
:10E0600082E69DE099A788A7DE0111961D017D013A
:10E0700010E000E0C6010E944520E8A5F9A58190C6
:10E080009190A190B190F9A7E8A7A50194010F94F0
:10E09000DE3F2B013C01D7014D925D926D927C9247
:10E0A000139720E030E040EA51EC0F943F4287FDA7
:10E0B0000AC020E030E040EA51E4C301B2010F940D
:10E0C0000F3918167CF4F801EE53F64EE4911E1643
:10E0D0004CF4B7FAB094B7F8B094F701808291820B
:10E0E000A282B382D7018D909D90AD90BD907D01AD
:10E0F00020E030E040EA51ECC501B4010F943F420A
:10E1000087FD3FC020E030E040EA51E4C501B401A2
:10E110000F940F391816ACF10F5F1F4FB4E0CB0E00
:10E12000D11C0330110509F0A5CF55EEE52E5BE0BB
:10E13000F52E10E0F10181919191A191B1911F0112
:10E14000F70181939193A193B1937F01812F0E9455
:10E15000B48B1F5F133071F70E949D9260E08DE5D4
:10E1600093E10E9408A363E972E084E690E00E94D4
:10E1700076A06AEB72E084E690E00E9476A00C94B0
:10E180008E5F0E94B1438BE793E10E94962E61E07F
:10E190008DE693E10E9408A368E270E088EC90E0CD
:10E1A0000E9476A00C948E5F0E9452A30C948E5F06
:10E1B0000E9463F00C948E5F61E083E50E942B2740
:10E1C00091E089270E9470F70C948E5F809137153B
:10E1D00082FF05C08064809337150C948E5F83FDA9
:10E1E00002C00C948E5F0F94920B0C948E5F0E9471
:10E1F000585B0C948E5F80E090E8ABE3B4E4F901E7
:10E2000080839183A283B3830C941F6780E090E89E
:10E21000ABE3B4E4F90184839583A683B7830C94BC
:10E220008E5F0E9430580C948E5F0E94DF430C94E6
:10E230008E5F0E94ED440C948E5F81E08093BE0A55
:10E2400010925A1260E083E50E942B2781110C94F2
:10E250008E5F0F94F7060C948E5F83E50E94632512
:10E26000882341F00E94252580935E090E9448275B
:10E270000C948E5F0E94B5438BEA93E10E94962E28
:10E2800080915E09882349F088EA93E10E94962EE6
:10E290008AE00E946E2E0C948E5F84EA93E1F6CFA2
:10E2A0000E94A42E0C948E5F0E94F3D081110C94D6
:10E2B0008E5F0C94916710915A050F942310609310
:10E2C0001212709313128093141290931512812FCF
:10E2D000012E000C990B209101122817190651F0FC
:10E2E00060E083E50E942B27682F812F0E942FD8A2
:10E2F0000C948E5F81E0F8CF111107C011E089E521
:10E300000E946325082F811307C0012FF11204C05A
:10E3100011E001E0FF24F39482E50E94B1258823F7
:10E3200011F40C9486600E9439256CA37DA38EA302
:10E330009FA320E030E0A9010F940F39882381F0DA
:10E34000111105C0011103C0FF2009F410C160E0E4
:10E35000CE0184960E9446910E948A2C0E94542CE1
:10E36000112309F480C0002309F47AC01092620DD1
:10E370001092630D1092640D1092650D1092660D4F
:10E380001092670D1092680D1092690D0E946C92A8
:10E390008AEA99E10E9445204B015C018EEA99E1ED
:10E3A0000E9445202B013C01AC019B01C501B40139
:10E3B0000F943F42181614F00C948C60A501940140
:10E3C000C301B2010F94D9409B01AC010F94753980
:10E3D00020E030E040E85FE30F94DF3F0F948D4290
:10E3E00020E030E048E452E40F94753968A379A343
:10E3F0008AA39BA320E030E040EC5FE3C301B201BD
:10E400000F947539905869837A838B839C8320E0BD
:10E4100030E040EC5FE3C501B4010F9475399058CA
:10E420006C8F7D8F8E8F9F8FAE01405E5F4FBE01E0
:10E430006F5F7F4FCE014C960E9405910E94919490
:10E440001092620D1092630D1092640D1092650D82
:10E450001092660D1092670D1092680D1092690D62
:10E4600080E00E948495002319F081E00E94849549
:10E47000FF2009F47CC083E00E943BBD811177C07E
:10E480000E946C922091E50B3091E60B4091E70BD6
:10E490005091E80B60E070E086E193E40F94DE3F7A
:10E4A0002B013C012091E90B3091EA0B4091EB0BE1
:10E4B0005091EC0B60E070E086E193E40F94DE3F56
:10E4C0004B015C0180916A0D90916B0DA0916C0DD8
:10E4D000B0916D0D8093530B9093540BA093550BFB
:10E4E000B093560B0091661310916713D8012D91CC
:10E4F0003D914D915C91C301B2010F94DE3F609359
:10E500004B0B70934C0B80934D0B90934E0BF8017B
:10E510002481358146815781C501B4010F94DE3FC6
:10E5200060934F0B7093500B8093510B9093520B51
:10E530008BE49BE00E94F91A882311F40C949260FA
:10E540001C8E1D8E1E8E1F8E88E0EBE4FBE0DE012C
:10E55000119601900D928A95E1F7BE01645E7F4F9E
:10E56000CE0101960F94680E82E00E9484950E946D
:10E570006C928091790A80937A0A8E2D0E945B2991
:10E580000E94878F0E949D920C948E5F0E94B143DF
:10E5900084E293E10E94962E0C948E5F882309F406
:10E5A000ADCEB6CE9F92AF92BF92CF92DF92EF9256
:10E5B000FF920F931F93CF93DF9300D01F921F9270
:10E5C000CDB7DEB7E1E8FBE10027BB27462F572F89
:10E5D000A82FAA2341F4A52F542FB85FAA2319F41A
:10E5E000A52F5527B85FA03138F45295A295452F35
:10E5F0004F70507FA42BBC5FA03428F4550FAA1F86
:10E60000550FAA1FBE5FA03818F4550FAA1FB39567
:10E61000550FAA1FEA0FF01F449151E0AA27B850E6
:10E6200081F1C8F0B0FF02C0440F551FB1FF04C014
:10E63000440F551F440F551FB2FF06C05295429517
:10E64000142F1F70407F512BB3FF1BC0A52F542FD9
:10E6500044270C944173B195B0FF02C0559547957E
:10E66000B1FF04C05595479555954795B2FF05C034
:10E670005295407F4295452B5F70B3FF02C0452FF6
:10E680005527DD24CC24BB24B2E0649FD018C108F8
:10E69000B00AB00B749FC018B108B00B849FB018BB
:10E6A000B109659FC018B108B00B759FB018B109CA
:10E6B000859FB0196A9FB018B1097A9FB0194D9D16
:10E6C000A12C99243327992722275D9DA00C911C0A
:10E6D000301F901F201FAD9D900C311D901F201FDB
:10E6E0004C9DA00C911C301F901F201F5C9D900C16
:10E6F000311D901F201FAC9D300D911D201F4B9D83
:10E70000900C311D901F201F5B9D300D911D201F0F
:10E71000AB9D900D211D4B9F300D911D201F5B9FC8
:10E72000900D211DAB9F200DB1E0BB24CC24DD2436
:10E73000639FD018C108B00AB00B739FC018B1080E
:10E74000B00B839FB018B109699FC018B108B00B16
:10E75000799FB018B109899FB019629FB018B109AB
:10E76000729FB019D61AC70AB80A20F0B1E03B0F61
:10E77000901F201F1124792F632F90E0822F0F907C
:10E780000F900F900F900F90DF91CF911F910F91ED
:10E79000FF90EF90DF90CF90BF90AF909F90089543
:10E7A00080916B1390916C13891B877089F4809111
:10E7B0006F0E81110DC08091DA129091DB12892BBE
:10E7C00039F481E090917D0A911103C080E00895B1
:10E7D00081E0089590E080E00895CF93C82FCB01A9
:10E7E0000E94962E86EE98E10E94962E87ED98E183
:10E7F000CC2311F08CED98E10E94962E8AE0CF9107
:10E800000C946E2E0F931F93CF938C01C62F80EE26
:10E8100093E10E94962EC8010E94962E8AE30E94E0
:10E820006E2E80E38C0F0E946E2E8AE0CF911F9196
:10E830000F910C946E2ECF93DF9380916B13909178
:10E840006C13891B8095877019F40E946D4BF5CF6E
:10E8500080916B138F5F8770A0916B1398E6A99FCF
:10E86000D0011124FD01EE53FA4FEF0119929A9550
:10E87000E9F798E09083A952BA4F90E1E1E9F3E11A
:10E8800001900D929A95E1F720916B1390916C1382
:10E89000291303C094E69093681380936B13DF9160
:10E8A000CF910C945B2A2F923F924F925F926F927E
:10E8B0007F928F929F92AF92BF92CF92DF92EF9210
:10E8C000FF920F931F93CF93DF93CDB7DEB76C9773
:10E8D0000FB6F894DEBF0FBECDBF8C015B015A832B
:10E8E0004983FC01EE5AFF4F2081318142815381DF
:10E8F00029873A874B875C87CA01B9010F9414397D
:10E900006B017C01D5012D913D914D915C910F944E
:10E9100075390F94BD402B013C01E981FA812081BA
:10E92000318142815381C701B6010F9475390F942B
:10E93000BD404B015C01C301B2010F945241698B90
:10E940007A8B8B8B9C8B683771058105910540F420
:10E9500028E730E040E050E0298B3A8B4B8B5C8B12
:10E96000C501B4010F9452416D877E878F87988BC4
:10E97000683771058105910540F448E750E060E093
:10E9800070E04D875E876F87788BF801E25AFF4F02
:10E990004080518062807380C301B2010F941639A8
:10E9A00069837A838B839C8369897A898B899C8923
:10E9B0000F9414396D8B7E8B8F8B988F20E030E015
:10E9C000A90169817A818B819C810F940F398823F9
:10E9D00009F4E1C1A7019601C701B6010F94753989
:10E9E0004B015C012D893E894F89588DCA01B901BF
:10E9F0000F9475399B01AC01C501B4010F94DE3F42
:10EA00004B015C0129813A814B815C81CA01B901CA
:10EA10000F94DF3F9B01AC01C501B4010F94D940B5
:10EA20000F94BD400F9452416D837E838F839887EE
:10EA300066277727CB0164197509860997090F9412
:10EA400016394B015C016D857E858F8598890F9401
:10EA500014392B013C0120E030E0A901C501B401CB
:10EA60000F940F39882309F49AC1A3019201C301BD
:10EA7000B2010F947539698F7A8F8B8F9C8FA701A4
:10EA80009601C701B6010F9475399B01AC01698DE0
:10EA90007A8D8B8D9C8D0F94DE3F6B017C01A501DF
:10EAA0009401C501B4010F94DF3F9B01AC01C70184
:10EAB000B6010F94D9400F948141D80195968D905D
:10EAC0009D90AD90BC909897750164012D813E8119
:10EAD0004F815885C21AD30AE40AF50A0F945241AD
:10EAE000C61AD70AE80AF90AF7FE8EC02D893E89B0
:10EAF0004F89588DCA01B9010F9475396B017C019A
:10EB000029813A814B815C81CA01B9010F94DF3FB1
:10EB100069877A878B879C8720E030E0A90169812B
:10EB20007A818B819C810F940F39882309F43BC132
:10EB3000C501B4010F94143929853A854B855C854C
:10EB40000F947539A70196010F94DE3F6D837E8384
:10EB50008F839887A3019201C301B2010F94753985
:10EB60009B01AC016D817E818F8198850F94DF3F81
:10EB70002B013C0120E030E040E850E469817A81DB
:10EB80008B819C810F9475399B01AC01C301B2014B
:10EB90000F94D9400F94BD402B013C0120E030E0A0
:10EBA000A9010F943F4218161CF0412C512C320140
:10EBB000C301B2010F9452416D837E838F83988786
:10EBC00086169706A806B90620F48D829E82AF822B
:10EBD000B8866D817E818F8198850F94143929853F
:10EBE0003A854B855C850F947539A70196010F9482
:10EBF000DF3F0F948D420F94524169877A878B874C
:10EC00009C87C12CD12C760169857A858B859C8562
:10EC100029893A894B895C89621B730B840B950B9C
:10EC20000F94143929813A814B815C810F94D9402A
:10EC300020E034E244EF59E40F9475390F945241C7
:10EC40004B015C0169857A858B859C852D853E8588
:10EC50004F855889621B730B840B950B0F941439E5
:10EC600029813A814B815C810F94D94020E034E2C4
:10EC700044EF59E40F9475390F9452412B013C0134
:10EC80003FE683169104A104B10408F090C0F4019A
:10EC9000EE0FFF1FEE0FFF1FEB53F64E8591959180
:10ECA000A591B4918983292E3A2EBD8B4FE6441647
:10ECB00051046104710408F083C0F201EE0FFF1FDC
:10ECC000EE0FFF1FEB53F64E4591559165917491F0
:10ECD0009A01CB014D815E816F817885D8019A962A
:10ECE0004D935D936D937C939D974C0D5D1D6E1DB3
:10ECF0007F1DF80146A757A760AB71ABEA5AFF4FDB
:10ED000049895A896B897C894083518362837383E3
:10ED1000D6968D929D92AD92BC92D997F80142AE53
:10ED200053AE64AE75AEFE96498140832182328235
:10ED30005D895383349620833183828393836985ED
:10ED40007A858B859C85D2966D937D938D939C93CC
:10ED5000D59778962D853E854F85588920833183B8
:10ED6000428353836C960FB6F894DEBF0FBECDBFBF
:10ED7000DF91CF911F910F91FF90EF90DF90CF9097
:10ED8000BF90AF909F908F907F906F905F904F90CB
:10ED90003F902F90089560E070E0CB0141CE60E09D
:10EDA00070E0CB0188CE60E070E0CB01F3CEC5010E
:10EDB000B4010E94D2726983272E382E9D8B76CFA4
:10EDC000C301B2010E94D2729B0184CF2F923F9265
:10EDD0004F925F926F927F928F929F92AF92BF926B
:10EDE000CF92DF92EF92FF920F931F93CF93DF9317
:10EDF000CDB7DEB7C557D1090FB6F894DEBF0FBE49
:10EE0000CDBF3B014A0159013E2C6D96DFAECEAE1F
:10EE10006D97DC012D913D914D915C91A1962CAFA8
:10EE20003DAF4EAF5FAFA1972091160D3091170DFA
:10EE30004091180D5091190DA1966CAD7DAD8EAD20
:10EE40009FADA1970F9475390F944C42AD966CAF5E
:10EE50007DAF8EAF9FAFAD97D3012D913D914D9179
:10EE60005C91A5962CAF3DAF4EAF5FAFA5972091BB
:10EE70001A0D30911B0D40911C0D50911D0DA59642
:10EE80006CAD7DAD8EAD9FADA5970F9475390F9488
:10EE90004C42E1966CAF7DAF8EAF9FAFE197D4014E
:10EEA0002D913D914D915C91A9962CAF3DAF4EAF08
:10EEB0005FAFA99720911E0D30911F0D4091200D3D
:10EEC0005091210DA9966CAD7DAD8EAD9FADA997EA
:10EED0000F9475390F944C42E5966CAF7DAF8EAFB1
:10EEE0009FAFE597D5012D913D914D915C9167962E
:10EEF0002CAF3DAF4EAF5FAF67972091220D3091A1
:10EF0000230D4091240D5091250D67966CAD7DAD7C
:10EF10008EAD9FAD67970F9475390F944C426B96E9
:10EF20006CAF7DAF8EAF9FAF6B978091CC0B83FFA3
:10EF30001CC06B962CAD3DAD4EAD5FAD6B97209375
:10EF40009D1330939E1340939F135093A013679685
:10EF50008CAD9DADAEADBFAD679780938D13909393
:10EF60008E13A0938F13B0939013D8012C90119609
:10EF7000BC91BDAFF801F2812296FFAF2297D80174
:10EF80001396BC912896BFAF289780916B139091F0
:10EF90006C13891B8095877019F40E946D4BF5CF17
:10EFA000E0916B13E696EFAFE697F0916B13FBAF32
:10EFB0008091B9099091BA09892B11F00C94A7801E
:10EFC0008091911390919213A0919313B091941307
:10EFD000AD964CAC5DAC6EAC7FACAD97481A590A9F
:10EFE0006A0A7B0A8091951390919613A0919713CA
:10EFF000B0919813E1968CAC9DACAEACBFACE197F0
:10F00000881A990AAA0ABB0A8091991390919A13B7
:10F01000A0919B13B0919C13E5962CAD3DAD4EADE8
:10F020005FADE597281B390B4A0B5B0B2FAB38AF55
:10F0300049AF5AAF80919D1390919E13A0919F1359
:10F04000B091A0136B962CAD3DAD4EAD5FAD6B97FF
:10F05000281B390B4A0B5B0B2FA338A749A75AA7CC
:10F06000232B242B252B09F490C08091CB0B8111ED
:10F0700032C0809142029091430201972091C912BF
:10F080003091CA122817390734F56B968CAD9DADB7
:10F09000AEADBFAD6B9780939D1390939E13A093DD
:10F0A0009F13B093A01367962CAD3DAD4EAD5FADF1
:10F0B000679720938D1330938E1340938F13509343
:10F0C00090130E94B54380EA9CE10E94962E1FA2F5
:10F0D00018A619A61AA634E0339E80011124025EF8
:10F0E0001D4F6FA178A589A59AA50F941639D8014F
:10F0F0002D913D914D915C910F9475396B017C017F
:10F1000020E030E0A9010F943F4287FF04C0F7FAE6
:10F11000F094F7F8F09420E030E84BE354E4609189
:10F12000220D7091230D8091240D9091250D0F9447
:10F130007539A70196010F940F3987FF26C06B968A
:10F140002CAD3DAD4EAD5FAD6B9720939D133093CD
:10F150009E1340939F135093A01367968CAD9DAD63
:10F16000AEADBFAD679780938D1390938E13A09330
:10F170008F13B09390130E94B54381E89CE10E94E5
:10F18000962E1FA218A619A61AA6D301C201882777
:10F19000B7FD83959927AA27BB278BA7B7FE03C086
:10F1A000E82FE260EBA72FA938AD49AD5AAD57FF64
:10F1B00003C03BA534603BA78FA198A5A9A5BAA51C
:10F1C000B7FF03C09BA598609BA7A4E03A9E80016F
:10F1D0001124025E1D4F6FA178A589A59AA50F94F1
:10F1E0001639F80120813181428153810F9475399C
:10F1F0006B017C0120E030E0A9010F943F4287FFC2
:10F20000C7C1C701B60190583BAD232F30E03CA3E6
:10F210002BA35BAD48E6549F90011124D901AE5356
:10F22000BA4FBCAFABAF20E030E040E05FE30F94FB
:10F23000DF3F0F9452416FA778AB89AB9AABEBAD30
:10F24000FCAD1082EA5BFF4F2BA520838FA998AD00
:10F25000A9ADBAAD2F968CAF9DAFAEAFBFAF2F9714
:10F26000B7FF0DC0B095A095909581959F4FAF4F7A
:10F27000BF4F2F968CAF9DAFAEAFBFAF2F978BA672
:10F280009CA6ADA6BEA6B7FE0BC022273327A901B8
:10F29000281939094A095B092BA73CA74DA75EA786
:10F2A0004BAA5CAA6DAA7EAA77FE0BC08827992775
:10F2B000DC0184199509A609B7098BAB9CABADABF2
:10F2C000BEAB2BA93CA94DA95EA9ABADBCAD559673
:10F2D0002D933D934D935C9358972BA53CA54DA53D
:10F2E0005EA559962D933D934D935C935C972F9615
:10F2F0002CAD3DAD4EAD5FAD2F975D962D933D93FB
:10F300004D935C939097C301B2010F9416392091ED
:10F3100002123091031240910412509105120F9481
:10F32000753927966CAF7DAF8EAF9FAF2797698BEE
:10F330007A8B8B8B9C8BC501B4010F94163920916D
:10F3400006123091071240910812509109120F9441
:10F35000753963966CAF7DAF8EAF9FAF63976D8B42
:10F360007E8B8F8B988F6FA978AD89AD9AAD0F94F6
:10F37000163920910A1230910B1240910C125091C3
:10F380000D120F9475394B015C01898E9A8EAB8EEC
:10F39000BC8E20910E1230910F124091101250919C
:10F3A0001112C701B6010F9475396B017C01CD8E26
:10F3B000DE8EEF8EF8A22BA93CA94DA95EA92630BE
:10F3C0003105410551050CF0E6C08BA59CA5ADA506
:10F3D000BEA50697A105B1050CF0DDC02F962CAD9A
:10F3E0003DAD4EAD5FAD2F9726303105410551053E
:10F3F0000CF0D1C020E030E0A901C701B6010F94A4
:10F400003F4287FF04C0F7FAF094F7F8F09488E6DB
:10F410004BA15CA1849F8001859F100D11240E5388
:10F420001A4F20E030E0A901C701B6010F94DF3F79
:10F43000D8011D966D937D938D939C93509788E68C
:10F44000ABA1BCA18A9FF0018B9FF00D1124EE535C
:10F45000FA4F2FA538A949A95AA921A332A343A33A
:10F4600054A32F968CAD9DADAEADBFAD2F972BA500
:10F470003CA54DA55EA582179307A407B50710F418
:10F48000DA01C9012BA93CA94DA95EA982179307EE
:10F49000A407B50710F4DA01C9012FA538A949A9B5
:10F4A0005AA982179307A407B50710F4DA01C90116
:10F4B00028E64BA15CA1249FF001259FF00D1124AB
:10F4C000EE53FA4F85A396A3A7A3B0A70697A1056D
:10F4D000B10508F41FC6DF01AE59BF4F8091CE0BB6
:10F4E0008C9311968091CF0B8C9331A6452846289A
:10F4F000472809F05F9888E6ABA1BCA18A9FF0017C
:10F500008B9FF00D1124EE53FA4F818D928DA38DB8
:10F51000B48D892B8A2B8B2B09F08A9888E62BA136
:10F520003CA1829FF001839FF00D1124EE53FA4F0E
:10F53000858D968DA78DB0A1892B8A2B8B2B29F0D9
:10F54000809108018170809306018FA598A9A9A9CF
:10F55000BAA9892B8A2B8B2B09F4FBC5809136091C
:10F56000882319F0815080933609809137098823C8
:10F5700019F0815080933709311068C0129880E1EA
:10F58000809336098091370981116CC0479A6AC00F
:10F59000C701B60139CE6D96EEADFFAD6D97C08057
:10F5A000D180E280F38020E030E0A901C701B601FC
:10F5B0000F940F39882379F088E62BA13CA1829F14
:10F5C000F001839FF00D1124EE53FA4FC586D686C5
:10F5D000E786F08A34CF27962CAD3DAD4EAD5FADBA
:10F5E0002797CA01B9010F9475396B017C016396A5
:10F5F0002CAD3DAD4EAD5FAD6397CA01B9010F941F
:10F6000075399B01AC01C701B6010F94DF3F6B0157
:10F610007C01A5019401C501B4010F9475399B01CA
:10F62000AC01C701B6010F94DF3F0F948D4228E66D
:10F630004BA15CA1249FF001259FF00D1124EE53F6
:10F64000FA4F658776878787908BF9CE8091360948
:10F65000811101C0129A91E0391294CF479880E14C
:10F6600080933709E090420DF090430D0091440DD6
:10F670001091450D76C52FA538A949A95AA9232B64
:10F68000242B252B09F406C12091360D3091370D1E
:10F690004091380D5091390D21966CAD7DAD8EADF8
:10F6A0009FAD21970F9475390F94BD400F9452412F
:10F6B0002B013C018FA598A9A9A9BAA9892B8A2B4E
:10F6C0008B2B09F4F0C0E091011294E0E99FF00166
:10F6D0001124EA51F64F20813181428153812FA7B5
:10F6E00038AB49AB5AAB20E030E0A9016FA578A94F
:10F6F00089A99AA90F940F39882309F4D4C08FA13E
:10F7000098A5A9A5BAA5181619061A061B060CF085
:10F71000CAC088E6ABA1BCA18A9F80018B9F100D57
:10F7200011240E531A4F1801B7E42B0E311C81E03F
:10F73000F1018083209181133091821340918313D2
:10F7400050918413A1966CAD7DAD8EAD9FADA19708
:10F750000F94DE3F6FA378A789A79AA720918513FE
:10F76000309186134091871350918813A5966CAD04
:10F770007DAD8EAD9FADA5970F94DE3F4B015C0133
:10F780002091891330918A1340918B1350918C13DF
:10F79000A9966CAD7DAD8EAD9FADA9970F94DE3F60
:10F7A0006B017C012FA138A549A55AA5CA01B90151
:10F7B0000F9475396FA378A789A79AA7A50194011B
:10F7C000C501B4010F9475399B01AC016FA178A5F7
:10F7D00089A59AA50F94DF3F4B015C01A701960113
:10F7E000C701B6010F9475399B01AC01C501B40185
:10F7F0000F94DF3F0F948D426B017C0120918D139C
:10F8000030918E1340918F135091901367966CAD89
:10F810007DAD8EAD9FAD67970F94DE3FA70196013A
:10F820000F94D9406B017C01F801E25BFF4FC0826D
:10F83000D182E282F38220E030E040E450E40F9491
:10F840003F4218160CF4FDC0A70196016FA578A9D8
:10F8500089A99AA90F9475399B01AC0160917F0920
:10F860007091800980918109909182090F94D9400B
:10F8700021962CAD3DAD4EAD5FAD21970F947539FE
:10F880000F9452416415750586059705B8F42B0150
:10F890003C0114C020913E0D30913F0D4091400D30
:10F8A0005091410DF9CE88E62BA13CA1829FF00139
:10F8B000839FF00D1124E75FF94F10828091320988
:10F8C00090913309A0913409B0913509EBADFCADAD
:10F8D000C18CD28CE38CF48C258D368D478D50A154
:10F8E0002FA338A749A75AA721A132A143A154A108
:10F8F0002FA738AB49AB5AAB2BA53CA54DA55EA5B0
:10F9000082179307A407B50708F49EC08BA99CA98A
:10F91000ADA9BEA9892B8A2B8B2BE1F06091B20592
:10F920007091B3058091B4059091B5056415750586
:10F930008605970578F40F94433F2BA93CA94DA960
:10F940005EA90F94533F241535054605570510F45D
:10F9500029013A01C114D104E104F104F1F06091EC
:10F96000B6057091B7058091B8059091B9056415F9
:10F9700075058605970588F42BA53CA54DA55EA5C4
:10F980000F94433FA70196010F94533F241535056B
:10F990004605570510F429013A012FA138A549A5BC
:10F9A0005AA5232B242B252B01F16091BA057091C8
:10F9B000BB058091BC059091BD0564157505860554
:10F9C000970598F42BA53CA54DA55EA50F94433F44
:10F9D0002FA138A549A55AA50F94533F24153505E5
:10F9E0004605570510F429013A018FA598A9A9A940
:10F9F000BAA9892B8A2B8B2B09F400C66091BE050E
:10FA00007091BF058091C0059091C1056415750581
:10FA10008605970508F0F2C52BA53CA54DA55EA56A
:10FA20000F94433F2FA538A949A95AA90F94533FD2
:10FA3000241535054605570508F0E0C529013A01AA
:10FA4000DDC5D1011C923ACF2BA93CA94DA95EA9D5
:10FA5000232B242B252BB9F16091B2057091B305AE
:10FA60008091B4059091B5056415750586059705D7
:10FA700050F50F9414392FA938AD49AD5AAD0F94F4
:10FA800075394B015C016BA97CA98DA99EA90F94C6
:10FA900014399B01AC01C501B4010F94D9404B014D
:10FAA0005C01C301B2010F9414399B01AC01C50183
:10FAB000B4010F940F3987FF06C0C501B4010F943C
:10FAC00052412B013C01C114D104E104F104A9F11C
:10FAD0006091B6057091B7058091B8059091B90510
:10FAE000641575058605970540F50F9414392FA9FF
:10FAF00038AD49AD5AAD0F9475394B015C01C70162
:10FB0000B6010F9414399B01AC01C501B4010F94E7
:10FB1000D9406B017C01C301B2010F9414399B01E0
:10FB2000AC01C701B6010F940F3987FF06C0C701AA
:10FB3000B6010F9452412B013C018FA198A5A9A5B4
:10FB4000BAA5892B8A2B8B2BB9F16091BA057091DC
:10FB5000BB058091BC059091BD05641575058605B2
:10FB6000970550F50F9414392FA938AD49AD5AAD0A
:10FB70000F9475396B017C016FA178A589A59AA5B1
:10FB80000F9414399B01AC01C701B6010F94D94001
:10FB90006B017C01C301B2010F9414399B01AC01CC
:10FBA000C701B6010F940F3987FF06C0C701B60120
:10FBB0000F9452412B013C012FA538A949A95AA9FC
:10FBC000232B242B252B09F419C56091BE057091B8
:10FBD000BF058091C0059091C10564157505860526
:10FBE000970508F00BC50F9414392FA938AD49AD0E
:10FBF0005AAD0F9475396B017C016FA578A989A95D
:10FC00009AA90F9414399B01AC01C701B6010F9456
:10FC1000D9406B017C01C301B2010F9414399B01DF
:10FC2000AC01C701B6010F940F3987FFE7C4C701C4
:10FC3000B6010F9452412B013C01E0C4A50194018F
:10FC4000C301B2010F94D9409B01AC016FA17BA508
:10FC50008FA59FA90F9475396FA37BA78FA79FAB23
:10FC600021E02BABB8C580E090E0A0E8BFE3279689
:10FC70008CAF9DAFAEAFBFAF2797E5C5F7FAF09455
:10FC8000F7F8F094A7019601C501B4010F943F4223
:10FC900018160CF03AC67501640137C6C701B601E3
:10FCA0000F940F3987FD09C020E030E0A901C5019C
:10FCB000B4010F943F4218162CF4A5019401C7011A
:10FCC000B6011FC6B7FAB094B7F8B094A501940175
:10FCD000C701B6010F940F3987FF17C6DCCF2FA0DD
:10FCE0003BA40FA51FA970C681E0C6C6CBA0DCA0AF
:10FCF00091C78BE0C82E87EDD82E83E2E82E8BE3E8
:10FD0000F82EC8C78B2D902FAA2DB32DF601858311
:10FD10009683A783B0870C94A186DCA2CBA20C9417
:10FD2000A18610916A13D12CC12C08E680916B1327
:10FD3000811709F48BC0812E912C089DC001099D6B
:10FD4000900D11249C012E533A4F1901D9018C9129
:10FD5000560183FD6FC05901C114D10409F46AC072
:10FD6000C6010E9499E3811165C0F601808181FD81
:10FD70004CC0D10115964D905D906D907C90189778
:10FD8000D60115962D913D914D915C9118972BA31D
:10FD90003CA34DA35EA3A30192016BA17CA18DA105
:10FDA0009EA10F940F3987FF30C0F60161897289D7
:10FDB0008389948990589B01AC010F94DF3FD60151
:10FDC0001D962D913D914D915C9150970F947539F1
:10FDD0009B01AC016BA17CA18DA19EA10F94DE3F84
:10FDE0006B017C01A30192010F940F3987FF0DC0B5
:10FDF000F101808181608083C5010E9499E388239D
:10FE0000E9F0D1018C918E7F8C93089DF001099DC2
:10FE1000F00D1124EE53FA4F218532854385548528
:10FE200065817681878190850F940F39811102C099
:10FE300010936A131F5F1770650178CFF101C582B7
:10FE4000D682E782F08610936A13DFCFD0906C13CE
:10FE500080906B1328E6D81409F4C7C08FEF880D83
:10FE60008770289FF0011124EE53FA4F908193FD83
:10FE7000BAC0312C212C1BA21BAE10E000E0F12CEB
:10FE8000E12CD81409F4C0C0F8E6DF9E80011124EB
:10FE90000E531A4FD8018C9183FDA9C015966D9110
:10FEA0007D918D919C9118970F948D42B62EC72EFF
:10FEB000A82E992EE114F10409F493C0F701808172
:10FEC00080FD04C0D8018C9180FF8BC0F701808138
:10FED00081608083C7010E9499E381117EC0D701B0
:10FEE00011966D917D918D919C9114970F948D42F7
:10FEF0006FA378A789A79AA79B01AC0160E070E087
:10FF000080E89FE30F94D9402B013C01AC019B0199
:10FF10006B2D7C2D8A2D992D0F94753969837A83E9
:10FF20008B839C83232D322D4BA15BADC301B2018A
:10FF30000F947539698B7A8B8B8B9C8BAE014F5FDD
:10FF40005F4FBE016F5E7F4FC7010E945374F70180
:10FF5000E95BFF4F8081882309F43FC0E0910112E3
:10FF6000B4E0EB9FF0011124EA51F64FD701A25BF8
:10FF7000BF4F2D913D914D915C9160817181828146
:10FF800093810F9475392091220D3091230D40916A
:10FF9000240D5091250D0F9475392B013C01AC01B6
:10FFA0009B016FA178A589A59AA50F9475390F9427
:10FFB0005241F701E65BFF4F71836083A301920119
:10FFC0006B2D7C2D8A2D992D0F9475390F945241EC
:10FFD000F701E45BFF4F71836083F70180818E7FBF
:10FFE0008083780108C0882E36CF8D2C42CFB32C69
:10FFF000C22CABA09BACD394FD2DF770DF2E3B2C15
:020000021000EC
:100000002C2CABA29BAE3DCF0115110509F482C08B
:10001000D8018C9181608C93C7010E9499E3811172
:1000200075C0F80161817281838194810F948D4242
:100030006B017C01AC019B0160E070E080E89FE314
:100040000F94D9404B015C012DEC3CEC4CE45DE39A
:100050000F94753969837A838B839C83A5019401FE
:10006000632D722D8BA19BAD0F947539698B7A8BA3
:100070008B8B9C8BAE014F5F5F4FBE016F5E7F4FDE
:10008000C8010E945374F801E95BFF4F8081882307
:10009000E9F1E091011224E0E29FF0011124EA511C
:1000A000F64FD801A25BBF4F2D913D914D915C91D0
:1000B00060817181828193810F9475392091220D25
:1000C0003091230D4091240D5091250D0F947539D9
:1000D0004B015C01AC019B01C701B6010F9475395E
:1000E0000F945241F801E65BFF4F718360832DEC62
:1000F0003CEC4CE45DE3C501B4010F9475390F94F9
:100100005241F801E45BFF4F71836083D8018C9109
:100110008E7F8C930E945B2A81E0CB58DF4F0FB615
:10012000F894DEBF0FBECDBFDF91CF911F910F912D
:10013000FF90EF90DF90CF90BF90AF909F908F9007
:100140007F906F905F904F903F902F90089580E048
:10015000E4CFE090460DF090470D0091480D1091CE
:10016000490D9701A801622D7DAD22968FAD229792
:1001700028969FAD28970F940F3987FD08C0E22C71
:10018000FDAC22960FAD229728961FAD289788E6E2
:10019000ABA1BCA18A9FF0018B9FF00D1124EE53FF
:1001A000FA4F85849684A784B088A501940160E005
:1001B00070E080E89FE30F94D94021966CAF7DAF4B
:1001C0008EAF9FAF21979701A8010F9475396B01EE
:1001D0007C0180916B1390916913891B8770229623
:1001E0008FAF2297A701960160E074E284E799E45B
:1001F0000F94D9400F944C422B013C0122968FADB5
:10020000229782508230A0F56091120D7091130DEB
:100210008091140D9091150D64197509860997093F
:1002200016161706180619061CF5660F771F881F85
:10023000991F2296BFAD22972B2F30E050E040E06F
:100240000F94753FCA01B9010F9416390F944B41B1
:10025000640D751D861D971D0F9416399B01AC0109
:1002600060E074E284E799E40F94D9406B017C016B
:10027000A7019601C501B4010F9475399B01AC012A
:100280000F9475392B966CAF7DAF8EAF9FAF2B97C8
:1002900088E6EBA1FCA18E9F80018F9F100D112499
:1002A0000E531A4F2B962CAD3DAD4EAD5FAD2B9737
:1002B000D80111962D933D934D935C931497959689
:1002C0002D913D914D915C9198972BA73CA74DA7FF
:1002D0005EA7CA01B9010F9414396FAB78AF89AF2B
:1002E0009AAF9B01AC01C701B6010F9475390F9409
:1002F000BD400F94524127966CAF7DAF8EAF9FAF3C
:100300002797F801EE5AFF4F6083718382839383AE
:10031000FE017196FCABEBAB9E012F5F3F4F2D961C
:100320003FAF2EAF2D9746E25DE061965FAF4EAFD7
:100330006197CE014D969AA389A36D963FAF2EAFDC
:100340006D9700E010E020E8222E3FE3332EABA9AA
:10035000BCA92D913D914D915D91BCABABABC7015B
:10036000B6010F9475394B015C016D96EEADFFAD92
:100370006D9781929192A192B1926D96FFAFEEAF7F
:100380006D9720E030E0A9010F943F4287FF04C041
:10039000B7FAB094B7F8B0946196AEADBFAD6197BF
:1003A0004D905D906D907D906196BFAFAEAF6197BF
:1003B000A5019401C301B2010F940F3987FF10C04A
:1003C000A5019401C301B2010F94D9405B014C0116
:1003D0009801A1010F940F3987FF02C08501140114
:1003E000E9A1FAA12BA93CA9E217F30709F0AFCFC5
:1003F0002D8D3E8D4F8D58A1C701B6010F947539D3
:100400006B017C01CD86DE86EF86F88A20E030E045
:10041000A9010F943F424601570187FF04C0B7FA74
:10042000B094B7F8B0944090320D5090330D609076
:10043000340D7090350DA5019401C301B2010F94E4
:100440000F3987FF10C0A5019401C301B2010F94B9
:10045000D9405B014C019801A1010F940F3987FF2E
:1004600002C08501140120E030E040E85FE3B801FC
:10047000C1010F940F3987FF66C09801A1016981FE
:100480007A818B819C810F94753969837A838B8300
:100490009C839801A1016D817E818F8198850F9445
:1004A00075396D837E838F8398879801A101698553
:1004B0007A858B859C850F94753969877A878B87B8
:1004C0009C879801A101C701B6010F9475396D870A
:1004D0007E878F87988B28E64BA15CA1249FC00163
:1004E000259F900D1124DC01AE53BA4F7D016D01A3
:1004F000B2E5CB0ED11C27966CAD7DAD8EAD9FAD18
:1005000027970F9414399801A1010F9475390F940E
:100510005241F60160837183828393839801A10124
:10052000B801C1010F9475392B962CAD3DAD4EAD80
:100530005FAD2B970F947539D70111966D937D930D
:100540008D939C9314972FA938AD49AD5AAD219640
:100550006CAD7DAD8EAD9FAD21970F947539219611
:100560006CAF7DAF8EAF9FAF219788E6EBA1FCA16A
:100570008E9F80018F9F100D11240E531A4FD801AA
:1005800055962D913D914D915C9158972BAB3CAB7D
:100590004DAB5EAB232B242B252B09F06CC8599651
:1005A0008D919D910D90BC91A02D892B8A2B8B2B29
:1005B00009F061C8F801858D968DA78DB0A1892BB2
:1005C0008A2B8B2B09F057C820913A0D30913B0DA7
:1005D00040913C0D50913D0D21966CAD7DAD8EADA1
:1005E0009FAD21970F9475390F94BD400F945241E0
:1005F0002B013C01F801E95BFF4F108288E64BA11B
:100600005CA1849F8001859F100D11240E531A4F09
:10061000F801E25AFF4F4082518262827382C30125
:10062000B2010F94143921962CAD3DAD4EAD5FADA6
:1006300021970F94D94021966CAF7DAF8EAF9FAFBD
:100640002197D80151966D937D938D939C935497E8
:10065000F801E95BFF4F80818823C1F17801B8E49C
:10066000EB0EF11CA0910112E4E0AE9FD001112429
:10067000AA51B64FF801E25BFF4F208131814281E0
:1006800053816D917D918D919C910F947539219637
:100690002CAD3DAD4EAD5FAD21970F9475392091D6
:1006A000220D3091230D4091240D5091250D0F9472
:1006B00075399B01AC0160E074E284EF99E40F941A
:1006C000D9400F945241D7016D937C9388E62BA1BA
:1006D0003CA1829FF001839FF00D1124EE53FA4F4D
:1006E00081819281A381B4812B968CAF9DAFAEAFF7
:1006F000BFAF2B97BC01CD010F948D426B017C01E4
:10070000A3E7B9E06196BFAFAEAF61972D960EAD8E
:100710001FAD2D97005F1F4F2596BFAFAEAF25973A
:100720002D962EAC3FAC2D976FA3DBA68FA7FFAA0B
:100730001BAAD1018D909D90AD90BD901D0120E030
:1007400030E0A901C501B4010F943F4287FF04C006
:10075000B7FAB094B7F8B0942596EEADFFAD2597F3
:1007600061917191819191912596FFAFEEAF25979F
:1007700020E030E0A9010F94DF3F2B013C01A501EF
:1007800094010F940F3987FF26C0FBA9FF2309F4BA
:1007900055CAA3019201B601C7010F9475392B0107
:1007A0003C012FA13BA54FA55FA9C501B4010F9442
:1007B00075399B01AC01C301B2010F940F3987FF5A
:1007C0000AC0A5019401C301B2010F94D9406FA3DF
:1007D0007BA78FA79FAB0215130509F0AACF22961E
:1007E0003FAD2297332309F47ACA80906D1390901D
:1007F0006E13A0906F13B09070132DEB37E346E8A3
:1008000055E3C501B4010F940F3987FD68CAC501CE
:10081000B4010F948D421B018C019B01AC01B60108
:10082000C7010F940F3987FF1ECA9101A801B601B5
:10083000C7010F94D94027966CAF7DAF8EAF9FAFA5
:10084000279716018701A1E7B3E12396BFAFAEAFAB
:100850002397412C512C90E8692E9FE3792E1BAAF7
:100860002396EEADFFAD23976191719181919191A6
:100870002396FFAFEEAF239727962CAD3DAD4EAD3F
:100880005FAD27970F9475394B015C012D96AEAD86
:10089000BFAD2D97CD90DD90ED90FD902D96BFAF23
:1008A000AEAF2D97BBA9BB2371F0A30192010F94AA
:1008B00075394B015C01A3019201C701B6010F9488
:1008C00075396B017C01A5019401C701B6010F9434
:1008D0000F3920E030E0A90187FFE0C9C701B60168
:1008E0000F943F4218164CF020E030E0A901C501FA
:1008F000B4010F940F3987FFC1C9A7019601C50143
:10090000B4010F94DE3F6B017C016196EEADFFAD4B
:10091000619761917191819191916196FFAFEEAF75
:10092000619720E030E0A9010F94DF3F4B015C01AB
:10093000A70196010F940F3987FF11C0A7019601F7
:10094000C501B4010F94D9409B01AC01C301B201B0
:100950000F9475392B013C01FBA9FF5FFBAB21E82C
:1009600033E123964EAD5FAD23972417350709F089
:1009700077CF5BA9552341F0A3019201B101C801D2
:100980000F9475391B018C0124EA30E74DE75FE3D2
:10099000B101C8010F9475396B017C0120912E09BA
:1009A00030912F0940913009509131090F940F393E
:1009B00087FF0AC02FA13BA54FA55FA9C701B601BC
:1009C0000F940F3987FD8BC98FA19BA5AFA5BFA938
:1009D00080932E0990932F09A0933009B093310989
:1009E00028E6ABA1BCA12A9FC0012B9F900D11242A
:1009F000FC01EE53FA4F7F019101A801B101C8013A
:100A00000F947539D70119966D937D938D939C93AF
:100A10001C9721966CAD7DAD8EAD9FAD2197905802
:100A20009B01AC010F94DF3FEBADFCAD2585368516
:100A3000478550890F9475399B01AC016BE077EDC8
:100A400083E29BE30F94DE3F9B01AC018BE097EDCB
:100A5000A3E2BBE3F70185839683A783B087108168
:100A60002B966CAD7DAD8EAD9FAD2B970F940F394E
:100A700018160CF439C983E0182B28E64BA15CA1A9
:100A8000249FC001259F900D11248E539A4FDC01A5
:100A90001C9320E1FE013196A1E7B3E101900D9294
:100AA0002A95E1F72B962CAD3DAD4EAD5FAD2B9762
:100AB00020936D1330936E1340936F135093701304
:100AC000AD962CAD3DAD4EAD5FADAD97209391137E
:100AD000309392134093931350939413E1962CAD5B
:100AE0003DAD4EAD5FADE1972093951330939613D6
:100AF0004093971350939813E5962CAD3DAD4EADB2
:100B00005FADE5972093991330939A1340939B130D
:100B100050939C136B962CAD3DAD4EAD5FAD6B9776
:100B200020939D1330939E1340939F135093A013D3
:100B3000A1962CAD3DAD4EAD5FADA1972093811335
:100B4000309382134093831350938413A5962CAD56
:100B50003DAD4EAD5FADA5972093851330938613C1
:100B60004093871350938813A9962CAD3DAD4EAD9D
:100B70005FADA9972093891330938A1340938B1309
:100B800050938C1367962CAD3DAD4EAD5FAD67971E
:100B900020938D1330938E1340938F1350939013A3
:100BA0008C599F4FE0912D0934E0E39FF00111240F
:100BB000E55AF14F4081518162817381DC014D938F
:100BC0005D936D937C93139790916B1380916C134D
:100BD000981303C084E680936813E6968FADE6977A
:100BE0008F5F877080936B1380916B1390916A1362
:100BF00081508770891709F429C910916B132090CF
:100C00006A1380916B13281609F48BC81150177062
:100C1000D12CC12C121509F484C8812E912CB8E670
:100C2000B89DF001B99DF00D1124EE53FA4F80816B
:100C300083FD73C8FCA3EBA3B1840285A384348431
:100C40004580568067807084A30192016B2D702FC0
:100C50008A2D932D0F940F39811108C0C114D1042E
:100C600009F46FC0D6018C9180FF6BC0B8E6B89DC7
:100C7000F001B99DF00D1124EE53FA4F808181FDF2
:100C80003DC0C114D10409F434C8F601C580D68032
:100C9000E780F08428E6289DF001299DF00D1124BD
:100CA000EE53FA4F618972898389948990589B0128
:100CB000AC010F94DF3FABA1BCA11D962D913D91DE
:100CC0004D915C9150970F9475399B01AC01C70110
:100CD000B6010F94DE3FD62EC72E8BAF9FA3262FD3
:100CE000372FAC016B2D702F8A2D932D0F940F3958
:100CF00087FD04C0BD2C0C2DABAC3FA02B2D302F9D
:100D00004A2D532DC301B2010F940F398823C9F026
:100D1000B8E6B89DC001B99D900D1124FC01EE53B9
:100D2000FA4F6F018081816080838BA19CA10E941A
:100D300099E3882311F40C94827ED6018C918E7FE6
:100D40008C9311501770822D20906A13281611F47D
:100D50000C94767E181711F40C94917E8F5F877037
:100D6000F3CFCF93C091A905CF7739F50E94C52A5B
:100D7000882319F180912F1590913015A09131158C
:100D8000B09132150097A105B105B9F0BC01CD01B4
:100D90006D597F4F8F4F9F4F24E630E040E050E089
:100DA0000F94533F60913315709134158091351530
:100DB000909136150F94533FC22F8C2FCF910895E9
:100DC00084E690E090934D0980934C091092850938
:100DD000109284090C94F7FA0F93AB0100918309E8
:100DE00021E0022724E839E0BC018CE499E00E946C
:100DF000F12A0F910895CF93DF9300D01F92CDB7C2
:100E0000DEB78091680A8823C1F083E390E09C8379
:100E10008B831A8219829E012F5F3F4F40E150E081
:100E200069E67AE0CE0103960E94154987EE9CE1BF
:100E30000E94962E8AE00E946E2E0F900F900F90C7
:100E40000F90DF91CF910895CF93DF9300D01F9241
:100E50001F92CDB7DEB781E08093680A80E1E9E6B2
:100E6000FAE0DF011D928A95E9F70E94FB8686E190
:100E70008D8382E390E09C838B831A8219829E018A
:100E80002F5F3F4F41E050E0BE016B5F7F4FCE01CF
:100E900003960E9415490F900F900F900F900F909E
:100EA000DF91CF910895CF92DF92EF92FF92CF938F
:100EB000DF93EC0108960E9486216B017C0120E003
:100EC00030E0A9010F940F3920E030E0A901882318
:100ED00059F0CE010E946E279B01AC01C701B601FB
:100EE0000F9475399B01AC01688579858A859B854E
:100EF0000F94DE3F688779878A879B87DF91CF9140
:100F0000FF90EF90DF90CF9008958C3221E0920710
:100F100014F08CE291E09093CC128093CB120D945C
:100F20002F10AF92BF92CF92DF92EF92FF920F936A
:100F30001F93CF93DF93C2E0DDE002EB15E082E187
:100F4000A82E8DE0B82EC12CD12C7601C3946991C6
:100F50007991899199910F941439288939894A890D
:100F60005B890F9475390F945241F8016193719325
:100F7000819391938F01C616D706E806F90610F4FF
:100F80006B017C01AC16BD0611F76FEF7FEFCB0153
:100F9000A70196010F94533F2093320930933309F0
:100FA0004093340950933509DF91CF911F910F91F0
:100FB000FF90EF90DF90CF90BF90AF9008950F9388
:100FC0001F93CF93DF9306E11DE0C2E0D2E1F80169
:100FD00021913191419151918F0160E070E080E861
:100FE0009FE30F94D9406993799389939993F2E1A0
:100FF000C231DF0761F70F94DA07DF91CF911F91BC
:101000000F910C94918790916B1380916C139813AE
:1010100006C08091B9099091BA09892B21F080E02E
:101020000E946D4BF0CF089590916B1380916C13DB
:10103000981308C08091B9099091BA09892B11F4CD
:101040000C94AC2A80E00E946D4BEECFCF92DF92E1
:10105000EF92FF92CF93DF932091010D222329F18C
:10106000EC0108960E9486216B017C0120E030E0B3
:10107000A9010F940F3920E030E0A901882359F02D
:10108000CE010E946E279B01AC01C701B6010F94EF
:1010900075399B01AC01688579858A859B850F949C
:1010A000DF3F688779878A879B87DF91CF91FF90A1
:1010B000EF90DF90CF900895AF92BF92CF92DF92E2
:1010C000EF920F931F93CF93DF93CDB7DEB7649763
:1010D0000FB6F894DEBF0FBECDBFA98ABA8ACB8AFD
:1010E000DC8AFC0180819181A281B38189839A830A
:1010F000AB83BC83FB0180819181A281B3818D830D
:101100009E83AF83B887FA0180819181A281B381E8
:1011100089879A87AB87BC87F90180819181A281F9
:10112000B3818D879E87AF87B88BCE0101960E94D1
:1011300026888091B9099091BA09892BF9F4CE01DA
:1011400041966C019E01235F3F4FAE01475F5F4FA9
:10115000BE016B5F7F4F40970E94E67664960FB6A4
:10116000F894DEBF0FBECDBFDF91CF911F910F91DD
:10117000EF90DF90CF90BF90AF90089580E0EECFDA
:101180007F928F929F92AF92BF92CF92DF92EF9217
:10119000FF920F931F93CF93DF937090D80BCAEAFF
:1011A000D5E09EE3C92E92E0D92E2EE1E22E22E078
:1011B000F22E00ED1BE0772009F45EC0F80180807C
:1011C0009180A280B38020E030E0A901C501B40184
:1011D0000F940F39882309F44FC020E030E040E03D
:1011E0005FE3C501B4010F9475399B01AC010F9405
:1011F00075392BED3FE049E450E40F9475399B01BC
:10120000AC0160E070E080E89FE30F94D9404B01AF
:101210005C0189929992A992B992F60161917191BA
:101220006F01072E000C880B990B0F9416392AE0DA
:1012300037ED43E25CE30F947539A50194010F94F7
:101240007539F70161937193819391937F010C5FDD
:101250001F4FF5E0C23BDF0709F0ADCFDF91CF9123
:101260001F910F91FF90EF90DF90CF90BF90AF90C4
:101270009F908F907F900895812C912C80E8A82ECC
:101280008FE3B82EC6CF0F931F93CF93DF9350E019
:10129000FC01E40FF51F8081440F551F440F551FBB
:1012A0004B5D564FEA01882329F188819981AA81F3
:1012B000BB81EB01088119812A813B810097A1053F
:1012C000B10569F40C591F4F2F4F3F4FDA010D93B1
:1012D0001D932D933C9313978FEF808306C0081BBB
:1012E000190B2A0B3B0B37FDF7CFDF91CF911F91E5
:1012F0000F910895188219821A821B82F6CF80916D
:101300006B1390916C13891B877019F490E080E047
:10131000089590916813992351F0833030F48FEF42
:10132000890F19F080936813F1CF109268138091A0
:101330006C1328E6829FC00111248E539A4FFC0142
:10134000208120FDE3CF20916C132F5F2770209325
:10135000691330916C1320916A13321304C02091E9
:10136000691320936A13089590916F0081E091FDB5
:1013700002C080E0089590916F009D7F90936F0070
:101380000895CF92DF92EF92FF92FC01C080D1804E
:10139000E280F3802091220D3091230D4091240DA5
:1013A0005091250DC701B6010F9475390F944C4229
:1013B00060939D1370939E1380939F139093A0133B
:1013C000C0928D13D0928E13E0928F13F0929013EF
:1013D00090916B1380916C13981731F0FF90EF9000
:1013E000DF90CF900C941B740E9403880E94B489F4
:1013F00040919D1350919E1360919F137091A01383
:101400004093A9095093AA096093AB097093AC0962
:10141000882331F0FF90EF90DF90CF900C945B2AFF
:10142000FF90EF90DF90CF9008954F925F926F9270
:101430007F928F929F92AF92BF92CF92DF92EF9264
:10144000FF920F931F93CF93DF93EC018B017A01EF
:101450006901F90180819181A281B381FA01408102
:10146000518162817381F80180809180A280B38074
:10147000488059806A807B80409281135092821309
:1014800060928313709284138092851390928613D6
:10149000A0928713B09288134093891350938A13B4
:1014A00060938B1370938C1380938D1390938E1392
:1014B000A0938F13B09390132091220D3091230DA0
:1014C0004091240D5091250DF6016081718182813A
:1014D00093810F9475390F944C424B015C0120911C
:1014E0001E0D30911F0D4091200D5091210DF701DF
:1014F00060817181828193810F9475390F944C4280
:101500006B017C0120911A0D30911B0D40911C0D37
:1015100050911D0DF80160817181828193810F943A
:1015200075390F944C422B013C012091160D3091DE
:10153000170D4091180D5091190D688179818A819C
:101540009B810F9475390F944C4260939113709363
:101550009213809393139093941340929513509207
:1015600096136092971370929813C0929913D09229
:101570009A13E0929B13F0929C1380929D13909289
:101580009E13A0929F13B092A01390916B13809121
:101590006C13981791F0DF91CF911F910F91FF90ED
:1015A000EF90DF90CF90BF90AF909F908F907F9003
:1015B0006F905F904F900C941B740E9403880E9460
:1015C000B4894091991350919A1360919B13709133
:1015D0009C130091951310919613209197133091BD
:1015E0009813C0909113D0909213E0909313F090C1
:1015F0009413C0929D09D0929E09E0929F09F092A7
:10160000A0090093A1091093A2092093A309309384
:10161000A4094093A5095093A6096093A709709364
:10162000A80940919D1350919E1360919F13709152
:10163000A0134093A9095093AA096093AB09709332
:10164000AC09882391F0DF91CF911F910F91FF900A
:10165000EF90DF90CF90BF90AF909F908F907F9052
:101660006F905F904F900C945B2ADF91CF911F9108
:101670000F91FF90EF90DF90CF90BF90AF909F9031
:101680008F907F906F905F904F900895CF92DF92F0
:10169000EF92FF92CF93DF93C82F0E94B48994E01A
:1016A000C99FE0011124FE01E356F64FC080D180AE
:1016B000E280F38081110E945B2ACE5FDD4EC7017C
:1016C000B6010F941639288139814A815B810F94C4
:1016D0007539DF91CF91FF90EF90DF90CF90089513
:1016E000CF92DF92EF92FF92CF93DF93C82F0E94A9
:1016F000B48994E0C99FE0011124FE01EF56F64F32
:10170000C080D180E280F38081110E945B2ACE5F8D
:10171000DD4EC701B6010F941639288139814A81FF
:101720005B810F947539DF91CF91FF90EF90DF903F
:10173000CF9008950E94B48990916C1390936B138D
:1017400090936A139093691394E69093681320ED35
:1017500033E03093BA092093B90981110E945B2AC2
:1017600081E0809390090895CF93DF9324E0829FD6
:10177000C0011124EC01CC54D34FFC01EB51F44FC8
:101780008752944FDC012D913D914D915C91608188
:101790007181828193810F94DF3F688379838A838B
:1017A0009B83DF91CF91089580FF04C09091E5095C
:1017B00090FD8E7F81FF05C09091E509969590FD83
:1017C0008D7F82FF06C09091E5099695969590FDD4
:1017D0008B7F08958F929F92AF92BF92CF92DF92AC
:1017E000EF92FF92CF93DF9320915702222309F4C7
:1017F0009EC0EC018091E509C82ED12CF12CE12C82
:1018000080FF2CC08090590290905A02A0905B02F9
:10181000B0905C02288139814A815B81C501B401A5
:101820000F943F42181624F488829982AA82BB82C0
:101830008090650290906602A0906702B090680266
:10184000288139814A815B81C501B4010F940F3928
:1018500087FF04C088829982AA82BB82D701C60111
:10186000B695A7959795879580FF2CC080905D02CF
:1018700090905E02A0905F02B09060022C813D814A
:101880004E815F81C501B4010F943F42181624F4C4
:101890008C829D82AE82BF828090690290906A02A3
:1018A000A0906B02B0906C022C813D814E815F81D3
:1018B000C501B4010F940F3987FF04C08C829D824B
:1018C000AE82BF8282E0F694E794D794C7948A955B
:1018D000D1F7C0FE2CC0C0906102D0906202E090AF
:1018E0006302F0906402288539854A855B85C701CB
:1018F000B6010F943F42181624F4C886D986EA86AA
:10190000FB86C0906D02D0906E02E0906F02F09066
:101910007002288539854A855B85C701B6010F9419
:101920000F3987FF04C0C886D986EA86FB86DF9117
:10193000CF91FF90EF90DF90CF90BF90AF909F90AE
:101940008F9008952F923F924F925F926F927F9265
:101950008F929F92AF92BF92CF92DF92EF92FF92BF
:101960000F931F93CF93DF93CDB7DEB7A8970FB632
:10197000F894DEBF0FBECDBF8BE49BE00E94EA8BE4
:101980008091CC0B83FD82C020916E0D30916F0D44
:101990004091700D5091710D6091570B7091580BE3
:1019A0008091590B90915A0B0F940F39882309F4A9
:1019B0006DC01091CB0B111165C0809142029091C6
:1019C000430201972091C9123091CA122817390792
:1019D0003CF40E94B5438CE499E10E94962E11E0FC
:1019E00020916E0D30916F0D4091700D5091710DE1
:1019F0006091570B7091580B8091590B90915A0B35
:101A00000F94DE3F6B017C0120E030E0A9010F94D0
:101A10003F4287FF04C0F7FAF094F7F8F094E091A2
:101A2000011224E0E29FF0011124E25EFD4F2081CB
:101A3000318142815381C701B6010F94753920E08D
:101A400030E84BE354E40F943F421816ECF40E9444
:101A5000B5438DE299E10E94962E8091570B9091AB
:101A6000580BA091590BB0915A0B80936E0D909327
:101A70006F0DA093700DB093710D87E59BE00E94F0
:101A8000C18904C010E0ACCF1111E7CF2AE037EDD7
:101A900043E25CE3609153027091540280915502DD
:101AA000909156020F9475396B017C01609171021F
:101AB00070917202072E000C880B990B0F94163947
:101AC0009B01AC01C701B6010F947539698B7A8B04
:101AD0008B8B9C8B8091010D882309F18090B00C39
:101AE0009090B10CA090B20CB090B30CC090530B7E
:101AF000D090540BE090550BF090560B20E030E066
:101B0000A901C501B4010F940F398823E1F1A701A0
:101B10009601C501B4010F943F421816A4F1A12CFF
:101B2000B12C6501E09001128E010F5E1F4F27E579
:101B30003BE043E55BE06FE47BE08BE49BE00E94ED
:101B40005C8880E1EBE4FBE0A2E6BDE001900D9251
:101B50008A95E1F7A8960FB6F894DEBF0FBECDBF09
:101B6000DF91CF911F910F91FF90EF90DF90CF9079
:101B7000BF90AF909F908F907F906F905F904F90AD
:101B80003F902F9008952091620D3091630D409108
:101B9000640D5091650D60914B0B70914C0B8091D1
:101BA0004D0B90914E0B0F94DE3F6D8B7E8B8F8B88
:101BB000988F2091660D3091670D4091680D50917E
:101BC000690D60914F0B7091500B8091510B90916A
:101BD000520B0F94DE3F698F7A8F8B8F9C8F2091F1
:101BE0006A0D30916B0D40916C0D50916D0DC701D8
:101BF000B6010F94DE3F6D8F7E8F8F8F98A320915B
:101C00006E0D30916F0D4091700D5091710D60917E
